:100000000C949A2C0C94E95A0C94BE5A0C94935A62
:100010000C94685A0C943D5A0C94125A0C94E7595B
:100020000C94BC590C94CB2C0C94CB2C0C94CB2C56
:100030000C94CB2C0D947E2A0C94CB2C0C94CB2CB2
:100040000C94CB2C0D94C00D0C94CB2C0C94CB2C7D
:100050000C94CB2C0C94CB2C0C940EFC0C94E15CEB
:100060000C94CB2C0D94A72F0D9444300C94CB2CD6
:100070000C94CB2C0C94CB2C0C94CB2C0C94CB2C24
:100080000C94CB2C0C94CB2C0C94CB2C0C94CB2C14
:100090000C94CB2C0C94CB2C0C94CB2C0C94CB2C04
:1000A0000C94CB2C0C94CB2C0C94CB2C0C94CB2CF4
:1000B0000C94CB2C0C94CB2C0C94CB2C0C94CB2CE4
:1000C0000C94CB2C0C94CB2C0C94CB2C0C94CB2CD4
:1000D0000C94CB2C0C94CB2C0C94CB2C0C94CB2CC4
:1000E0000C94CB2C90549354825486548C54CA5400
:1000F00097549B54A154A554A954AF54B354B75426
:10010000CA54BD54C154C554CE5BD35BD85BE25BCB
:10011000EC5B655CF65BFE5B065C105C1A5C245C69
:10012000335C3D5C655C475C515C5B5CF875F87505
:10013000FF75FF75FF7506760676067613760D76E3
:100140000D760D761601DC00D800120110010401B5
:100150000A0104010001E6000401DE00084AD73B61
:100160003BCE016E84BCBFFDC12F3D6C74319ABD86
:1001700056833DDA3D00C77F11BED9E4BB4C3E91AA
:100180006BAAAABE000000803F05A84CCDB2D44E99
:10019000B93836A9020C50B9918688083CA6AAAA9B
:1001A0002ABE000000803F000D941C190D94BF066C
:1001B0000D94F42F0D94F30B0D94E32F0D9419303F
:1001C0000D94C0070D9451080D94C8010D9413307F
:1001D0000D942F070D94950A0D941B030D9464291B
:1001E0000D94040A0D9426190D94260B0D942B16CC
:1001F0000D94DC040D942D160D94691A0D94730959
:100200000D940F300D9428160D941C300D949428E5
:100210000D94E2080D940B300D94CF170D941D2B07
:100220000D9407300D94FF2F0D94EA1C0D94DD2FD3
:100230004E414E494E495459494E46CDCCCC3D0ACB
:10024000D7233C17B7D13877CC2B329595E6241FAE
:10025000B14F0A000020410000C84200401C462067
:10026000BCBE4CCA1B0E5AAEC59D74434F4D4D5576
:100270004E49434154494F4E0044525952554E0045
:100280004552524F525300494E464F004543484F46
:100290000020746F6F206C6F6E67206578747275C4
:1002A00073696F6E2070726576656E7465640A009E
:1002B00020636F6C6420657874727573696F6E204B
:1002C00070726576656E7465640A0047322F473335
:1002D0002062616420706172616D65746572730A79
:1002E00000205A3A200020593A20004265642058E4
:1002F0003A20004E6F206D6F76652E00456E6420AB
:1003000066696C65206C6973740A00426567696E82
:100310002066696C65206C6973740A004D31323552
:10032000005344207072696E74696E67206279743C
:100330006520004E6F74205344207072696E74699A
:100340006E670A0046696C652064656C6574656457
:100350003A0044656C6574696F6E206661696C650E
:10036000642C2046696C653A20006F70656E2066CB
:1003700061696C65642C2046696C653A2000507296
:10038000696E742074696D653A2000000125311D85
:1003900040FF24301CFF45232F1B0A07FFFF0408E2
:1003A00006FF06222B1AFFFF043803FF36FFFFFF6C
:1003B000FFFFFF50726F7465637465642050696E4F
:1003C0000A006D0046696C616D656E742075736519
:1003D000643A200053746174733A20002C204C6FEF
:1003E0006E67657374206A6F623A2000546F74619F
:1003F0006C2074696D653A200053746174733A20FF
:10040000002C204661696C65643A20002C20466906
:100410006E69736865643A20005072696E74733A4D
:10042000200053746174733A2000457874727564C7
:100430006572202573004C756C7A426F74204D698B
:100440006E692032204C43442072656164792E002D
:100450008C028702800279026B026F666600444557
:100460004255473A006F6B004361703A454D455223
:1004700047454E43595F5041525345523A310A0065
:100480004361703A434153455F4C494748545F428A
:1004900052494748544E4553533A300A004361701D
:1004A0003A544F47474C455F4C49474854533A30BC
:1004B0000A004361703A534F4654574152455F50CA
:1004C0004F5745523A300A004361703A4C45564501
:1004D0004C494E475F444154413A310A00436170F0
:1004E0003A5A5F50524F42453A310A004361703ADE
:1004F0004155544F4C4556454C3A310A00436170C2
:100500003A5052494E545F4A4F423A310A004361D1
:10051000703A50524F47524553533A300A004361A4
:10052000703A4155544F5245504F52545F54454DC7
:10053000503A310A004361703A454550524F4D3AA6
:10054000310A004649524D574152455F4E414D4593
:100550003A4D61726C696E20204649524D574152A6
:10056000455F56455253494F4E3A312E312E352E66
:1005700037312045585452554445525F54595045DF
:100580003A4165726F7374727564657220534F558A
:100590005243455F434F44455F55524C3A6874742B
:1005A00070733A2F2F636F64652E616C6570686F8E
:1005B000626A656374732E636F6D2F646966667516
:1005C00073696F6E2F4D41524C494E2050524F541B
:1005D0004F434F4C5F56455253494F4E3A312E30A0
:1005E000204D414348494E455F545950453A4C755A
:1005F0006C7A426F74204D696E692032204C4344FE
:100600002045585452554445525F434F554E543A35
:100610003120555549443A65353530323431312D24
:10062000643436642D343231642D626133612D615E
:1006300032303132366437393330660A0020643A5A
:100640000020693A0020703A0020643A0020693A9C
:100650000020703A0043290A0061626C656420281A
:100660006D696E2074656D702000436F6C64206549
:10067000787472756465732061726520004B642024
:100680000023646566696E65202044454641554CEB
:10069000545F004B69200023646566696E65202005
:1006A00044454641554C545F004B7020002364651F
:1006B00066696E65202044454641554C545F0050A4
:1006C0004944204175746F74756E652066696E6962
:1006D00073686564212050757420746865206C61AE
:1006E0007374204B702C204B6920616E64204B6426
:1006F00020636F6E7374616E74732066726F6D2009
:1007000062656C6F7720696E746F20436F6E6669E7
:100710006775726174696F6E2E680A0050494420D3
:100720004175746F74756E65206661696C656421CE
:100730002074696D656F75740A00504944204175D5
:10074000746F74756E65206661696C6564212054F0
:10075000656D706572617475726520746F6F206865
:100760006967680A00204B643A2000204B693A20F0
:1007700000204B703A20000A20436C617373696358
:1007800020504944200A002054753A2000204B751F
:100790003A2000206D61783A2000206D696E3A2081
:1007A0000020643A200020626961733A20004265AB
:1007B00064204C6576656C696E6720004661696CE3
:1007C000656420746F20656E61626C6520426564AB
:1007D000204C6576656C696E670A00426564204C42
:1007E0006576656C20436F7272656374696F6E2005
:1007F0004D61747269783A004F6666736574732050
:100800006170706C696564004572723A20546F6F54
:10081000206661722100546F6F20666172206672DB
:100820006F6D207265666572656E636520706F69B5
:100830006E740A003A20007A5F6D696E3A20202DAE
:1008400032207A5F6D61783A202035005A204F6659
:100850006673657420004163746976652045787419
:1008600072756465723A2000556E6B6E6F776E20FC
:10087000636F6D6D616E643A202200206673616360
:100880007469766500206F7400206F7470770020A3
:100890007332676100207332676200206F6C610001
:1008A000206F6C62002073740020656E00207473EA
:1008B0007465705F6176673A002063736163743AB0
:1008C00000206176675F73673A00207367743A00AF
:1008D00020737465616C746800207673656E3A00ED
:1008E0002F00206968723A002045303A0020667374
:1008F00061637469766500206F7400206F7470778F
:1009000000207332676100207332676200206F6CD1
:100910006100206F6C62002073740020656E0020FF
:1009200074737465705F6176673A00206373616306
:10093000743A00206176675F73673A0020736774CA
:100940003A0020737465616C746800207673656E7C
:100950003A002F00206968723A00205A3A00206657
:100960007361637469766500206F7400206F747022
:100970007700207332676100207332676200206F56
:100980006C6100206F6C62002073740020656E0043
:100990002074737465705F6176673A0020637361D9
:1009A00063743A00206176675F73673A002073676B
:1009B000743A0020737465616C7468002076736506
:1009C0006E3A002F00206968723A0020593A0020E0
:1009D000667361637469766500206F7400206F74BC
:1009E00070770020733267610020733267620020E5
:1009F0006F6C6100206F6C62002073740020656E64
:100A0000002074737465705F6176673A00206373C9
:100A10006163743A00206176675F73673A00207300
:100A200067743A0020737465616C74680020767393
:100A3000656E3A002F00206968723A0020583A002B
:100A4000544D4332313330205374617475733A0A14
:100A5000007A5F6D61783A20007A5F6D696E3A20A6
:100A600000795F6D61783A2000785F6D696E3A2099
:100A7000005265706F7274696E6720656E6473747E
:100A80006F70207374617475730A00000020002376
:100A900000260029002C002F003200000100000376
:100AA00001060109012569730025696D2025697317
:100AB000002569682025696D202569730025696412
:100AC000202569682025696D2025697300256979CD
:100AD00020256964202569682025696D20256973B2
:100AE0000025753A2530327500253032753A2530AB
:100AF00032750025756420253032753A25303275FF
:100B0000001FFFFFFFFFFFFF600000000001FF402C
:100B10000000000000FF8000000000007F83CF0085
:100B2000000C303F87FF80000C301F867980000C5E
:100B3000000F8C30C7838C30E78C30CFC7CC31F3BB
:100B40008C30DCECEC33B98C30D86C6C33198C30D5
:100B5000D06C0C33198C30D86C0C33198C30DC6CA5
:100B60000E3B198C30CF7C079F198C30C77C038FCC
:100B70001940000000000002600000000000061F95
:100B8000FFFFFFFFFFF82020506C616E6E65724220
:100B9000756666657242797465733A200020467204
:100BA0006565204D656D6F72793A2000436F6D70F9
:100BB000696C65643A204A616E20323220323031ED
:100BC000380A00207C20417574686F723A202841F1
:100BD0006C657068204F626A6563747320496E6348
:100BE0002E2C204C756C7A426F7420476974205209
:100BF00065706F7369746F7279290A004A616E209B
:100C00003232203230313830393A31363A343000ED
:100C1000204C61737420557064617465643A2000DF
:100C2000312E312E350A004D61726C696E002053F1
:100C30006F6674776172652052657365740A00206F
:100C40005761746368646F672052657365740A0046
:100C50002042726F776E206F7574205265736574D1
:100C60000A002045787465726E616C205265736568
:100C7000740A00506F77657255700A007374617260
:100C8000740A006572726F722077726974696E6798
:100C900020746F2066696C650A00456E6473746F1A
:100CA00070732025632025632025632025630020A1
:100CB0005A3A0020593A0020583A00656E6473741D
:100CC0006F7073206869743A2000446F6E652073FA
:100CD0006176696E672066696C652E0A004D32394F
:100CE000004D6F76652059004D6F7665205A00459E
:100CF00078747275646572004D6F766520302E31A0
:100D00006D6D004D6F766520316D6D004D6F7665B0
:100D10002031306D6D004D6F76652061786973000C
:100D20004578747275646572004D6F7665205A005F
:100D30004D6F76652059004D6F76652058004578D7
:100D4000747275646572004D6F7665205A004D6F40
:100D500076652059004D6F76652058004D6F766599
:100D60006D656E7400436F6F6C646F776E004661E3
:100D70006E2073706565640046616E2073706565F2
:100D8000640042656400426564004E6F7A7A6C6567
:100D9000004E6F7A7A6C65004D61696E0056547230
:100DA0006176206D696E005654726176206D696EB1
:100DB000005654726176206D696E00566D696E0042
:100DC000566D696E00566D696E00566D61782045EE
:100DD00000566D6178204500566D617820450056BB
:100DE0006D6178205A00566D6178205A00566D6109
:100DF00078205A00566D6178205900566D61782030
:100E00005900566D6178205900566D617820580060
:100E1000566D6178205800566D61782058004D6FEE
:100E200074696F6E00416D6178204500416D617895
:100E3000204500416D6178205A00416D6178205A4B
:100E400000416D6178205900416D61782059004161
:100E50006D6178205800416D6178205800412D74F3
:100E6000726176656C00412D74726176656C00412B
:100E70002D7265747261637400412D7265747261C4
:100E8000637400416363656C00416363656C004D8E
:100E90006F74696F6E0000060900FE00000000001C
:100EA00001090008FE000005080806000040F0C81F
:100EB0008888987810050808060000C0F888888897
:100EC0008888F80505050600012030F8302005085F
:100ED000080600002070F820202020E005090906FF
:100EE00000FF2070A8A8B8888870200509090600AE
:100EF000FFE080C0B0A8283028280509090600FFB7
:100F0000F8A88888888888A8F8050A0A0600FE20BC
:100F10005050505088A8A88870030303060003406F
:100F2000A04000060900FE070192032120FFFF08F0
:100F3000FF07FF000000060000010707060200800F
:100F4000808080800080030202060105A0A00507C2
:100F5000070600005050F850F850500507070600EB
:100F6000002078A07028F020050707060000C0C800
:100F700010204098180507070600006090A040A8C0
:100F80009068020303060104C040800307070601BE
:100F90000020408080804020030707060100804039
:100FA000202020408005050506000120A870A8200B
:100FB0000505050600012020F82020020303060293
:100FC000FFC04080050101060003F802020206028C
:100FD00000C0C00505050600010810204080050777
:100FE0000706000070888888888870030707060154
:100FF0000040C040404040E0050707060000708800
:1010000008708080F8050707060000F81020100817
:1010100008F005070706000010305090F810100582
:101020000707060000F880F0080888700507070623
:101030000000708080F0888870050707060000F8BF
:1010400008102020202005070706000070888870FF
:10105000888870050707060000708888780808707F
:10106000020505060200C0C000C0C0020606060256
:10107000FFC0C000C04080040707060000102040E9
:1010800080402010050303060002F800F80407075B
:101090000601008040201020408005070706000060
:1010A00070880810200020050707060000708808D7
:1010B00068A8A870050707060000708888F8888867
:1010C00088050707060000F08888F08888F0050783
:1010D000070600007088808080887005070706007A
:1010E00000F08888888888F0050707060000F880E7
:1010F00080F08080F8050707060000F88080F08007
:101100008080050707060000708880B88888700511
:101110000707060000888888F8888888010707067E
:1011200002008080808080808005070706000038EC
:101130001010101090600507070600008890A0C0EE
:10114000A09088050707060000808080808080F8D6
:1011500005070706000088D8A8888888880507073B
:101160000600008888C8A898888805070706000038
:1011700070888888888870050707060000F08888CE
:10118000F080808005070706000070888888A89096
:1011900068050707060000F08888F0A0908805071A
:1011A00007060000788080700808F0050707060031
:1011B00000F820202020202005070706000088884E
:1011C00088888888700507070600008888888888CE
:1011D00050200507070600008888888888A85005E1
:1011E00007070600008888502050888805070706F2
:1011F000000088888850202020050707060000F896
:101200000810204080F8030707060100E080808076
:101210008080E005050506000180402010080307D6
:1012200007060100E02020202020E005030306003F
:1012300004205088050101060000F802020206029F
:1012400005804005050506000070087888780507C8
:10125000070600008080B0C88888F00505050600F4
:1012600000708080887005070706000008086898ED
:101270008888780505050600007088F880700507E5
:10128000070600003048E0404040400506060600E2
:10129000FF7088887808700507070600008080B016
:1012A000C888888801070706020080008080808047
:1012B000800308080601FF200020202020A0400411
:1012C0000707060000808090A0C0A09003070706D3
:1012D0000100C04040404040E0050505060000D048
:1012E000A8A8A8A8050505060000B0C88888880534
:1012F000050506000070888888700506060600FF50
:10130000F08888F080800506060600FF78888878D7
:101310000808050505060000B0C8808080050505A1
:1013200006000070807008F00407070600004040C7
:10133000E040404030050505060000888888986830
:10134000050505060000888888502005050506006B
:10135000008888A8A8500505050600008850205080
:10136000880506060600FF88888878087005050548
:10137000060000F8102040F803070706010020408F
:101380004080404020010707060200808080808066
:101390008080030707060100804040204040800510
:1013A0000202060002689000000006000000000033
:1013B000060000000000060000000000060000001B
:1013C000000006000000000006000000000006000B
:1013D0000000000006000000000006000000000001
:1013E00006000000000006000000000006000000EB
:1013F00000000600000000000600000000000600DB
:1014000000000000060000000000060000000000D0
:1014100006000000000006000000000006000000BA
:1014200000000600000000000600000000000600AA
:1014300000000000060000000000060000000000A0
:10144000060000000000060000000000060000008A
:10145000000006000000000006000000000006007A
:101460000000000006000000000006000000000070
:10147000060000010707060200800080808080804F
:101480000507070600002070A8A0A8702005070720
:10149000060000304040E04050A805050506000069
:1014A0008870507088050707060000885020F820D3
:1014B000F8200107070602008080800080808005F8
:1014C00008080600003048205050209060030101B9
:1014D000060107A0050707060000F888B8B8B88815
:1014E000F8050707060001700878887800F80505F8
:1014F000050600012850A05028050303060001F846
:1015000008080202020602064080050707060000DE
:10151000F888A88898A8F8050101060006F80404D0
:101520000406000360909060050707060000202075
:10153000F8202000F804050506000360902040F024
:10154000030505060003E020E020E0020202060297
:101550000640800508080600FF8888888898E8808B
:101560008005070706000078989878181818020276
:1015700002060202C0C00202020602FF408003050A
:101580000506000340C04040E00507070600017063
:101590008888887000F8050505060001A0502850CD
:1015A000A00507070600008890A858B80808050796
:1015B000070600008890B8489820380508080600FB
:1015C00000C040C048D838080805070706000020BA
:1015D0000020408088700508080600004020007048
:1015E00088F888880508080600001020007088F830
:1015F00088880508080600002050007088F8888850
:101600000508080600006890007088F888880508BA
:10161000080600005000708888F8888805080806C9
:1016200000002050207088F8888805070706000011
:101630003860A0B8E0A0B80508080600FF708880F0
:101640008088702060050808060000402000F880AF
:10165000F080F8050808060000081000F880F08007
:10166000F8050808060000205000F880F080F80512
:1016700007070600005000F880F080F8030808060D
:101680000100804000E0404040E0030808060100FF
:10169000204000E0404040E003080806010040A070
:1016A00000E0404040E0030707060100A000E040E2
:1016B0004040E0050707060000704848E8484870C9
:1016C00005080806000068900088C8A898880508E2
:1016D0000806000040207088888888700508080681
:1016E00000001020708888888870050808060000AF
:1016F00020500070888888700508080600006890EF
:1017000000708888887005080806000050007088FE
:1017100088888870050505060001885020508805D6
:1017200008080600FF1070A8A8A8A87040050808BF
:101730000600004020888888888870050808060010
:101740000010208888888888700508080600002016
:1017500050008888888870050808060000500088B6
:1017600088888888700508080600001020885020A6
:101770002020200509090600FFC04070484870403D
:1017800040E00408080601FF609090A09090E0807F
:1017900005080806000040200070087888780508D1
:1017A00008060000102000700878887805080806F0
:1017B00000002050007008788878050808060000AE
:1017C00068900070087888780507070600005000C8
:1017D00070087888780508080600002050207008F6
:1017E000788878050606060000D02878A0A850055D
:1017F00006060600FF708088702060050808060055
:10180000004020007088F88070050808060000106D
:1018100020007088F880700508080600002050003D
:101820007088F8807005070706000050007088F87F
:10183000807003080806010080400040C04040E07E
:1018400003080806010020400040C04040E00308B3
:101850000806010040A00040C04040E00307070622
:101860000100A00040C04040E0050707060000A0BE
:1018700040A010788870050808060000689000B045
:10188000C8888888050808060000402000708888FD
:10189000887005080806000010200070888888708D
:1018A0000508080600002050007088888870050828
:1018B0000806000068900070888888700507070691
:1018C000000050007088888870050505060001201A
:1018D00000F800200507070600FF1070A8A8A870F0
:1018E00040050808060000402000888888986805A0
:1018F00008080600001020008888889868050808F5
:1019000006000020500088888898680507070600B0
:1019100000500088888898680509090600FF102093
:1019200000888888F808700407070601FFC0406037
:10193000506040E00508080600FF5000888888785D
:1019400008705A00590058000920000000000000EB
:10195000000000000000007FFFE000000000000029
:101960000000000000007000E00000000000000027
:10197000000000000061F8600000000000000000AE
:101980000000000041F820000000000000000000FE
:1019900000000040F02000000000000000000000F7
:1019A0000000406020000000000000000000000077
:1019B000005801A07F8000000000000000410400EA
:1019C0005C63A0FFC0000000000000002082005EF9
:1019D000F7A0FFC0000000000000002082005EF7BA
:1019E000A0FFC0000000000000004104005C63A0F4
:1019F0007F80000000000000008208005801A07FE6
:101A00008000000000000001041000406020FFC0C2
:101A10000000000000000104100040F020FFC000A2
:101A200000000000000082080041F820FFC0000014
:101A3000000000000041040061F8603F0000000069
:101A4000000000000000007000E01E000000000028
:101A5000000001FFFF807FFFE00C0000000000009D
:101A60000001FFFF800000000000000000000000F7
:101A7000000000007FFFE000000000000000000008
:101A80000000007000E00000000000000000000006
:101A90000000630C60000000000000000000000077
:101AA00000470E20000000000000000000000000C1
:101AB0004F0F200000000000000000000000005F49
:101AC0000FA00000000000000000000000005E0702
:101AD000A07F800000000000000041040040602062
:101AE000FFC00000000000000020820040F020FF46
:101AF000C00000000000000020820040F020FFC075
:101B0000000000000000004104004060207F8000D1
:101B10000000000000008208005E07A07F80000037
:101B200000000000010410005F0FA0FFC0000000D3
:101B3000000000010410004F0F20FFC00000000053
:101B4000000000820800470E20FFC00000000000D7
:101B50000000410400630C603F0000000000000032
:101B6000000000007000E01E000000000000000106
:101B7000FFFF807FFFE00C0000000000000001FF7D
:101B8000FF800000005265776970696E67005072CF
:101B90006F62696E67206661696C65640050726F80
:101BA00062696E67206661696C65640050524F42DD
:101BB00045204641494C20434C45414E204E4F5A0A
:101BC0005A4C450A005265776970696E670A00527F
:101BD00065776970696E670050726F62696E672021
:101BE0006661696C65640050726F62696E67206639
:101BF00061696C65640050524F4245204641494C32
:101C000020434C45414E204E4F5A5A4C450A0052F3
:101C100065776970696E670A0050726F62696E67F6
:101C2000206661696C65640A0050726F62696E6754
:101C3000206661696C656400205A3A200020593A98
:101C4000200042656420583A200000000A0B020977
:101C50000C0D0E0807030401000000000000000046
:101C60000000000000000000000000000000000074
:101C70000000000000001211100000000000000031
:101C80000000000000000000000000000000000054
:101C9000486F6D65202573257325732066697273FF
:101CA00074002066697273740A005A005900580063
:101CB000486F6D652000536C6565702E2E2E0020D8
:101CC000706F736974696F6E206F7574206F662012
:101CD00072616E67652E0A003F50726F6265200068
:101CE0000A0A426564204C6576656C20436F727207
:101CF000656374696F6E204D61747269783A002073
:101D00002B000A436F7272656374656420426564D8
:101D1000204865696768742076732E2042656420C8
:101D2000546F706F6C6F67793A0A00202B000A427B
:101D300065642048656967687420546F706F6772C6
:101D4000617068793A0A2020202B2D2D2D204241E8
:101D5000434B202D2D2B0A2020207C2020202020CA
:101D60002020202020207C0A204C207C20202020A5
:101D7000282B29202020207C20520A2045207C204E
:101D8000202020202020202020207C20490A2046BE
:101D9000207C20282D29204E20282B29207C2047FC
:101DA0000A2054207C2020202020202020202020B9
:101DB0007C20480A2020207C20202020282D29203B
:101DC0002020207C20540A2020207C20202020203D
:101DD0002020202020207C0A2020204F2D2D20464E
:101DE000524F4E54202D2D2B0A2028302C30290AFA
:101DF000004D65616E206F662073616D706C656467
:101E000020706F696E74733A200020643A200020BD
:101E1000623A200045716E20636F6566666963698A
:101E2000656E74733A20613A200052756E6E696E69
:101E30006720696E204452592D52554E206D6F64B3
:101E4000650A00473239204175746F20426564206D
:101E50004C6576656C696E670A0028422961636B80
:101E600000284629726F6E740028522969676874C9
:101E700000284C29656674003F4E756D62657220BE
:101E80006F662070726F626520706F696E74732068
:101E9000697320696D706C61757369626C65202867
:101EA00032206D696E696D756D292E0A003F2856C6
:101EB000296572626F7365206C6576656C20697345
:101EC00020696D706C61757369626C652028302DB6
:101ED00034292E0A004C756C7A426F74204D696E5D
:101EE000692032204C43442072656164792E00528F
:101EF0006573756D696E67207072696E7400436CEE
:101F000069636B20746F20726573756D652E2E2E5C
:101F1000002F2F200053657474696E67205472611E
:101F200076656C20416363656C65726174696F6E80
:101F30003A200053657474696E672052657472614B
:101F4000637420416363656C65726174696F6E3A96
:101F5000200053657474696E67205072696E742036
:101F6000416363656C65726174696F6E3A200053FA
:101F7000657474696E67205072696E7420616E6456
:101F80002054726176656C20416363656C65726193
:101F900074696F6E3A2000205A00205900580020C2
:101FA000204D61783A2000205A0020590058002026
:101FB000204D696E3A20004F6E20004F6666005338
:101FC0006F667420656E6473746F70733A200020BE
:101FD00061786973206472697665722063757272C4
:101FE000656E743A2000747275650066616C736585
:101FF0000020617869732074656D70657261747515
:102000007265207072657761726E2074726967679D
:10201000657265643A2000207072657761726E2087
:10202000666C616720636C65617265640A00207389
:102030007465616C746843686F70206D617820739B
:10204000706565642073657420746F20002064726D
:102050006976657220686F6D696E672073656E734F
:10206000697469766974792073657420746F2000CF
:102070004E6F2063617365206C696768740A0000A5
:10208000002100240027002A002D00300033000129
:10209000010000040107010A0153442063617264D6
:1020A000206F6B0A006F70656E526F6F74206661EF
:1020B000696C65640A00766F6C756D652E696E6972
:1020C00074206661696C65640A00534420696E6916
:1020D00074206661696C0A006175746F25692E67EA
:1020E000004D3234004D323320257300577269742D
:1020F000696E6720746F2066696C653A20006F70A6
:10210000656E206661696C65642C2046696C653A71
:1021100020006F70656E206661696C65642C2046D6
:10212000696C653A200046696C652073656C65636F
:102130007465640A002053697A653A200046696C28
:1021400065206F70656E65643A20006F70656E2063
:102150006661696C65642C2046696C653A200020D4
:1021600066696C653A20004E6F7720002220706F00
:1021700073002220706172656E743A2200535542DA
:10218000524F5554494E452043414C4C2074617286
:102190006765743A22004B494C4C45442E2000742C
:1021A0007279696E6720746F2063616C6C2073753F
:1021B000622D67636F64652066696C65732077695B
:1021C000746820746F6F206D616E79206C65766520
:1021D0006C732E204D4158206C6576656C206973B8
:1021E0003A004572726F723A0043616E6E6F7420EE
:1021F0006F70656E20737562646972200065636834
:102200006F3A00544845524D414C2052554E41576B
:1022100041592042454400546865726D616C2052FA
:10222000756E6177617900544845524D414C20529A
:10223000554E4157415920453100544845524D4172
:102240004C2052554E41574159204530004E6F2089
:102250004C696E65204E756D626572207769746891
:1022600020636865636B73756D2C204C61737420FB
:102270004C696E653A200053544F505045442E200F
:10228000005072696E7465722073746F707065644B
:102290002064756520746F206572726F72732E20D2
:1022A00046697820746865206572726F7220616E6D
:1022B0006420757365204D39393920746F2072653B
:1022C00073746172742E202854656D706572617428
:1022D0007572652069732072657365742E2053656D
:1022E000742069742061667465722072657374610C
:1022F0007274696E67290A004E6F20436865636BCC
:1023000073756D2077697468206C696E65206E75D1
:102310006D6265722C204C617374204C696E653A55
:102320002000636865636B73756D206D69736D6103
:102330007463682C204C617374204C696E653A207C
:10234000004C696E65204E756D6265722069732060
:102350006E6F74204C617374204C696E65204E75ED
:102360006D6265722B312C204C617374204C696E48
:10237000653A20004D313130004D3331004D383455
:1023800020582059205A204500534420726561642A
:10239000206572726F720A004D3000436F6D706C71
:1023A0006574656400446F6E65207072696E74694F
:1023B0006E672066696C650A0020496E76616C69FB
:1023C000642065787472756465722000000040C0F6
:1023D0000000E0C0000000000000224300003E4377
:1023E00000003743202F002042403A0020403A00AE
:1023F00048656174696E6720646F6E652E00436F77
:102400006F6C696E6720646F6E652E0020573A000E
:102410004578747275646572202573004C756C7A0A
:10242000426F74204D696E692032204C4344207203
:10243000656164792E0042656420646F6E652E00CC
:1024400020573A004265642068656174696E672EA2
:102450000042656420636F6F6C696E672E004D31BA
:10246000343520533C696E6465783E206F75742066
:102470006F662072616E67652028302D31290A0051
:102480004C756C7A426F74204D696E692032204C15
:102490004344204F66662E00205A3A0020593A00E5
:1024A00020436F756E7420583A0020453A00205A38
:1024B0003A0020593A00583A0020746F6F206C6F30
:1024C0006E6720657874727573696F6E20707265BF
:1024D00076656E7465640A0020636F6C64206578AD
:1024E00074727573696F6E2070726576656E74654F
:1024F000640A007C3C3E5E2B3D3F2F5B5D3B2C2AFB
:10250000225C00010210202008081020401020400A
:1025100080020102010804020101020408102040A7
:1025200080804020100804020180040201804020C5
:1025300010080402010804020101020408102040EE
:10254000800102040810204080000022002500289D
:10255000002B002E003100340002010000050108AC
:10256000010B010505050507050808080802020218
:10257000020A0A080804040404010101010101011E
:10258000010303030303030303040707070C0C0CF5
:102590000C0C0C0C0C0202020206060606060606CD
:1025A000060B0B0B0B0B0B0B0B290A00206279742B
:1025B00065733B20637263200053657474696E67B2
:1025C000732053746F726564202800202863616C47
:1025D00063756C6174656429210A0020213D200027
:1025E000454550524F4D20435243206D69736D61F4
:1025F000746368202D202873746F7265642920002D
:10260000290A002062797465733B2063726320009D
:102610002073746F7265642073657474696E677378
:1026200020726574726965766564202800204D61AA
:10263000726C696E3D563430290A00284545505267
:102640004F4D3D00454550524F4D207665727369A0
:102650006F6E206D69736D617463682000436172F1
:10266000642072656D6F76656400436172642069F1
:102670006E7365727465640000060900FE060189C8
:1026800002FE20FFFE07FE06FE0000000600070116
:102690000606060200808080800080030303060196
:1026A00003A0A0A00507070600FF5050F850F850FF
:1026B000500509090600FE2070A8A07028A8702007
:1026C0000608080600FF40A84810204854080507DF
:1026D000070600FF6090906098906801030306026F
:1026E000038080800207070602FF40808080808090
:1026F000400207070602FF80404040404080050539
:10270000050600008850F8508805050506000020E1
:1027100020F820200204040602FEC040408005018B
:1027200001060002F8020202060200C0C00406060A
:10273000060100101020408080040606060100609B
:10274000909090906003060606010040C040404013
:10275000E00406060601006090102040F004060622
:10276000060100F020601010E005060606000010CB
:10277000305090F810040606060100F080E01010BA
:10278000E00406060601006080E090906004060602
:10279000060100F01010204040040606060100600B
:1027A00090609090600406060601006090907010A2
:1027B00060020505060200C0C000C0C0020707068F
:1027C00002FEC0C000C0404080050505060000189C
:1027D00060806018050303060001F800F805050590
:1027E000060000C0300830C00407070601006090F2
:1027F00010604000400506060600007090A8B080FA
:1028000070050606060000205088F8888805060630
:10281000060000F088F08888F004060606010060D3
:102820009080809060040606060100E090909090F1
:10283000E0040606060100F080E08080F004060651
:10284000060100F080E0808080040606060100603A
:102850009080B090600406060601009090F0909081
:1028600090030606060100E040404040E0050606F1
:102870000600003810101090600406060601009053
:10288000A0C0A09090040606060100808080808091
:10289000F005060606000088D8A8A8888804060661
:1028A00006010090D0B090909005060606000070DA
:1028B0008888888870040606060100E09090E08011
:1028C000800407070601FF609090D0B060100406F6
:1028D00006060100E09090E09090040606060100D4
:1028E000609040209060050606060000F820202039
:1028F0002020040606060100909090909060040647
:1029000006060100909090F0606005060606000043
:102910008888A8A8D88805060606000088502020C8
:1029200050880506060600008888502020200406EE
:1029300006060100F010204080F0030606060100A4
:10294000E080808080E00406060601008080402050
:102950001010030606060100E020202020E00503F9
:10296000030600032050880501010600FEF802025C
:102970000206020480400404040601007090907076
:102980000406060601008080E09090E0040404063E
:10299000010070808070040606060100101070901F
:1029A000907004040406010060B0C07004060606BE
:1029B0000100205040E040400406060601FE609001
:1029C000907010600406060601008080E0909090F0
:1029D0000306060601004000C04040E00308080668
:1029E00001FE200060202020A04004060606010011
:1029F0008080A0C0A090030606060100C0404040B1
:102A000040E0050404060000D0A8A88804040406D9
:102A10000100E09090900404040601006090906032
:102A20000406060601FEE09090E08080040606069B
:102A300001FE709090701010040404060100A0D0F4
:102A4000808004040406010070C030E0040606061D
:102A500001004040E0405020040404060100909032
:102A60009070040404060100909060600504040660
:102A7000000088A8A850040404060100906060903B
:102A80000406060601FE909090709060040404060F
:102A90000100F02040F003070706010020404080BD
:102AA0004040200107070602FF80808080808080F0
:102AB00003070706010080404020404080040202D6
:102AC00006010350A0FFFFFFFFFFFFFFFFFFFFFF17
:102AD000FFFFFFFFFFFFFFFFFFFFFFFFFFFFFFFF06
:102AE000FFFFFFFFFFFF00000006000701060606CC
:102AF00002008000808080800406060601FF2070AE
:102B0000A0A070200507070600FF304840F04040B5
:102B1000F8050505060000A8508850A80506060619
:102B200000008850F820F8200107070602FF808087
:102B300080008080800407070601FF70806090603D
:102B400010E0030101060105A00607070600007852
:102B50008494A494847803050506010160A06000B4
:102B6000E00505050600002850A0502804030306D0
:102B70000100F01010040101060102F0060707062B
:102B800000007884B4A4A48478040101060105F04F
:102B90000403030601026090600507070600FF209A
:102BA00020F8202000F803050506010140A0204080
:102BB000E0030505060101C0204020C00202020614
:102BC000020440800405050601FF9090B0D0800506
:102BD000060606000078E8E86828280101010602D8
:102BE00002800202020602FE408003050506010182
:102BF00040C04040E003050506010140A04000E060
:102C0000050505060000A0502850A005080806008C
:102C1000FF40C04050703078100508080600FF40A3
:102C2000C04050680810380508080600FFC0204062
:102C300030F0307810040707060100200020608083
:102C40009060050707060000402020507088880526
:102C50000707060000102020507088880507070627
:102C600000002050205070888805070706000028C3
:102C7000502050708888050707060000500020503B
:102C8000708888050707060000205020507088884B
:102C900005060606000078A0F0A0A0B80408080603
:102CA00001FE6090808090602040040707060100CC
:102CB0004020F080E080F00407070601002040F08B
:102CC00080E080F00407070601002050F080E080DB
:102CD000F00407070601005000F080E080F00307D1
:102CE000070601008040E0404040E003070706017E
:102CF000002040E0404040E003070706010040A0FC
:102D0000E0404040E0030707060100A000E040402B
:102D100040E00506060600007048E84848700407D1
:102D20000706010050A090D0B0909004070706015C
:102D3000004020609090906004070706010020404A
:102D4000609090906004070706010020506090900A
:102D5000906004070706010050A060909090600406
:102D60000707060100500060909090600505050679
:102D7000000088502050880408080601FF1070B039
:102D8000B0D0D0E08004070706010040209090906A
:102D90009060040707060100204090909090600426
:102DA00007070601002050909090906004070706E6
:102DB00001005000909090906005070706000010F9
:102DC00020885020202004060606010080E0909014
:102DD000E0800406060601006090A0A090A0040711
:102DE000070601004020007090907004070706015C
:102DF00000204000709090700407070601002050EA
:102E0000007090907004070706010050A0007090B9
:102E10009070040606060100500070909070040740
:102E200007060100205020709090700504040600F1
:102E30000070A8B0780406060601FE70808070203D
:102E40004004070706010040200060B0C07004077E
:102E50000706010020400060B0C0700407070601AB
:102E60000020500060B0C07004060606010050004B
:102E700060B0C070030707060100804000C04040FA
:102E8000E0030707060100204000C04040E00307C0
:102E90000706010040A000C04040E003060606010E
:102EA00000A000C04040E0040707060100306010A9
:102EB0007090906004070706010050A000E0909019
:102EC000900407070601004020006090906004070E
:102ED000070601002040006090906004070706018B
:102EE000002050006090906004070706010050A089
:102EF000006090906004060606010050006090900B
:102F0000600505050600002000F800200404040602
:102F1000010070B0D0E004070706010040200090D7
:102F20009090700407070601002040009090907078
:102F300004070706010020500090909070040606D8
:102F40000601005000909090700409090601FE20CF
:102F500040009090907090600408080601FE808008
:102F6000E09090E080800408080601FE50009090F8
:102F700090709060506C65617365207265736574C4
:102F8000005052494E5445522048414C544544004B
:102F90005072696E7465722068616C7465642E206D
:102FA0006B696C6C28292063616C6C6564210A0074
:102FB000656E7175657565696E6720220000004059
:102FC000C000003E43000037430000484200004874
:102FD0004200002042000000005761726E696E6777
:102FE0003A20486F6D696E672042756D70204469A4
:102FF0007669736F72203C20310A000202040000DF
:103000000000000000000000004000002543000018
:10301000454300003743FF01014D36303020486FF3
:1030200074656E6420746F6F20636F6C6420746FBE
:10303000206368616E67652066696C616D656E749A
:103040000A001000C90210012C0140012201700188
:103050001801B0010E01F00104015002FA00B002A3
:10306000F0003003E600D003DC009004D2007005CD
:10307000C800A006BE000008B400B009AA00D00B2A
:10308000A000600E960060118C00001582002019CF
:103090007800C01D6E00A0226400B0275A00902C5A
:1030A000500000314600E0343C0010383200903AC5
:1030B0002800603C1E00A03D1400803E0A00203F16
:1030C00000006265640A002C2073797374656D20BA
:1030D00073746F7070656421204865617465725FF8
:1030E00049443A200048656174696E6720666169E9
:1030F0006C6564204245440048656174696E6720D0
:103100006661696C65640048656174696E67206614
:1031100061696C65640048656174696E6720666109
:10312000696C6564204530001000AD0330016A0110
:1031300050022B0170030A019004F500B005E50070
:10314000D006D800F007CE001009C500300ABE0036
:10315000500BB700700CB100900DAB00B00EA60084
:10316000D00FA200F0109D001012990030139500AE
:103170005014920070158E0090168B00B0178700C7
:10318000D0188400F0198100101B7E00301C7B00D9
:10319000501D7900701E7600901F7300B0207000E3
:1031A000D0216E00F0226B001024690030256600EB
:1031B000502663007027610090285E00B0295C00F3
:1031C000D02A5900F02B5600102D5400302E5100FB
:1031D000502F4E0070304B0090314800B032450007
:1031E000D0334200F0343E0010363B003037370019
:1031F0005038330070392E00903A2900B03B23003C
:10320000D03C1B00F03D1100103F0100F03F0000DA
:103210004572723A204D494E54454D502042454426
:10322000004D494E54454D50207472696767657270
:103230006564004572723A204D494E54454D502008
:103240004531004572723A204D494E54454D50204B
:103250004530004572723A204D415854454D50203A
:10326000424544004D415854454D502074726967A1
:103270006765726564004572723A204D4158544545
:103280004D50204531004572723A204D4158544509
:103290004D50204530004572726F7220777269740C
:1032A000696E6720746F20454550524F4D210A00CA
:1032B00056652D6A65726B0056652D6A65726B00E6
:1032C00056652D6A65726B00567A2D6A65726B00C1
:1032D000567A2D6A65726B0056792D6A65726B009D
:1032E00056792D6A65726B0056792D6A65726B008E
:1032F00056782D6A65726B0056782D6A65726B0080
:1033000056782D6A65726B004D6F74696F6E00455B
:1033100073746570732F6D6D004573746570732FD2
:103320006D6D005A73746570732F6D6D005A7374F0
:103330006570732F6D6D005973746570732F6D6DAB
:10334000005973746570732F6D6D005873746570D8
:10335000732F6D6D005873746570732F6D6D004D14
:103360006F74696F6E004F6666004F6E2000456E89
:103370006473746F702061626F727400537465704F
:10338000732F6D6D004A65726B00416363656C65F8
:10339000726174696F6E0056656C6F636974790051
:1033A0005A204F666673657400416476616E63658A
:1033B000642053657474696E67730043616E6E6F49
:1033C0007420656E746572207375626469723A2048
:1033D00000022E2E004D61696E0020204E6F7A7A19
:1033E0006C653A200020004261636B004D696E6994
:1033F0006D756D2054656D70206973203132302EEB
:103400000048656174696E67206661696C65640077
:1034100045787472756465206D6F726500526573CE
:10342000756D65207072696E7400524553554D4537
:10343000204F5054494F4E533A0020204E6F7A7A15
:103440006C653A20006368616E6765006F66207482
:1034500068652066696C616D656E7400576169749A
:1034600020666F72207374617274005052494E541A
:10347000205041555345440020204E6F7A7A6C65A8
:103480003A2000200066696C616D656E7420756E6F
:103490006C6F6164005761697420666F72005052EE
:1034A000494E54205041555345440020204E6F7AD8
:1034B0007A6C653A20002000506C65617365207756
:1034C0006169742E2E2E0048656174696E67206EE6
:1034D0006F7A7A6C65005052494E542050415553D2
:1034E00045440020204E6F7A7A6C653A2000200017
:1034F00068656174206E6F7A7A6C652E0050726513
:10350000737320627574746F6E20746F005052492B
:103510004E54205041555345440020204E6F7A7A36
:103520006C653A2000746F20636F6E74696E756508
:103530002E2E2E00616E642070726573732062758A
:1035400074746F6E00496E736572742066696C6185
:103550006D656E74005052494E542050415553458C
:10356000440020204E6F7A7A6C653A200020006675
:10357000696C616D656E74206C6F61640057616980
:103580007420666F72005052494E5420504155537A
:1035900045440020204E6F7A7A6C653A2000200066
:1035A00066696C616D656E742065787472756465AA
:1035B000005761697420666F72005052494E542062
:1035C00050415553454400746F20726573756D65A5
:1035D000005761697420666F72207072696E7400A2
:1035E0005052494E54205041555345440024F4D480
:1035F0003050C38E20C2A24017828B7011127A9174
:103600000D816CD90AA861E108C75866076151436A
:10361000061E4B5D05C145A7041A411104093D98DA
:1036200003713931034036DB0265339102D43054E3
:1036300002802E1D02632CEE01752AC501B028A060
:1036400001102781018F2564012B244B01E02234D6
:1036500001AC211F018D200D01801FFC00841EED97
:1036600000971DDF00B81CD200E61BC600201BBC63
:1036700000641AB200B219A8000A19A0006A1899C9
:1036800000D117910040178B00B516840031167ECB
:1036900000B31579003A157300C7146F0058146A07
:1036A00000EE1366008813630025135E00C7125BEB
:1036B000006C12570015125400C111510070114FC7
:1036C0000021114B00D61049008D104700461044D0
:1036D0000002104200C00F4000800F3E00420F3C2D
:1036E00000060F3B00CB0E3800930E37005C0E3502
:1036F00000270E3400F30D3200C10D3100900D3063
:1037000000600D2E00320D2D00050D2C00D90C2B64
:1037100000AE0C2900850C29005C0C2700350C2715
:10372000000E0C2600E80B2400C40B2400A00B2381
:10373000007D0B23005A0B2100390B2100180B20B0
:1037400000F80A1F00D90A1E00BB0A1E009D0A1DB0
:1037500000800A1D00630A1C00470A1B002C0A1B7C
:1037600000110A1A00F7091A00DD091900C4091925
:1037700000AB091900920917007B091800630917AB
:10378000004C09160036091600200916000A091512
:1037900000F5081500E0081400CC081400B808145F
:1037A00000A4081400900813007D0812006B081391
:1037B00000580812004608120034081100230811AE
:1037C000001208110001081100F0071000E00710B6
:1037D00000D0071000C0071000B0070F00A10710AD
:1037E0000091070E0083070F0074070F0065070E96
:1037F0000057070E0049070E003B070D002E070E6D
:103800000020070D0013070D0006070D00F9060C38
:1038100000ED060D00E0060C00D4060C00C8060CF6
:1038200000BC060C00B0060C00A4060B0099060CA8
:10383000008D060B0082060B0077060B006C060B52
:103840000061060A0057060B004C060A0042060AF1
:103850000038060A002E060A0024060A001A060A84
:10386000001006090007060A00FD050900F4050915
:1038700000EB050900E2050900D9050900D005099A
:1038800000C7050900BE050900B5050800AD05081B
:1038900000A50509009C050800940508008C050892
:1038A00000840508007C050800740508006C050705
:1038B00000650508005D050700560508004E050770
:1038C00000470507004005080038050700310507D7
:1038D000002A050700230507001C0506001605073A
:1038E000000F0507000805060002050700FB040697
:1038F00000F5040700EE040600E8040600E20407F1
:1039000000DB040600D5040600CF040600C9040647
:1039100000C3040600BD040600B7040600B1040598
:1039200000AC040600A6040600A00405009B0406E3
:103930000095040500900406008A0405008504052E
:1039400000800406007A0405007504050070040573
:10395000006B04050066040500610405005C0405B5
:103960000057040500520405004D040500480405F5
:1039700000430405003E0404003A04050035040534
:1039800000300404002C040500270404002304056F
:10399000001E0404001A04040016040500110404A7
:1039A000000D0404000904050004040400000404DC
:1039B00000FC030400F8030400F4030400F0030413
:1039C00000EC030400E8030400E4030400E0030443
:1039D00000DC030400D8030400D4030400D0030473
:1039E00000CC030400C8030300C503030024F4044F
:1039F000D9201BC40C5C0E9804C4095F02650771D2
:103A000001F405F900FB04B30048048700C1036911
:103A1000005803550003034500BE023A00840231FA
:103A20000053022A002902250004022000E4011CA0
:103A300000C8011900AF0117009801140084011398
:103A400000710110006101100051010E0043010DD1
:103A50000036010B002B010B0020010B00150109A2
:103A6000000C01090003010800FB000800F3000836
:103A700000EB000700E4000600DE000600D80006A8
:103A800000D2000600CC000500C7000500C20005FA
:103A900000BD000400B9000400B5000400B100043A
:103AA00000AD000400A9000400A5000300A200036B
:103AB000009F0004009B0003009800030095000293
:103AC0000093000300900003008D0002008B0003B0
:103AD00000880002008600020084000300810002CA
:103AE000007F0002007D0002007B000200790002DE
:103AF00000770001007600020074000200720001ED
:103B000000710002006F0002006D0001006C0002F5
:103B1000006A000100690002006700010066000100
:103B20000065000100640002006200010061000104
:103B300000600001005F0002005D0001005C000108
:103B4000005B0001005A000100590001005800010B
:103B5000005700010056000100550001005400010B
:103B60000053000000530001005200010051000109
:103B700000500001004F0001004E0000004E000107
:103B8000004D0001004C0001004B0000004B000103
:103B9000004A0001004900010048000000480001FF
:103BA00000470001004600000046000100450000FB
:103BB00000450001004400010043000000430001F3
:103BC00000420000004200010041000000410001ED
:103BD00000400001003F0000003F0001003E0000E7
:103BE000003E0001003D0000003D0001003C0000DF
:103BF000003C0000003C0001003B0000003B0001D5
:103C0000003A0000003A00010039000000390001CC
:103C100000380000003800000038000100370000C4
:103C200000370001003600000036000000360001B9
:103C300000350000003500000035000100340000B0
:103C400000340000003400010033000000330000A5
:103C50000033000100320000003200000032000199
:103C60000031000000310000003100010030000090
:103C70000030000000300001002F0000002F000085
:103C8000002F0000002F0001002E0000002E000079
:103C9000002E0001002D0000002D0000002D00006E
:103CA000002D0001002C0000002C0000002C000062
:103CB000002C0001002B0000002B0000002B000056
:103CC000002B0001002A0000002A0000002A00004A
:103CD000002A00010029000000290000002900003E
:103CE0000029000000290001002800000028000031
:103CF0000028000000280000002800010027000024
:103D00000027000000270000002700000027000116
:103D1000002600000026000000260000002600000B
:103D200000260001002500000025000000250000FD
:103D300000250000002500000025000100240000EF
:103D400000240000002400000024000000240001E2
:103D500000230000002300000023000000230000D7
:103D600000230000002300000023000100220000C7
:103D700000220000002200000022000000220000BB
:103D800000220001002100000021000000210000AD
:103D9000002100000021000000210000002100019E
:103DA0000020000000200000002000000020000093
:103DB0000020000000200000002000000020000182
:103DC000001F0000001F0000001F0000001F000077
:103DD000001F0000001F0000001F0001001E000067
:103DE000001E0000001E0000001E0000004D3834C0
:103DF00020582059205A2045004D6F766520617863
:103E000069730044697361626C65207374657070D6
:103E1000657273004D383400426564204C657665E8
:103E20006C696E67004732382058590A4D31303975
:103E300020533137350A473238205A0A4D3130394C
:103E400020523134350A4731320A4732390A4D316E
:103E50003034205330004175746F20686F6D6500F9
:103E6000473238004D61696E004D3530320A4D35AC
:103E70003030004C6F61642073657474696E6773D1
:103E800000526573746F7265206661696C73616658
:103E9000650053746F72652073657474696E67731F
:103EA00000416476616E6365642053657474696E65
:103EB0006773004D61696E000A003B204545505212
:103EC0004F4D20496E6465783A20005570646174E6
:103ED000696E67207A6F666673657420696E204527
:103EE0004550524F4D3A20000600060006000600DD
:103EF000060006000600060006003FC01F800F00F7
:103F0000060006000F001F803FC0060006000600E6
:103F100006000600060006000600060007F8000C72
:103F20000C0010020020010060018040008040036E
:103F3000E04001C040008040000040000060000000
:103F40002000001000000C0C0007F80001FE000328
:103F500003000400800800401800601000207C006E
:103F60002038002010002000002000002000006009
:103F700000004000008003030001FE00FFFFFF7F00
:103F800080FFC0FFC0FFC07F807F80FFC0FFC0FFF9
:103F9000C03F001E000C005A204F66667365740017
:103FA0005A204F666673657400466C6F7700466CE6
:103FB0006F770046616E2073706565640046616EC0
:103FC0002073706565640042656400426564004E5C
:103FD0006F7A7A6C65004E6F7A7A6C650053706503
:103FE0006564005370656564004D61696E004D6FD6
:103FF000766520580048617264636F64656420448C
:10400000656661756C742053657474696E6773209E
:104010004C6F616465640A002823000028230000B7
:10402000C8000000E803000000009643000096432B
:1040300000009643000020420000C8420000C84231
:104040000000C8420000D243204500205A00202032
:104050004D39303720580053746570706572206D8B
:104060006F746F722063757272656E74733A0A00B2
:1040700020453000205A0020590020580053746514
:1040800070706572206472697665722063757272F1
:10409000656E743A0A0020204D383531205A005A96
:1040A0002D50726F6265204F666673657420286DAF
:1040B0006D293A0A0020440020490020204D333069
:1040C0003420500020440020490020204D3330315E
:1040D0002050005049442073657474696E67733AC8
:1040E0000A0020460020420020480020204D3134A4
:1040F000352053004D6174657269616C206865619B
:1041000074757020706172616D65746572733A0ABE
:104110000020204D3432302053004175746F20420E
:104120006564204C6576656C696E673A0A00205AB2
:104130000020590020204D323036205800486F6D45
:1041400065206F66667365743A0A00204500205A40
:104150000020590020580020420020540020204D0B
:10416000323035205300416476616E6365643A20D5
:10417000533C6D696E5F66656564726174653E206F
:10418000543C6D696E5F74726176656C5F666565DF
:1041900064726174653E20423C6D696E5F73656751
:1041A0006D656E745F74696D655F6D733E20583C1C
:1041B0006D61785F78795F6A65726B3E205A3C6DFD
:1041C00061785F7A5F6A65726B3E20453C6D61780D
:1041D0005F655F6A65726B3E0A00205400205200E2
:1041E00020204D323034205000416363656C65728D
:1041F0006174696F6E2028756E6974732F7332292C
:104200003A20503C7072696E745F616363656C3E06
:1042100020523C726574726163745F616363656CA4
:104220003E20543C74726176656C5F616363656CBB
:104230003E0A00204500205A0020590020204D321F
:1042400030312058004D6178696D756D2041636390
:10425000656C65726174696F6E2028756E69747320
:104260002F7332293A0A00204500205A00205900B5
:1042700020204D3230332058004D6178696D756DC6
:10428000206665656472617465732028756E697453
:10429000732F73293A0A00204500205A0020590044
:1042A00020204D393220580053746570732070659A
:1042B0007220756E69743A0A0020204D3230302029
:1042C00044300A0020204D32303020440020446920
:1042D0007361626C65640A0046696C616D656E7439
:1042E0002073657474696E67733A0020204D313411
:1042F000392043203B20556E69747320696E20433A
:10430000656C736975730A002020473231202020C4
:10431000203B20556E69747320696E206D6D0A0014
:10432000526573656E643A20002042002050006F91
:104330006B0020647269766572206F7665727465B1
:104340006D7065726174757265207761726E696EE9
:1043500067210A003A20004B494C4C45442E20006E
:104360004B494C4C20636175736564206279204B26
:10437000494C4C20627574746F6E2F70696E0A0020
:104380004B494C4C45442E20004B494C4C2063611A
:104390007573656420627920746F6F206D75636832
:1043A00020696E6163746976652074696D65202D7E
:1043B0002063757272656E7420636F6D6D616E64DB
:1043C0003A20000201050800FF060121023520FF06
:1043D000FF07FF06FF0900502216568080808000EC
:1043E00080153353A0A0A00257575050F850F850F2
:1043F000500257572070A07028702013355580A0A8
:1044000040A02002475740A0A040A0A05025135331
:104410008080801226564080808080401226568000
:1044200040404040800245559060F06090025555F4
:104430002020F82020113353604080044151F011B6
:10444000335340E040024656101020408080123620
:104450005640A0A0A0A04012365640C0404040E0C8
:104460000246566090106080F0024656F0206010C0
:1044700090600246562060A0F02020024656F08050
:10448000E01090600246566080E0909060024656D0
:10449000F0102020404002465660906090906002EC
:1044A0004656609090701060122555C0C000C0C084
:1044B0001136566060006040801236562040808081
:1044C0004020034353F000F0123656804020204035
:1044D0008012365640A0204000400158583048987D
:1044E000A8A8904030024656609090F09090024606
:1044F00056E090E09090E002465660908080906098
:10450000024656E090909090E0024656F080E0809F
:1045100080F0024656F080E080808002465660902F
:1045200080B090600246569090F09090901236566F
:10453000E040404040E002465670202020A040026B
:10454000465690A0C0A0A0900246568080808080F1
:10455000F002465690F0F090909002465690D0F0BF
:10456000B0B090024656609090909060024656E03F
:104570009090E08080014757609090D0B06010022A
:104580004656E09090E09090024656609040209011
:1045900060123656E04040404040024656909090AF
:1045A00090906002465690909090606002465690BF
:1045B0009090F0F090024656909060609090025675
:1045C00056888850202020024656F010204080F067
:1045D000123656E080808080E0024656808040207F
:1045E0001010123656E020202020E016325240A053
:1045F000014151F016225280400244547090907054
:104600000246568080E09090E012345460808060D2
:1046100002465610107090907002445460B0C06012
:10462000024656205040E0404001455560907010D1
:10463000600246568080E09090901236564000C04E
:104640004040E01137572000202020A0400246566D
:10465000808090E09090123656C040404040E0028A
:104660005454D0A8A8A8024454E090909002445416
:1046700060909060014555E090E080800145557064
:1046800090701010024454A0D0808012345460C046
:1046900020C00246564040E04050200244549090D2
:1046A0009070123454A0A0A04002545488A8A8507E
:1046B0000244549060609001455590907090600263
:1046C0004454F02040F0024757304020C020403092
:1046D000221656808080808080024757C02040305C
:1046E0004020C006425250A0FFFFFFFFFFFFFFFF28
:1046F000FFFFFFFFFFFFFFFFFFFFFFFFFFFFFFFFCA
:10470000FFFFFFFFFFFFFFFFFF090050221656804B
:1047100000808080800146562070A0A07020024654
:10472000562050E04050A0025555887050708802C5
:1047300056568850F820F820221757808080008035
:1047400080800247577080E0907010E0173151A0D0
:1047500002565670A8C8C8A87014355560A06000ED
:10476000E003435350A050123353E0202014315142
:10477000E002565670E8D8E8D870173151E015338A
:104780005340A04012355540E04000E014355540FC
:10479000A02040E0143555C020C020C01622524051
:1047A00080014555909090E08002565678E8E86880
:1047B000282824115180112252408014355540C0C0
:1047C0004040E014355540A04000E0034353A05062
:1047D000A0024757808080A060F020024757808069
:1047E000A0D010207002475780408060A0F02012B7
:1047F000365640004080A04002475740206090F06D
:10480000909002475720406090F090900247576088
:10481000906090F0909002475750A06090F0909078
:1048200002475790006090F0909002475760906068
:1048300090F0909002465670A0A0F0A0B0014757AB
:10484000609080809060400247574020F080E08078
:10485000F00247572040F080E080F0024757609018
:10486000F080E080F00247579000F080E080F01286
:1048700037578040E0404040E01237572040E0404A
:104880004040E012375740A0E0404040E012375728
:10489000A000E0404040E00256567048E8484870AA
:1048A00002475750A090D0B09090024757402060E8
:1048B000909090600247572040609090906002472F
:1048C000576090609090906002475750A060909021
:1048D000906002475790006090909060123353A010
:1048E00040A002465670B0B0D0D0E00247574020FA
:1048F0009090909060024757204090909090600276
:104900004757609090909090600247579000909029
:104910009090600257571020885020202002465661
:1049200080E09090E0800246566090A0A090A002A7
:104930004757402000709090700247572040007009
:104940009090700247572050007090907002475727
:1049500050A0007090907002465650007090907079
:1049600002475760906070909070025454F068B0A5
:1049700078113555608080604002475740200060C4
:10498000B0C06002475720400060B0C06002475787
:1049900060900060B0C060024656500060B0C060D9
:1049A000123757804000C04040E012375720400087
:1049B000C04040E012375740A000C04040E01236EF
:1049C00056A000C04040E0024757A040A0107090A1
:1049D0006002475750A000E0909090024757402057
:1049E0000060909060024757204000609090600205
:1049F00047576090006090906002475750A0006059
:104A0000909060024656900060909060123555403C
:104A100000E0004002445470B0D0E002475740200C
:104A20000090909070024757204000909090700244
:104A3000475760900090909070024656900090907A
:104A40009070014858204000909070906001475746
:104A50008080E090E08080014757900090907090B7
:104A60006001050700FE0500FB01F220FFFE05FEC8
:104A700005FE02004002152580808000800532423C
:104A8000A0A002556550F850F8500146562070C05D
:104A900030E0200255659010204048025565608046
:104AA0006890680512228080022535408080804011
:104AB0000225358040404080043343A040A00333AA
:104AC0004340E0400122324080043141E0021121A4
:104AD00080025565081020408002455560909090F6
:104AE00060022535C040404040024555E0106080DE
:104AF000F0024555E0106010E00245552060A0F03E
:104B000020024555F080E010E00245556080E090BD
:104B100060024555F010204040024555609060907D
:104B2000600245556090701060031323800080027E
:104B300014248000808002354520408040200333CB
:104B400043E000E00235458040204080024555E0CA
:104B5000106000400255657088B8A8700245556025
:104B60009090F090024555E090E090E0023545606D
:104B700080808060024555E0909090E0023545E0ED
:104B800080E080E0023545E080E08080024555709D
:104B900080B090700245559090F09090023545E0BD
:104BA000404040E00245553010109060024555905D
:104BB000A0C0A09002354580808080E002556588C5
:104BC000D8A8888802455590D0B09090024555608D
:104BD00090909060024555E09090E08001465660CC
:104BE0009090906010024555E09090E090024555FD
:104BF00070806010E0023545E0404040400245557D
:104C000090909090600245559090A0A0400255650C
:104C100088A8A8A8500245559090609090024555EC
:104C20009090701060023545E0204080E00225350C
:104C3000C0808080C0025565804020100802253564
:104C4000C0404040C005324240A0024151F0052220
:104C50003280400244547090907002455580E0903C
:104C600090E002344460808060024555107090905E
:104C70007002445460B0C0600235452040E04040BE
:104C800000465670909070106002455580E09090FC
:104C9000900215258000808080002737400040402A
:104CA0004040800245558090A0E09002152580800C
:104CB000808080025464F0A8A8A8024454E0909038
:104CC0009002445460909060004656E09090E080DE
:104CD00080004656709090701010023444A0C0803E
:104CE0008002445470C030E002354540E04040202E
:104CF000024454909090700244549090A04002540A
:104D000064A8A85050023444A04040A000465690E9
:104D10009090701060024454F02040F002354560DD
:104D2000408040600215258080808080023545C02B
:104D3000402040C005425250A0FFFFFFFFFFFFFF91
:104D4000FFFFFFFFFFFFFFFFFFFFFFFFFFFFFFFF73
:104D5000FFFFFFFFFFFFFFFFFFFF020040FFFFFF1E
:104D6000FFFFFFFFFFFFFFFFFFFFFFFFFFFFFFFF53
:104D7000FFFFFFFFFFFFFFFFFFFFFFFFFFFFFFFF43
:104D8000FFFFFFFFFFFFFFFFFFFFFFFFFFFFFFFF33
:104D9000FFFFFFFFFFFFFFFFFFFFFFFFFFFFFFFF23
:104DA000FFFFFFFFFFFFFFFFFFFFFFFFFFFFFFFF13
:104DB000FFFFFFFFFFFFFFFFFFFFFFFF01060D00EB
:104DC000FE09016602D620FFFE0BFE0AFE0D006002
:104DD000221969808080808080800080183363A0E1
:104DE000A0A00357675050F850F85050025969205E
:104DF00078A0A0702828F02002596948A8501020F7
:104E00004050A89002586840A0A040A09890682800
:104E10001363808080113B6B2040408080808080C5
:104E2000404020113B6B804040202020202040400B
:104E30008006556520A870A8200455652020F8201C
:104E400020113363604080065161F811336340E004
:104E500040025969080810102040408080025969BA
:104E60002050888888888850200259692060A020B6
:104E700020202020F802596970888808102040807E
:104E8000F8025969F80810207008088870025969FA
:104E9000101030505090F81010025969F88080B00E
:104EA000C80808887002596970888080F0888888EE
:104EB00070025969F80810102020404040025969DA
:104EC0007088888870888888700259697088888896
:104ED000780808887011386840E040000040E040E1
:104EE00011386840E04000006040800259690810B5
:104EF00020408040201008045464F80000F8025953
:104F0000698040201008102040800259697088880C
:104F100008102020002002596970888898A8A8B03D
:104F200080780259692050888888F88888880259D2
:104F300069F048484870484848F0025969708880CC
:104F4000808080808870025969F048484848484805
:104F500048F0025969F8808080F0808080F802591A
:104F600069F8808080F08080808002596970888034
:104F700080809888887002596988888888F888882D
:104F80008888123969E040404040404040E0025982
:104F900069381010101010109060025969888890BC
:104FA000A0C0A0908888025969808080808080801D
:104FB00080F80259698888D8A8A888888888025902
:104FC0006988C8C8A8A8989888880259697088888C
:104FD000888888888870025969F0888888F080807D
:104FE0008080015A6A70888888888888A87008023A
:104FF0005969F0888888F0A090888802596970887B
:1050000080807008088870025969F82020202020CC
:1050100020202002596988888888888888887002BA
:10502000596988888888505050202002596988889A
:105030008888A8A8A8A8500259698888505020508C
:1050400050888802596988885050202020202002EA
:105050005969F808101020404080F8113B6BE0803F
:105060008080808080808080E0025969808040401C
:105070002010100808113B6BE02020202020202069
:105080002020E0085363205088015161F82A2262F1
:105090008040025666700878889868025969808056
:1050A00080F088888888F0025666708880808870D2
:1050B00002596908080878888888887802566670D6
:1050C00088F880887002596930484040F04040407C
:1050D000400058687088888878088870025969800C
:1050E0008080B0C8888888881238684000C04040F6
:1050F0004040E0004A6A100030101010109090609C
:1051000002596980808090A0C0A09088123969C03F
:1051100040404040404040E0025666D0A8A8A8A8C1
:1051200088025666B0C88888888802566670888863
:10513000888870005868F0888888F08080800058DF
:10514000687888888878080808025666B0C8808021
:1051500080800256667088601088700258684040EF
:10516000F040404048300256668888888898680237
:1051700056668888885050200256668888A8A8A855
:1051800050025666885020205088005868888888C9
:105190009868088870025666F810204080F8015B15
:1051A0006B1820202020C020202020182219698080
:1051B0008080808080808080015B6BC020202020E8
:1051C0001820202020C008536348A890FFFFFFFF4D
:1051D000FFFFFFFFFFFFFFFFFFFFFFFFFFFFFFFFDF
:1051E000FFFFFFFFFFFFFFFFFFFFFFFFFF0D00605F
:1051F0002219698000808080808080800358682028
:1052000070A8A0A0A8702002596930484040E04032
:105210004048B003566688705050708802596988BB
:10522000885050F820F82020221969808080800062
:1052300080808080124A6A609080609090601090B8
:10524000601A3262A0A00359697088A8D8C8D8A88B
:105250008870045767700878887800F803566628C5
:1052600050A0A05028045363F80808163161E003E9
:1052700059697088E8D8D8E8D888700A5161F81759
:105280004464609090600357672020F8202000F865
:1052900007356540A02040E007356540A04020C0AC
:1052A0002A226240800058688888888898E8808030
:1052B00002596978E8E8E8E868282828262161C0CA
:1052C000202262408007356540C04040E0045767B7
:1052D000708888887000F8035666A050282850A06F
:1052E000025A6A40C04040E00818283808025A6A4A
:1052F00040C04040E01028081038025A6A40A040E0
:1053000020A0481828380802596920002020408031
:10531000888870025A6A40200020508888F888885F
:10532000025A6A10200020508888F88888025A6A39
:1053300030480020508888F88888025A6A2850002F
:1053400020508888F88888025A6A50500020508877
:1053500088F88888025A6A20502020508888F88867
:105360008802596958A0A0A0B0E0A0A0B8005B6B6B
:105370007088808080808088702040025A6A402037
:1053800000F88080F08080F8025A6A102000F880CF
:1053900080F08080F8025A6A304800F88080F080FF
:1053A00080F8025A6A505000F88080F08080F8122D
:1053B0003A6A804000E04040404040E0123A6A20B3
:1053C0004000E04040404040E0124A6A609000E007
:1053D0004040404040E0123A6AA0A000E040404017
:1053E0004040E0025969F0484848E8484848F0021F
:1053F0005A6A2850008888C8A8988888025A6A4043
:10540000200070888888888870025A6A102000708E
:10541000888888888870025A6A304800708888882E
:10542000888870025A6A2850007088888888887036
:10543000025A6A50500070888888888870035565C1
:105440008850205088015B6B08709898A8A8A8C85D
:10545000C87080025A6A40200088888888888870CE
:10546000025A6A10200088888888888870025A6AE0
:1054700030480088888888888870025A6A505000AE
:1054800088888888888870025A6A10200088885026
:105490002020202002596980F0888888F080808050
:1054A000025969609090A0A0908888B00259694024
:1054B00020007008788898680259691020007008E8
:1054C0007888986802596930480070087888986828
:1054D0000259692850007008788898680259695004
:1054E0005000700878889868025A6A304830007016
:1054F0000878889868025666702870A0A8500058EE
:10550000687088808088702040025969402000704F
:1055100088F88088700259691020007088F88088A7
:10552000700259693048007088F8808870025969A3
:105530005050007088F8808870123969804000C02F
:1055400040404040E0123969204000C040404040A7
:10555000E0124969609000C040404040E012396963
:10556000A0A000C040404040E0025A6A50206010B5
:10557000708888888870025969285000B0C8888867
:10558000888802596940200070888888887002598C
:105590006910200070888888887002596930480036
:1055A00070888888887002596928500070888888B7
:1055B0008870025969505000708888888870035735
:1055C00067202000F8002020015868087098A8A8DB
:1055D000C8708002596940200088888888986802CD
:1055E000596910200088888888986802596930486D
:1055F000008888888898680259695050008888888F
:10560000889868005B6B10200088888898680888F4
:1056100070005A6A8080B0C88888C8B08080005BFB
:105620006B505000888888986808887000000000D7
:10563000000000000000000000000000000000006A
:105640000000000000000000000000000000000C4E
:10565000000000000000000C00000000000000122C
:1056600000000000000000230000000000000021F6
:10567000000000000000004C800000000000005E00
:10568000800000000000009240000000000000A127
:105690004000000000000121200000000000027F07
:1056A000900000000000020010000000000007FF52
:1056B000F8000000000004000800000000000800DE
:1056C00004000000000008000600000000001000B8
:1056D000020000000000301E010000000000207FDA
:1056E00081000000000041FFE0800000000043FC5A
:1056F000F08000000000873B7840000000018EDB56
:10570000FC60000000010FEBCC20000000021FED48
:10571000B610000000021FDEB6100000000439CDF4
:105720007F080000000436E0FF08000000087EC08B
:10573000BB84000000187F005D86000000107FC061
:10574000ED82000000203CC07301000000203B33CC
:105750007F01000000701BE77E03800000C81DEE83
:10576000DE04C00000880FDEDC04400001240FDFEF
:105770003C092000012607DBF8192000027203E72C
:10578000F0139000025101FFE02290000489007F95
:10579000802448000904801E004824000BFE4000BD
:1057A00000DFF40010004000008002001FFFFFFF38
:1057B000FFFFFE00000000000000000000000000ED
:1057C0000000000000000000000000001022103C5B
:1057D0003C0E1F0010221004221104001022100899
:1057E00022110400102210083C1104001022101095
:1057F0002211040010221020221104001E1C1E3C45
:105800003C0E04000000000000000000000000004A
:105810000000000000000000000000000000000088
:105820000000000000000000000000000000000078
:105830000000000000000000000000000000000068
:105840000000000000000000000000000000000058
:105850000000000000000000000000000000000048
:10586000000000000000000000004D3630302042F3
:1058700030005072696E7420706175736564004DFC
:1058800031323500004D3234005072696E7420613F
:10589000626F72746564004E6F20534420636172BE
:1058A00064005072696E742066726F6D20534400FC
:1058B00053746F70207072696E7400526573756DE9
:1058C00065207072696E7400506175736520707226
:1058D000696E740041626F7574204669726D7761FC
:1058E0007265004368616E67652066696C616D650D
:1058F0006E7400436F6E66696775726174696F6E6E
:105900000054656D7065726174757265004D6F76D7
:10591000656D656E740054756E6500496E666F2026
:1059200073637265656E004B494C4C45442E2000F4
:1059300023D642F511241FBECFEFD1E2DEBFCDBF8B
:1059400000E00CBF14E0A0E0B2E0E4E4F1E802E023
:105950000BBF02C007900D92A834B107D9F727E119
:10596000A8E4B4E001C01D92AC3AB207E1F71CE232
:10597000C9E9DCE200E006C021970109802FFE01A1
:105980000F94303FC839D10780E00807A9F70E947B
:105990002B5D0D9491400C9400002F923F924F92FA
:1059A0005F926F927F928F929F92AF92BF92CF92AF
:1059B000DF92EF92FF920F931F93CF93DF93CDB7B8
:1059C000DEB7CB59D1090FB6F894DEBF0FBECDBFFD
:1059D0000091620620E6029F800111240E511B4FA8
:1059E0008091F31680FF1AC0EDEFF1E284917F0100
:1059F0003FEFE31AF30A811102C0780104C00F944B
:105A0000452EF701F3CFD7018D917D01882319F041
:105A10000F94452EF8CF8AE00F94452E109267041C
:105A2000109266048FE380937C0410927B041092A2
:105A30007A0410926204109263041092640410922B
:105A40006504F80180810F5F1F4F8032D1F38E34DF
:105A5000B1F4818190ED980F9A3020F08D3211F0E1
:105A60008B3269F43296DF0131962C9120532A3023
:105A7000D0F3CD01FC01019620812032D9F3F093BF
:105A8000B515E093B4157F01BFEFEB1AFB0A108147
:105A90006AE270E0C7010F946240009731F0FC01A8
:105AA000319780818032E1F311821D3429F0143561
:105AB00019F0173409F0CBC0F70180812FEFE21AFB
:105AC000F20A8032C9F380538A3008F0C0C01093C4
:105AD0007C0420917A0430917B044AE03196429F05
:105AE000C001439F900D1124DF0111972C9130E0EC
:105AF00020533109280F391F808180538A3070F379
:105B000030937B0420937A04DF0131968C918032AC
:105B1000D9F31D34D1F42E31310591F03CF4273105
:105B2000310571F02C31310581F40AC0253731057A
:105B300064F02737310524F0203A43E0340729F494
:105B4000B0936704A093660482C010926704109219
:105B500066040091B41561E070E0CD0101964C91AE
:105B6000442309F474C0413299F41D3489F420327D
:105B7000310571F4909367048093660463E270E0EA
:105B80000F946240009709F462C0DC011C925FC070
:105B90005FEBD52ED40EE9E1ED15C0F1FC01BE2F6F
:105BA000AF2F51915032D9F38B2F9A2FE0EDE50FA3
:105BB000EA3040F0E3EDE50FE23020F05B3211F027
:105BC0000C941D48DC01AD2CB12C750143E0F5941B
:105BD000E7944A95E1F7A7014E595B4F7A014D2DA5
:105BE0004770FB0102C0EE0FFF1F4A95E2F7AF01BD
:105BF000F7015081452B4083109711F0A01B01C085
:105C0000A0E0F501E85BFB4FA0830AC04091660469
:105C100050916704452B21F4B0936704A093660468
:105C2000DC014C9141544A3110F4DC0196CFFC0167
:105C3000DF0131969C9190539A30D0F3AD01CA01A7
:105C40004F5F5F4FDC01EC91E032C9F3EECF809102
:105C50007C048D3411F40C946536843511F40C9465
:105C6000BE47873411F00C94004880917A049091DB
:105C70007B048A31910509F4F4C6BCF484309105A3
:105C800044F4823091050CF01FC197FF2BC00C9497
:105C90001A488430910509F4E0C60C9711F00C9471
:105CA0001A480E94B68C0C941A488E31910509F45A
:105CB0007DC73CF48C31910509F464C70CF4D8C657
:105CC00066C78B35910509F4F7C78C35910509F442
:105CD000F8C78A35910511F00C941A48109279048E
:105CE0000C941A4880917302882311F40C941A487A
:105CF0000E94568D87E99FE00F9451270E94D75C40
:105D00008091F31683FD8FC0C090A30FD090A40F95
:105D1000E090A50FF090A60F20913E0730913F072D
:105D20004091400750914107C701B6010F94D73702
:105D3000882309F478C080914E15811138C0609194
:105D40007E0270917F02072E000C880B990B0F9436
:105D5000DD379B01AC0160914A1570914B15809124
:105D60004C1590914D150F94D73787FF20C0C092E6
:105D70003E07D0923F07E0924007F0924107EDEFD7
:105D8000F1E284918F010F5F1F4F882321F00F9460
:105D9000452EF801F6CFE0EBF2E084918F010F5F22
:105DA0001F4F882321F00F94452EF801F6CFC090A5
:105DB000A30FD090A40FE090A50FF090A60F209114
:105DC0003E0730913F074091400750914107C7017E
:105DD000B6010F94403C20E030E048E453E40F94D7
:105DE000673E181604F5C0923E07D0923F07E09236
:105DF0004007F0924107EDEFF1E284918F010F5FD0
:105E00001F4F882321F00F94452EF801F6CFE1E9CA
:105E1000F2E084918F010F5F1F4F882321F00F94D0
:105E2000452EF801F6CF2091970F3091980F4091B1
:105E3000990F50919A0F60913207709133078091BA
:105E40003407909135070F94D73781111DC02091E9
:105E50009B0F30919C0F40919D0F50919E0F609130
:105E600036077091370780913807909139070F9462
:105E7000D737811109C06091250270912602809167
:105E80002702909128021AC06091840270918502C5
:105E9000072E000C880B990B0F94DD3720912502FB
:105EA0003091260240912702509128020F943C38ED
:105EB0002AE037ED43E25CE30F943C380E942EACBD
:105EC0000E9424AC0C941A4820917302222311F4EE
:105ED0000C941A4811E0029709F010E00E94568DC8
:105EE00082E50E949DB1882309F45CC10E9437B10C
:105EF0006B017C014090320750903307609034076B
:105F00007090350720913607309137074091380758
:105F10005091390763962CAF3DAF4EAF5FAF63979B
:105F20008091970F9091980FA091990FB0919A0F2F
:105F300067968CAF9DAFAEAFBFAF679720919B0FB9
:105F400030919C0F40919D0F50919E0F6F962CAFFA
:105F50003DAF4EAF5FAF6F9720E030E0A901C701C2
:105F6000B6010F94D737882309F45DC5A3019201C8
:105F700067966CAD7DAD8EAD9FAD67970F94D737AB
:105F8000811111C063962CAD3DAD4EAD5FAD6397F1
:105F90006F966CAD7DAD8EAD9FAD6F970F94D7377B
:105FA000882309F440C520E030E0A901C701B6010B
:105FB0000F94D737881F8827881F18130BC080E0DD
:105FC00090E0A0E8BFE3AB968CAF9DAFAEAFBFAFA4
:105FD000AB970AC020E030E040E85FEBAB962CAF17
:105FE0003DAF4EAF5FAFAB97A301920167966CAD2B
:105FF0007DAD8EAD9FAD67970F94403CA3966CAF7F
:106000007DAF8EAF9FAFA39763962CAD3DAD4EADE8
:106010005FAD63976F966CAD7DAD8EAD9FAD6F97A5
:106020000F94403CA7966CAF7DAF8EAF9FAFA79704
:10603000A3962CAD3DAD4EAD5FADA397CA01B9019E
:106040000F943C384B015C01A7962CAD3DAD4EAD95
:106050005FADA797CA01B9010F943C389B01AC0111
:10606000C501B4010F94413C0F94AC3E6B966CAFEC
:106070007DAF8EAF9FAF6B9720E030E040E05FE3F5
:106080000F943C384B015C01A7019601C701B60192
:106090000F943C386B017C01A5019401C501B4014A
:1060A0000F943C389B01AC01C701B6010F94403CF2
:1060B0000F94AC3E9B01AC01AB966CAD7DAD8EAD4B
:1060C0009FADAB970F943C384B015C0167962CADAC
:1060D0003DAD4EAD5FAD6797C301B2010F94413C3A
:1060E00020E030E040E05FE30F943C386B017C013E
:1060F000A7966CAD7DAD8EAD9FADA79790586B9672
:106100002CAD3DAD4EAD5FAD6B970F941D3D9B012A
:10611000AC01C501B4010F943C389B01AC01C7012F
:10612000B6010F94413CA30192010F94403C6B01D6
:106130007C016F962CAD3DAD4EAD5FAD6F97639614
:106140006CAD7DAD8EAD9FAD63970F94413C20E06B
:1061500030E040E05FE30F943C382B013C016B964C
:106160002CAD3DAD4EAD5FAD6B97A3966CAD7DADE7
:106170008EAD9FADA3970F941D3D9B01AC01C50152
:10618000B4010F943C389B01AC01C301B2010F94E0
:10619000413C63962CAD3DAD4EAD5FAD63970F9422
:1061A000403C14C089E40E949DB1882329F00E94DC
:1061B00037B16B017C0103C0C12CD12C76018AE47C
:1061C0000E949DB18823F9F00E9437B16F966CAFA1
:1061D0007DAF8EAF9FAF6F9720E030E0A901C70180
:1061E000B6010F94D73781111EC020E030E0A9011D
:1061F0006F966CAD7DAD8EAD9FAD6F970F94D73719
:10620000811111C010C420E030E0A901C701B6011E
:106210000F94D737882309F406C46F961CAE1DAEC1
:106220001EAE1FAE6F97D701C601B05863968CAFF4
:106230009DAFAEAFBFAF63976F962CAD3DAD4EAD8A
:106240005FAD6F97505867962CAF3DAF4EAF5FAFC5
:1062500067979C01AD01BC01CD010F943C384B0107
:106260005C0167962CAD3DAD4EAD5FAD6797CA0141
:10627000B9010F943C389B01AC01C501B4010F94E6
:10628000413C0F94AC3EE7966CAF7DAF8EAF9FAFB5
:10629000E7978091320790913307A0913407B0912E
:1062A00035076B968CAF9DAFAEAFBFAF6B97A701B5
:1062B0009601BC01CD010F94413CAB966CAF7DAF14
:1062C0008EAF9FAFAB972091360730913707409143
:1062D000380750913907A3962CAF3DAF4EAF5FAF53
:1062E000A3976F962CAD3DAD4EAD5FAD6F97A39666
:1062F0006CAD7DAD8EAD9FADA3970F94413CEF96F5
:106300006CAF7DAF8EAF9FAFEF978091970F90915D
:10631000980FA091990FB0919A0FAF968CAF9DAF47
:10632000AEAFBFAFAF97AB962CAD3DAD4EAD5FAD51
:10633000AB97BC01CD010F94403C6B017C012091D7
:106340009B0F30919C0F40919D0F50919E0FE396B3
:106350002CAF3DAF4EAF5FAFE397EF962CAD3DADA9
:106360004EAD5FADEF97E3966CAD7DAD8EAD9FAD5D
:10637000E3970F94403C4B015C0180913A07909168
:106380003B07A0913C07B0913D07C158DF4F888380
:106390009983AA83BB83CF57D0409C01AD01609104
:1063A0009F0F7091A00F8091A10F9091A20F0F9459
:1063B000403CA7966CAF7DAF8EAF9FAFA797209163
:1063C0003E0730913F074091400750914107CD571C
:1063D000DF4F288339834A835B83C358D040609161
:1063E000A30F7091A40F8091A50F9091A60F0F9409
:1063F000403CEB966CAF7DAF8EAF9FAFEB97A701A4
:10640000960163966CAD7DAD8EAD9FAD63970F9495
:106410003C382B013C01A501940167966CAD7DAD24
:106420008EAD9FAD67970F943C389B01AC01C301C3
:10643000B2010F94413C2B013C01A50194016396EC
:106440006CAD7DAD8EAD9FAD63970F943C384B0125
:106450005C01A701960167966CAD7DAD8EAD9FADD9
:1064600067970F943C389B01AC01C501B4010F94B0
:10647000403CA30192010F94B43C6B017C0120E0ED
:1064800030E0A9010F94D73787FF0AC02BED3FE01A
:1064900049EC50E4C701B6010F94413C6B017C010B
:1064A000112351F02BED3FE049EC50E4C701B60158
:1064B0000F94403C6B017C0120E030E0A901C70152
:1064C000B6010F94D737811128C0AF962CAD3DADE2
:1064D0004EAD5FADAF976B966CAD7DAD8EAD9FADA4
:1064E0006B970F94D737811118C0E3962CAD3DAD53
:1064F0004EAD5FADE397A3966CAD7DAD8EAD9FAD18
:10650000A3970F94D737811108C01BEDC12E1FE050
:10651000D12E19ECE12E10E4F12EE7962CAD3DAD15
:106520004EAD5FADE797C701B6010F943C389B01B4
:10653000AC010F943C384B015C01A7962CAD3DADEE
:106540004EAD5FADA797CA01B9010F943C389B01CE
:10655000AC01C501B4010F94413C0F94AC3E4B011A
:106560005C012FE632E143E85AE30F94D73787FD09
:1065700056C2C501B4010F94B63D0F948A3DA19651
:106580007FAF6EAFA197672B31F481E090E0A196C9
:106590009FAF8EAFA197A196AEADBFADA197BD0144
:1065A00080E090E00F94DB374B015C019B01AC0174
:1065B000C701B6010F941D3D6B966CAF7DAF8EAFDA
:1065C0009FAF6B97A5019401A7966CAD7DAD8EAD85
:1065D0009FADA7970F941D3DE7966CAF7DAF8EAF33
:1065E0009FAFE797A5019401EB966CAD7DAD8EADA5
:1065F0009FADEB970F941D3DEB966CAF7DAF8EAFCB
:106600009FAFEB976B962CAD3DAD4EAD5FAD6B97ED
:10661000CA01B9010F943C3820E030E040E05FE36C
:106620000F943C389B01AC0160E070E080E89FE390
:106630000F94403CA7966CAF7DAF8EAF9FAFA797EE
:10664000C158DF4F288139814A815B81CF57D040C3
:1066500029873A874B875C87CD57DF4F888199819F
:10666000AA81BB81C358D0408D879E87AF87B88BE6
:106670006091840270918502072E000C880B990BA3
:106680000F94DD3720912502309126024091270298
:10669000509128020F943C382AE037ED43E25CE346
:1066A0000F943C38AF966CAF7DAF8EAF9FAFAF9776
:1066B0000E94CB5C9B01AC0128533F4F4F4F5F4F73
:1066C000E3962CAF3DAF4EAF5FAFE39760964FAC14
:1066D000609761965FAC619762966FAC62976396C4
:1066E0007FAC639722242394312CB9E1DB2EA19651
:1066F0004EAD5FADA1972416350609F44CC10E943A
:1067000097FD0E94CB5CDC01CB01E3962CAD3DAD47
:106710004EAD5FADE397821B930BA40BB50BB7FD9A
:1067200011C00E94CB5C9B01AC0128533F4F4F4FDF
:106730005F4FE3962CAF3DAF4EAF5FAFE39780E086
:106740000F94E823DA94DD2009F44BC0A7962CAD12
:106750003DAD4EAD5FADA79767966CAD7DAD8EAD8F
:106760009FAD67970F943C384B015C016B962CAD45
:106770003DAD4EAD5FAD6B97B201C3010F943C3898
:10678000A50194010F94413C7B018C01A7962CAD8F
:106790003DAD4EAD5FADA797B201C3010F943C383C
:1067A0004B015C016B962CAD3DAD4EAD5FAD6B9773
:1067B00067966CAD7DAD8EAD9FAD67970F943C38FD
:1067C0009B01AC01C501B4010F94403C2B013C017D
:1067D000C701D80167968CAF9DAFAEAFBFAF6797CB
:1067E0005BC0B10180E090E00F94DB376B962CAD7D
:1067F0003DAD4EAD5FAD6B970F943C384B015C01E6
:106800000F941A3D6B017C01C501B4010F94A23EA7
:106810004B015C01A701960163966CAD7DAD8EAD19
:106820009FAD63970F943C382B013C01A501940167
:106830006F966CAD7DAD8EAD9FAD6F970F943C386C
:106840009B01AC01C301B2010F94413C2B013C01FF
:10685000A501940163966CAD7DAD8EAD9FAD639740
:106860000F943C384B015C01A70196016F966CAD0B
:106870007DAD8EAD9FAD6F970F943C389B01AC0101
:10688000C501B4010F94403C67966CAF7DAF8EAFED
:106890009FAF6797F9E1DF2E9201A301AB966CAD34
:1068A0007DAD8EAD9FADAB970F94413C69837A83EC
:1068B0008B839C8367962CAD3DAD4EAD5FAD6797E6
:1068C000EF966CAD7DAD8EAD9FADEF970F94413CD3
:1068D0006D837E838F839887E7962CAD3DAD4EAD5B
:1068E0005FADE79769857A858B859C850F94413CE0
:1068F00069877A878B879C87EB962CAD3DAD4EAD33
:106900005FADEB976D857E858F8598890F94413CAF
:106910006D877E878F87988BCE0101960F945127C4
:10692000C090FB0689819A81AB81BC8188A399A321
:10693000AAA3BBA38D819E81AF81B8858CA39DA3A3
:10694000AEA3BFA389859A85AB85BC8588A799A787
:10695000AAA7BBA7AE01485D5F4FBE016C5D7F4F2C
:10696000CE0180960E9420CAAF96ECACFDAC0EAD75
:106970001FADAF979E01235F3F4FAE01485D5F4F54
:10698000BE016C5D7F4FCE0180960E9408BC3FEF38
:10699000231A330AACCEC090FB068091970F9091DA
:1069A000980FA091990FB0919A0F88A399A3AAA3C9
:1069B000BBA380919B0F90919C0FA0919D0FB091D4
:1069C0009E0F8CA39DA3AEA3BFA380919F0F909118
:1069D000A00FA091A10FB091A20F88A799A7AAA775
:1069E000BBA7AE01485D5F4FBE016C5D7F4FCE011E
:1069F00080960E9420CAAF96ECACFDAC0EAD1FADE8
:106A0000AF9723EA3FE0AE01485D5F4FBE016C5D8A
:106A10007F4FCE0180960E9408BC0E9424AC0E9449
:106A2000D75C0C941A48E2EEF1E284918F010F5F7B
:106A30001F4F882321F00F94452EF801F6CFEBEC81
:106A4000F2E084918F010F5F1F4F882311F40C94A3
:106A50001A480F94452EF801F4CF0E94088D0C942B
:106A60001A4881E0809373021092F3090C941A483B
:106A70000E946F7481110C941A4880E50E949DB1A8
:106A8000882321F00E9407B1262F01C020E06091E9
:106A90003A0770913B0780913C0790913D07C12CCC
:106AA000D12C30EEE32E30E4F32EC982DA82EB8271
:106AB000FC82C12CD12C44E3E42E43E4F42ECD829D
:106AC000DE82EF82F886C12CD12C50EAE52E51E40B
:106AD000F52EC986DA86EB86FC86C12CD12CE0EC3B
:106AE000EE2EEFE7FE2ECD86DE86EF86F88A213089
:106AF00071F1223021F518A219A21AA21BA220E0DE
:106B000030E040EA51E40F94413C6B017C0120E00D
:106B100030E047E353E40F94673E181634F4C12C79
:106B2000D12C97E3E92E93E4F92ECBAEDCAEEDAE9B
:106B3000FEAEBE01605E7F4FCE01CB9611C020E05D
:106B400030E040EA51E40F94D73787FF0BC018A21A
:106B500019A21AA21BA2BE01605E7F4FCE01099648
:106B60000E9413AC18A219A21AA21BA2AE01405E89
:106B70005F4FBE016B5F7F4FCE0101960E940FAC4D
:106B80000C941A4880E00E94A78B0C941A4881E06C
:106B900080938F0424982C9A149A0E946E7D1092F0
:106BA0008F04249A2C9814980C941A4820E030E012
:106BB000A901609132077091330780913407909159
:106BC00035070F94413C6B017C0188E50E949DB123
:106BD000882321F00E9437B16B017C01C8A2D9A2A1
:106BE000EAA2FBA220E030E0A90160913607709193
:106BF000370780913807909139070F94413C6B011A
:106C00007C0189E50E949DB1882321F00E9437B163
:106C10006B017C01C982DA82EB82FC824090090719
:106C200050900A0760900B0770900C0720910507A1
:106C300030910607409107075091080768A179A194
:106C40008AA19BA10F94403C4B015C0122E630E1FC
:106C500040E450EC0F94673E87FF02C00C941A4842
:106C600022E430E042E253E4C501B4010F94D73787
:106C7000181614F40C941A48A3019201C701B60126
:106C80000F94403C6B017C0121E338E040EE50EC76
:106C90000F94673E87FF02C00C941A4822E430E04C
:106CA0004EE353E4C701B6010F94D737181614F416
:106CB0000C941A480C942D4881E0809379040C942C
:106CC0001A480E942F7D0C941A4880917A04909162
:106CD0007B048D37910509F489C70CF0E6C08E342A
:106CE000910509F4D3C40CF05AC08931910509F417
:106CF00085C234F58431910509F4FEC194F48131E3
:106D0000910509F4EEC144F4029710F00C941A486E
:106D10000E949E7C0C941A48429709F4E7C70C9491
:106D20001A488631910509F42EC20CF428C2873125
:106D3000910509F42EC2489709F441C20C941A48EF
:106D40008F31910509F416C47CF48B31910509F457
:106D500073C20CF463C28C31910509F4A9C24E9739
:106D600009F4B0C20C941A488B34910509F484C418
:106D70004CF48032910509F4B3C38A9709F426C410
:106D80000C941A488C34910509F47AC48D34910519
:106D900011F00C941A480E94EEDA0C941A488B36C3
:106DA000910509F411C7DCF58535910509F4A2C7F1
:106DB000C4F48235910509F490C74CF481359105EE
:106DC00011F00C941A480E943DB30C941A48833574
:106DD000910509F486C78435910509F487C70C9499
:106DE0001A488836910509F461C57CF48C35910503
:106DF00011F00C941A481AE5C12E13E0D12E02E4CA
:106E0000E02E07E0F02E10E079C78936910509F4ED
:106E100073C68A36910509F4B8C60C941A488337AC
:106E2000910509F4EBC7ECF48E36910509F490C591
:106E30004CF48D36910511F00C941A480E947BB6E3
:106E40000C941A488F36910509F495C5823791053F
:106E500011F00C941A480E94CAFF0E9421B20C94AF
:106E60001A488737910511F40C94993F74F48537CB
:106E7000910511F40C94903F8637910511F00C9414
:106E80001A480E9439950C941A488837910511F4D4
:106E90000C94A83F8937910511F00C941A48109270
:106EA0008E0410928D040C941A48833651E0950795
:106EB00011F40C94BB470CF083C08D3C910511F488
:106EC0000C94BF3FCCF58E3B910509F45AC6BCF437
:106ED0008139910511F40C94AF3F34F48C3891054D
:106EE00009F4ECC50C941A488639910511F40C94F8
:106EF000B33F8B39910509F419C60C941A48893CA3
:106F0000910511F40C94B73F4CF4883C910511F0B5
:106F10000C941A480E9493940C941A488B3C910547
:106F200011F40C94BB3F8C3C910511F00C941A4861
:106F30000E94E7930C941A48823E910511F40C9438
:106F4000CB3FECF4833D910511F40C94C33F4CF41A
:106F50008E3C910511F00C941A480E9428930C94D1
:106F60001A488C3D910511F40C94C73F8D3D910555
:106F700011F00C941A480E9471920C941A488E32A7
:106F8000B1E09B0711F40C9413416CF48C32F1E0E6
:106F90009F0711F40C94CF3F8D32914011F40C9463
:106FA000F93F0C941A488F3231E0930711F40C9496
:106FB00067418033914011F40C9496400C941A4828
:106FC0008C3152E0950711F40C9468460CF041C0E6
:106FD0008C3AB1E09B0711F40C946645ECF48139CE
:106FE000F1E09F0711F40C940A454CF4803991406C
:106FF00011F00C941A480E94CAFF0C941A48823966
:1070000041E0940711F40C940E45843A914011F438
:107010000C9412450C941A48853FA1E09A0711F48C
:107020000C9454464CF4843F914011F00C941A484F
:107030000E940CE20C941A48863FF1E09F0711F47D
:107040000C945746873F914011F40C945A460C9487
:107050001A488F3833E0930711F40C94B247ECF4DC
:10706000833553E0950711F40C9473463CF488354E
:10707000924011F40C94A9460C941A488A38E3E023
:107080009E0711F40C94AF478B38934011F00C9489
:107090001A480E94548F0C941A48823923E09207B0
:1070A00011F40C94B8477CF4803943E0940711F450
:1070B0000C94B5478139934011F00C941A480E9402
:1070C000BC8F0C941A48803AA3E09A0709F445C291
:1070D000873E934011F00C941A480E94288F0C941C
:1070E0001A4860E083EF92E00E94C5EC179816986A
:1070F000159814980C941A48EBE0F3E084918F01F2
:107100000F5F1F4F882321F00F94452EF801F6CF13
:1071100010925B0F40E050E0BA0187E09DE00E94D2
:10712000E3CD8BE1E7E0FDE0DE01159601900D92E5
:107130008A95E1F78091050D9091060D9C838B83D4
:1071400082EC93E09A83898340E050E0BE016F5F58
:107150007F4F81EF93E00E9440A2CE0101960E94F2
:107160006EF5ECEFF2E084918F010F5F1F4F8823E3
:1071700011F40C941A480F94452EF801F4CF0E9494
:107180009CA70C941A481092AF0C1092B00C0C945F
:107190001A48E0916604F09167048081882329F001
:1071A000803209F410823196F8CF40E061E080919E
:1071B0006604909167040E946FA40C941A48198287
:1071C0001A821B821C8218A219A21AA21BA28091E9
:1071D000B80F882341F040E0BE016F5F7F4FCE01C2
:1071E00080960E94CDF28091B00C882319F081E046
:1071F0008093AF0C0E941C740C941A481092AF0C30
:1072000085E89CE00E94AC9E8CE193E090936B0932
:1072100080936A090E941CAD0C941A488091B00CAE
:10722000882311F40C941A4883E50E949DB18111C2
:107230000C9483480C941A488091B00C882351F127
:10724000E1E2F3E084918F010F5F1F4F882321F06B
:107250000F94452EF801F6CF6091520F7091530FA5
:107260008091540F9091550F4AE00F949E2E8FE21B
:107270000F94452E60914E0F70914F0F8091500FDB
:107280009091510F4AE00F949E2E8AE00F94452E64
:107290000C941A48E3E3F3E084918F010F5F1F4FD2
:1072A000882311F40C941A480F94452EF801F4CF5A
:1072B00040E060E080916604909167040E946FA4B2
:1072C0000C941A488091B00C882311F40C941A483D
:1072D00081EA9EE00E94E5CE81EA9EE00E9416CF00
:1072E0001092AE0C1092AD0CE0906604F090670422
:1072F0008091B00C882311F40C941A480E94C8DACB
:107300001D8218861C821B8282EC93E09A838983FB
:1073100083E09DE09093230D8093220DF7018081FF
:107320008F3209F068C06FE270E0C7010F946240CD
:107330008C010F5F1F4F9E012F5F3F4F49010115C9
:10734000110509F45EC06FE270E0C8010F9462405D
:107350006C01009709F456C00817190708F052C0CD
:107360005C01A01AB10AA501B801CE0180960F9464
:107370008240E0E2F0E0EC0FFD1FEA0DFB1D108201
:107380008E01005E1F4FD8018D918D01882319F069
:107390000F94452EF8CF8AE00F94452E6091220D70
:1073A0007091230D6115710511F06C5F7F4F21E025
:1073B000AE01405E5F4FCE0105960E9420D581113F
:1073C00012C0BE01605E7F4F8AE693E00E9434994E
:1073D0008EE20F94452E8AE00F94452EC4010E9440
:1073E0006EF50C941A489092230D8092220D86011E
:1073F0000F5F1F4FA4CF84E29DE09093230D8093F5
:10740000220D87016091220D7091230D6115710588
:1074100011F06C5F7F4F18A21BA222E0A801CE01E1
:1074200080960E9420D5811102C0F12C14C0CE019B
:1074300080960E9436DA8823C1F361E0CE018096FF
:107440000E94CACE009789F325EEFC0120831BA27F
:107450000E94F4CAF82ECE0180960E942156FF2089
:1074600009F1E4E4F3E084917F012FEFE21AF20ADC
:10747000882321F00F94452EF701F5CFD8018D9187
:107480008D01882319F00F94452EF8CF8AE00F94D0
:10749000452E1092520F1092530F1092540F1092CB
:1074A000550F18C0E2E5F3E084917F01BFEFEB1ABE
:1074B000FB0A882321F00F94452EF701F5CFF80140
:1074C00081918F01882319F00F94452EF8CF8EE219
:1074D0000F94452ECE0101960E946EF50C941A4829
:1074E0008091AF0C81110E94CAFFE0906604F09079
:1074F000670480E50E946EB1182F882319F00E945E
:1075000028B1182F8091B00C882311F40C941A48DC
:10751000412F61E0C7010E946FA483E50E949DB1E5
:10752000882381F00E9407B1AB01BC014093520F48
:107530005093530F6093540F7093550F81EA9EE060
:107540000E94E3CD8091B00C882319F081E08093F4
:10755000AF0C11110C941A484DCE80916604909195
:10756000670421E02093AE0C40E060E00E946FA42D
:107570000C941A4885E89CE00E94809E68A379A339
:107580008AA39BA3BE016F5F7F4FCE0180960E94AE
:10759000615560E0CE0101960E94E3ECEDEFF1E26F
:1075A00084918F010F5F1F4F882321F00F94452E88
:1075B000F801F6CFBE016F5F7F4F8EE793E00E9428
:1075C00034998AE00F94452E0C941A4883E50E9462
:1075D0009DB1882311F40C941A480E9417B1E82E2B
:1075E00080E50E949DB1811112C081E0E11001C0CF
:1075F00080E080938F04882329F024982C9A149A91
:107600000C941A48249A2C9814980C941A4880E5E3
:107610000E949DB1882339F00E9407B18B0177FF4A
:1076200004C00C941A480DE010E0902FEBE8F3E052
:1076300088E28E0F2491921729F031968E13FACF9B
:107640000C949448E2EEF1E284918F010F5F1F4F9A
:10765000882321F00F94452EF801F6CFE3EBF3E0F9
:1076600084918F010F5F1F4F882311F40C941A48E7
:107670000F94452EF801F4CF0E941C740C941A4804
:1076800085E89CE00E94AC9E0C941A4883E50E9419
:107690009DB1882359F00E9407B16E34710531F411
:1076A00085E89CE00E948A9B0C941A4818A219A2B3
:1076B0001AA21BA2E2E2F4E084918F010F5F1F4F38
:1076C000882321F00F94452EF801F6CFE9E1F4E08C
:1076D00084918F010F5F1F4F882321F00F94452E57
:1076E000F801F6CF6091920C7091930C80E090E0DD
:1076F0004AE00F949E2EECE0F4E084918F010F5F3E
:107700001F4F882321F00F94452EF801F6CF60918A
:10771000940C7091950C80E090E04AE00F949E2EBE
:10772000E1E0F4E084918F010F5F1F4F882321F087
:107730000F94452EF801F6CF6091920C7091930C46
:107740008091940C9091950C681B790B8091850C1D
:10775000815021E030E0823010F020E030E0621B08
:10776000730B80E090E04AE00F949E2E8AE00F9425
:10777000452EE9EFF3E084918F010F5F1F4F8823BF
:1077800021F00F94452EF801F6CF8091960C909140
:10779000970CA091980CB091990C88A399A3AAA3D7
:1077A000BBA3BE016F5F7F4FCE0180960E946155E3
:1077B000ECEEF3E084918F010F5F1F4F811106C043
:1077C0009E012F5F3F4F7901890104C00F94452E20
:1077D000F801F0CFD8018D918D01882319F00F9415
:1077E000452EF8CF80919A0C90919B0CA0919C0C07
:1077F000B0919D0C88A399A3AAA3BBA3BE016F5F00
:107800007F4FCE0180960E946155ECEDF3E08491AC
:107810008F010F5F1F4F882321F00F94452EF80131
:10782000F6CFF70181917F01882319F00F94452E3F
:10783000F8CF8AE00F94452EE4EDF3E084918F01B8
:107840000F5F1F4F882321F00F94452EF801F6CFCC
:10785000E4ECF3E084918F010F5F1F4F882321F048
:107860000F94452EF801F6CF20E030E04AE754E4CB
:1078700060919E0C70919F0C8091A00C9091A10C36
:107880000F941D3D42E00F941E2FE2ECF3E0849133
:107890008F010F5F1F4F882321F00F94452EF801B1
:1078A000F6CF8AE00F94452E0C941A4888E690E0B3
:1078B0000E94A9B181110C941A488091F31683FF9C
:1078C00002C00C941A4883E50E949DB1882311F4EC
:1078D0000C941A480E9437B10F94853D709371063D
:1078E0006093700680E00E945BFA0E9437B120E04E
:1078F00030E040E752E40F94D73718163CF00E946E
:10790000EEDA60E086E394E00E94C5EC0E9437B1B5
:1079100020914A1530914B1540914C1550914D15C1
:107920000F94673E181614F00C941A4882E093E006
:107930009F938F938AE294E09F938F931F920E946C
:10794000D3DA0F900F900F900F900F900C941A486D
:107950008EE40E949DB1882311F40C941A480E9471
:1079600007B1609398157093991580939A15909329
:107970009B150C941A4883E50E949DB1882319F049
:107980000E9417B101C080E08093F316EDEFF1E2A1
:1079900084918F010F5F1F4F882321F00F94452E94
:1079A000F801F6CFEEE5F4E084918F010F5F1F4FF1
:1079B000882321F00F94452EF801F6CF8091F3161D
:1079C0008823A1F180E5C82E84E0D82EE12CF12C8B
:1079D00020E08091F31690E00E2C02C095958795DB
:1079E0000A94E2F780FF17C0BB24B394B20E22239F
:1079F00019F08CE20F94452EF60125913491F9018E
:107A0000849189010F5F1F4F882321F00F94452E29
:107A10009801F5CF2B2DFFEFEF1AFF0A32E0C30ECE
:107A2000D11C45E0E416F104A1F643C0EAE5F4E018
:107A300084918F010F5F1F4F8823D9F10F94452E3A
:107A4000F801F6CF8AE50E946EB1882311F40C94F8
:107A50009B460E9437B16B017C0120E030E040E0A2
:107A600050EC0F94673E87FF02C00C948D4620E0D7
:107A700030E040EA50E4C701B6010F94D73718163A
:107A800014F40C948D46C0921E07D0921F07E0920A
:107A90002007F092210780E00E94969160911E07D6
:107AA00070911F07809120079091210742E00F9469
:107AB0001E2F8AE00F94452E0C941A488091F316DD
:107AC00083FF02C00C941A4883E50E949DB188236D
:107AD00011F40C941A480E9437B10F94853D673910
:107AE000710514F066E970E070936F0660936E069E
:107AF0000E9410FA0C941A4889E690E00E94A9B1FD
:107B000081110C945F4AE5E6F4E084918F010F5FE8
:107B10001F4F882321F00F94452EF801F6CF0E94C5
:107B2000C1B38AE00F94452E0C945F4A83E50E940E
:107B30009DB1882311F40C941A480E9417B18093C8
:107B4000A1158D3318F08CE38093A1150E94CB5CB6
:107B50006B017C012091A11530E0A8EEB3E00F94F9
:107B6000313CDC01CB018C0D9D1DAE1DBF1D8093F2
:107B70009D1590939E15A0939F15B093A0150C94FE
:107B80001A480E9444B40C941A4883E50E949DB19F
:107B9000882339F00E9407B18B016F3F710519F0FE
:107BA00010F00FEF10E080E50E949DB1811106C03A
:107BB00010936D0600936C060C941A480E9417B13E
:107BC00081110C941A48F4CF80E50E949DB1811177
:107BD00006C010926D0610926C060C941A480E9412
:107BE00007B1672B11F00C941A48F3CF8CE40E9474
:107BF0006EB1882319F00E9437B104C060E070E0D4
:107C000080E090EC27966CAF7DAF8EAF9FAF27974B
:107C10008AE50E949DB1882319F00E9437B103C004
:107C200060E070E0CB0120E030E040E251E40F94EE
:107C3000413C23966CAF7DAF8EAF9FAF239788E515
:107C40000E949DB1882319F00E9437B103C060E003
:107C500070E0CB0120E030E040E251E40F94413C81
:107C60006BAF7CAF8DAF9EAF89E50E949DB188233D
:107C700019F00E9437B103C060E070E0CB0120E052
:107C800030E04EE353E40F94413C20E030E040E22A
:107C900051E40F94403C68A379A38AA39BA3198263
:107CA0001A821B821C828091B80F81110C941A4891
:107CB000C12CE12C8E010F5F1F4F9E01205E3F4FB4
:107CC000AE01455C5F4FBE01615C7F4FCE018D5BB5
:107CD0009F4F0E945BF10C941A48109278040C9408
:107CE0001A4881E0809378040C941A480E94F6B2F6
:107CF0000C941A480E94E0B20C941A48D6018D9157
:107D00006D010E946EB1882309F46DC0133009F033
:107D100063C00E9437B14B015C0120E030E040EAD3
:107D200051E40F94D73787FF4EC0A50194016091AD
:107D30004E0770914F0780915007909151070F9413
:107D40001D3D2B013C019B01AC0160912D107091F8
:107D50002E1080912F10909130100F943C3860932A
:107D60002D1070932E1080932F1090933010A3013C
:107D700092016091870670918806809189069091A2
:107D80008A060F943C386093870670938806809328
:107D9000890690938A0660915210709153108091D9
:107DA0005410909155100F94DB37A30192010F945A
:107DB0003C380F948A3D6093521070935310809317
:107DC00054109093551080924E0790924F07A092B6
:107DD0005007B092510707C00E9437B1F701608386
:107DE0007183828393831F5FF4E0EF0EF11C1430E4
:107DF00009F084CF0F94B7150C941A48E3E4F5E02A
:107E000084918F010F5F1F4F882321F00F94452E1F
:107E1000F801F6CFE5E3F5E084918F010F5F1F4F86
:107E2000882321F00F94452EF801F6CFEEE1F5E01E
:107E300084918F010F5F1F4F882321F00F94452EEF
:107E4000F801F6CFEEE0F5E084918F010F5F1F4F50
:107E5000882321F00F94452EF801F6CFEDEFF4E0E2
:107E600084918F010F5F1F4F882321F00F94452EBF
:107E7000F801F6CFECEEF4E084918F010F5F1F4F15
:107E8000882321F00F94452EF801F6CFEDEDF4E0B4
:107E900084918F010F5F1F4F882321F00F94452E8F
:107EA000F801F6CFE8ECF4E084918F010F5F1F4FEB
:107EB000882321F00F94452EF801F6CFE2EBF4E091
:107EC00084918F010F5F1F4F882321F00F94452E5F
:107ED000F801F6CFEDE9F4E084918F010F5F1F4FB9
:107EE000882321F00F94452EF801F6CFE0E8F4E066
:107EF00084918F010F5F1F4F882321F00F94452E2F
:107F0000F801F6CFE8E6F4E084918F010F5F1F4F90
:107F1000882311F40C941A480F94452EF801F4CFDD
:107F200060E080916604909167040E94E3EC0C94F9
:107F30001A4881E080938F0424982C9A149A0E9406
:107F4000794A10928F04249A2C9814980C941A4809
:107F500081E080938E0480938D040C941A480E94D3
:107F600052B30C941A480E94E0940C941A480E9450
:107F70006E940C941A480E944C940C941A480E94D7
:107F80007D930C941A480E9498920C941A480E946F
:107F90008C920C941A480E9426920C941A4883E5FD
:107FA0000E949DB1882319F00E9407B102C064E0CD
:107FB00071E079A368A380E50E949DB1882339F020
:107FC0000E9407B1693823E1720730F402C068EEFD
:107FD00073E07A83698304C088E893E19A83898394
:107FE000BE01605E7F4FCE0101960E94E6A80C9410
:107FF0001A4885E40E949DB1811110C080E50E945D
:108000006EB1882391F00E9437B160937F15709311
:108010008015809381159093821507C00E9417B137
:10802000882361F3E2EEF1E270C089E40E946EB150
:10803000882381F00E9437B12CEA35EC47E25EE3F9
:108040000F943C3860937B1570937C1580937D155D
:1080500090937E1584E40E946EB1882381F00E9483
:1080600037B12CEA35EC47E25EE30F941D3D609397
:108070007715709378158093791590937A150DEF95
:1080800011E2F8018491882329F00F5F1F4F0F94AC
:10809000452EF7CF40917F15509180156091811545
:1080A0007091821585E496E00E94D7982CEA35EC11
:1080B00047E25EE360917B1570917C1580917D15A0
:1080C00090917E150F941D3DAB01BC0181E496E0BB
:1080D0000E94BA982CEA35EC47E25EE3609177158E
:1080E000709178158091791590917A150F943C389C
:1080F000AB01BC018DE396E00E94BA988AE00F9430
:10810000452E98C70F94452EF80184918F010F5F7B
:108110001F4F8111F7CF0DE013E0D8018D918D0134
:10812000882309F4C6CC0F94452EF7CF80E50E9432
:108130006EB1882351F00E9437B16093731570932C
:108140007415809375159093761589E40E946EB12D
:10815000882381F00E9437B12CEA35EC47E25EE3D8
:108160000F943C3860936F15709370158093711560
:108170009093721584E40E946EB1882381F00E946E
:1081800037B12CEA35EC47E25EE30F941D3D609376
:108190006B1570936C1580936D1590936E15EDEFC4
:1081A000F1E284918F010F5F1F4F882321F00F941C
:1081B000452EF801F6CF40917315509174156091DA
:1081C00075157091761581E596E00E94D7982CEA96
:1081D00035EC47E25EE360916F1570917015809108
:1081E0007115909172150F941D3DAB01BC018DE48A
:1081F00096E00E94BA982CEA35EC47E25EE3609183
:108200006B1570916C1580916D1590916E150F9492
:108210003C38AB01BC0189E496E00E94BA988AE040
:108220000F94452E07C783E50E946EB1182F88234F
:1082300071F00E9437B10F94853D70937F02609377
:108240007E0221E0672B09F020E020934E1580E5A7
:108250000E946EB1882359F020917E0230917F02F6
:10826000232B11F00E9428B180934E15E3C6111103
:10827000E1C6EDEFF1E284918F010F5F1F4F88237C
:1082800021F00F94452EF801F6CF80914E15811103
:1082900003C062EF72E002C060E673E08AE696E037
:1082A0000E94349960917E0270917F0289E596E088
:1082B0000E941B99E5E5F6E084918F010F5F1F4F47
:1082C000882309F4B7C60F94452EF801F5CF85E44D
:1082D0000E949DB1882321F00E9407B11B0102C0BA
:1082E000212C312C83E40E949DB1882349F00E9407
:1082F00007B1CA56DF4F79836883C659D04008C09A
:10830000E5E0F0E0CA56DF4FF983E883C659D04074
:1083100085E50E946EB1C457DF4F8883CC58D040AA
:10832000882339F00E9428B1C457DF4F8883CC5886
:10833000D04037FC07C0C12CD12CB6E1EB2EB3E402
:10834000FB2E06C0C12CD12CACE8EA2EA2E4FA2EFA
:1083500083E50E949DB1882321F00E9437B16B0113
:108360007C012114310411F4109268040E94CB5C4A
:108370002B013C01C1010196029718F40EE113E0B4
:108380000BC001E313E0D8018D918D01882309F41E
:1083900090CB0F94452EF7CFF80181918F01882360
:1083A00019F00F94452EF8CF8AE00F94452E0E94C5
:1083B000A6FA8FE7FFEF2F163F0619F480931D10E2
:1083C00002C080931F10C701B6010F94853D072E90
:1083D000000C880B990B0F94DD37EC966FAFEC9780
:1083E000AC967FAFAC97E0968FAFE097C158DF4F68
:1083F0009883CF57D04081E08093A502C257DF4FCA
:10840000488259826A827B82CE58D040C856DF4F5C
:10841000488259826A827B82C859D040CD57DF4F4B
:108420001882C358D04020E4E4962FAFE4973CE193
:10843000E8963FAFE89746E4C957DF4F4883C758EF
:10844000D040C857DF4F1882C858D040C757DF4FB9
:108450001882C958D040C657DF4F1882CA58D0403A
:10846000C557DF4F1882CB58D040AB961CAE1DAE1F
:108470001EAE1FAEAB97A7961CAE1DAE1EAE1FAEB6
:10848000A797C12CD12C7601FFE78F2E912CA12C20
:10849000B12C8FE790E0A0E0B0E06B968CAF9DAF81
:1084A000AEAFBFAF6B97CE56DF4F188219821A82DC
:1084B0001B82C259D04091E0C357DF4F9883CD58FB
:1084C000D040A1961FAE1EAEA19760961FAE6097DA
:1084D00064961FAE649700E010E08091A5028823A7
:1084E00009F491C20E94CB5C6F966CAF7DAF8EAFEA
:1084F0009FAF6F9780910D10882309F436C10E94B9
:1085000063FBAFEF2A163A0679F4B091CE06609677
:10851000BFAF6097E091CF066496EFAF649700918C
:10852000D0061091D1060EC0F0914A156096FFAFAB
:10853000609720914B1564962FAF649700914C156E
:1085400010914D1560962FAD609764963FAD64977E
:10855000A801C857DF4F6881C858D040C757DF4FC0
:108560007881C958D040C657DF4F8881CA58D0405B
:10857000C557DF4F9881CB58D0400F94D73787FF2E
:108580001AC060963FAD6097C857DF4F3883C85810
:10859000D04064964FAD6497C757DF4F4883C958A2
:1085A000D040C657DF4F0883CA58D040C557DF4F69
:1085B0001883CB58D04060962FAD609764963FAD3E
:1085C0006497A801CD57DF4F6881C358D040E49627
:1085D0007FADE497E8968FADE897C957DF4F988154
:1085E000C758D0400F94673E1816B4F460965FAD3C
:1085F0006097CD57DF4F5883C358D04064968FADF6
:108600006497E4968FAFE497E8960FAFE897C95761
:10861000DF4F1883C758D040C357DF4F9881CD58DC
:10862000D040EC962FADEC97AC963FADAC97E09672
:108630004FADE097C158DF4F5881CF57D04060967B
:108640006FAD609764967FAD6497802F992309F48E
:108650006DC0912F0F94673E18160CF086C06F9670
:108660004CAD5DAD6EAD7FAD6F9744195509660990
:108670007709DB01CA0188589341A109B109B7FD07
:1086800074C06B968CAD9DADAEADBFAD6B978819C8
:108690009909AA09BB09B595A79597958795EFEF15
:1086A0002E163E0619F480931D1002C080931F10F1
:1086B000CE56DF4F488359836A837B83C259D040AB
:1086C000EC96FFADEC97C857DF4FF883C858D04001
:1086D000AC962FADAC97C757DF4F2883C958D04011
:1086E000E0963FADE097C657DF4F3883CA58D04079
:1086F000C158DF4F4881CF57D040C557DF4F48831F
:10870000CB58D0406F968CAD9DADAEADBFAD6F97E1
:10871000C257DF4F88839983AA83BB83CE58D0404A
:10872000C357DF4F1882CD58D0401FC0912F0F94F0
:10873000D73787FF1AC06F968CAD9DADAEADBFAD7C
:108740006F97C257DF4F288139814A815B81CE58AC
:10875000D040821B930BA40BB50BAC01BD01485854
:1087600053416109710977FFF5C420E030E040EA28
:1087700051E4EC966FADEC97AC967FADAC97E0967C
:108780008FADE097C158DF4F9881CF57D0400F94FD
:10879000413C9B01AC0160966FAD609764967FADE4
:1087A0006497C8010F94673E18166CF4EAE3F7E08B
:1087B00084918F010F5F1F4F882309F43BC40F94EE
:1087C000452EF801F5CF80E398EFAFEFBFEFC85625
:1087D000DF4F288139814A815B81C859D040821B93
:1087E000930BA40BB50B6F962CAD3DAD4EAD5FADAD
:1087F0006F97820F931FA41FB51FB7FD13C00E9470
:10880000C1B38AE00F94452E6F968CAD9DADAEAD91
:10881000BFAD6F97C856DF4F88839983AA83BB8308
:10882000C859D0406F968CAD9DADAEADBFAD6F97C2
:10883000880F991FAA1FBB1FC257DF4F288139819C
:108840004A815B81CE58D040821B930BA40BB50BA1
:1088500084199509A609B70981389F44A241B10539
:1088600068F0ECE1F7E084918F010F5F1F4F8823E0
:1088700009F4E0C30F94452EF801F5CFA1964EAD53
:108880005FADA197CA56DF4F88819981C659D04004
:10889000841795070CF0B4C0EFEBF6E084918F01DC
:1088A0000F5F1F4F882321F00F94452EF801F6CF5C
:1088B0009FEF2916390619F001EF13E002C006EF09
:1088C00012E0B8018DEA96E00E943499B701A60142
:1088D00089EA96E00E94D7988AE00F94452EB80165
:1088E00087E996E00E943499A7964CAD5DAD6EADD8
:1088F0007FADA79783E996E00E94D7988AE00F940E
:10890000452EB80181E896E00E943499AB964CADB3
:108910005DAD6EAD7FADAB978DE796E00E94D798C9
:108920008AE00F94452EC457DF4FA881CC58D04021
:10893000AA2309F47FC32320209489F5C0927315DC
:10894000D0927415E0927515F09276152CEA35ECFC
:1089500047E25EE3A7966CAD7DAD8EAD9FADA79768
:108960000F943C3860936F15709370158093711558
:10897000909372152CEA35EC47E25EE3AB966CAD52
:108980007DAD8EAD9FADAB970F941D3D60936B1584
:1089900070936C1580936D1590936E154BC3C092B8
:1089A0007F15D0928015E0928115F09282152CEA05
:1089B00035EC47E25EE3A7966CAD7DAD8EAD9FAD25
:1089C000A7970F943C3860937B1570937C15809328
:1089D0007D1590937E152CEA35EC47E25EE3AB966D
:1089E0006CAD7DAD8EAD9FADAB970F941D3D60938B
:1089F0007715709378158093791590937A151AC32B
:108A00000E94F3EC6ACD8091A502811113C30E94EC
:108A1000A6FA10C381E00E94C9AB0CC380E00E949B
:108A2000C9AB08C386E50E946EB1882321F08BEDA7
:108A300097E00E94A67583E50E946EB1182F8823E7
:108A400019F00E9428B1182F83E50E946EB1882387
:108A500019F0812F0E946BAAF0905D15111103C0CF
:108A6000EDEFF1E21AC0F110FBCFE2EEF1E28491FA
:108A70008F010F5F1F4F882321F00F94452EF801BF
:108A8000F6CFECEBF7E084918F010F5F1F4F882347
:108A900039F30F94452EF801F6CF84918F010F5FC3
:108AA0001F4F882321F00F94452EF801F6CFF110C7
:108AB00003C06EEF72E002C06AEF72E08EEA97E0E8
:108AC0000E9434998AE00F94452EB4C290E9C92ED1
:108AD00094E0D92E22E3E22E27E0F22E32ED232E6F
:108AE00036E0332E00E010E0E22DE0956096EFAF27
:108AF0006097D1018D911D01882309F4A3C0F7016E
:108B00004080518062807380F801EA57FD4F2081D8
:108B1000318142815381F801E759FB4F60817181B6
:108B2000828193810F94413C20E030E040E05FE39C
:108B30000F943C389B01AC01C301B2010F94673E16
:108B4000181644F4F801E354F04D85909590A590E3
:108B5000B49003C0812C912C5401F801EB5FF84FC5
:108B60002081318142815381C301B2010F94403C85
:108B70009B01AC01C501B4010F94403C4B015C0169
:108B800020E030E040EA51EC0F94673E87FD2BC0B7
:108B900020E030E040EA51E4C501B4010F94D7373A
:108BA00018160CF1D6012D913D914D915C91C501A6
:108BB000B4010F94403C9B01AC01C301B2010F947E
:108BC000413CF7016083718382839383D6018D9248
:108BD0009D92AD92BC92139760968FAD6097820D77
:108BE0000E9489AC2FC0E2EEF1E284918F010F5F09
:108BF0001F4F882321F00F94452EF801F6CFE6E1B0
:108C0000F8E084918F010F5F1F4F882321F00F94AC
:108C1000452EF801F6CF61E088E098E00E94C5ECAF
:108C20000E945C6D88E290E09A83898388EC90E0F2
:108C300099A388A3BE016F5F7F4FCE0180960E94EB
:108C4000E6A8F8C1B4E0CB0ED11C0C5F1F4FE4E0E6
:108C5000EE0EF11C0C30110509F04BCF0E9417B03D
:108C60000E9421B260E088EF97E00E94C5EC83E9A2
:108C700092E099A388A304E610E01A830983BE0159
:108C8000605E7F4FCE0101960E94E6A88AEB92E0DB
:108C900099A388A31A830983BE01605E7F4FCE012A
:108CA00001960E94E6A8C6C10E948ADCC3C10F9447
:108CB000C721C0C183E50E946EB1882319F00E94CC
:108CC00028B101C081E091E089270F94EE1CB2C168
:108CD00083E50E946EB1882309F4ACC10E9428B1DB
:108CE0008093C504A7C1EDEFF1E284918F010F5F7E
:108CF0001F4F882321F00F94452EF801F6CFECE4A6
:108D0000F8E084918F010F5F1F4F882311F40C94BA
:108D1000223D0F94452EF801F4CFE7E3F8E084916B
:108D20008F010F5F1F4F882311F40C94593D0F944E
:108D3000452EF801F4CF40911E0750911F07609116
:108D400020077091210784E398E00E94D7980C9443
:108D5000593D0E946F74882319F081E00E94A78B0F
:108D600085E40E946EB1882319F00E9437B104C0D7
:108D700060E070E080E090EC2F966CAF7DAF8EAF3E
:108D80009FAF2F978AE50E949DB1882319F00E941A
:108D900037B104C060E070E080E291E42B966CAFE4
:108DA0007DAF8EAF9FAF2B9788E50E949DB1882342
:108DB00019F00E9437B104C060E070E080E291E4F5
:108DC00027966CAF7DAF8EAF9FAF279789E50E9446
:108DD0009DB1882319F00E9437B104C060E070E0B3
:108DE00084E393E423966CAF7DAF8EAF9FAF239760
:108DF00085E50E946EB1882319F00E9437B104C046
:108E000060E070E088EC92EC6BAF7CAF8DAF9EAF12
:108E10008CE40E946EB1882319F00E9437B103C020
:108E200060E070E0CB0168A379A38AA39BA382E4EE
:108E30000E949DB1882321F00E9407B1F62E02C046
:108E400085E0F82ED090850C8091B80F811181C0FB
:108E5000CC24C394EF2C8E01055C1F4F9E01215C36
:108E60003F4FAE014D5B5F4FBE01695B7F4FCE014F
:108E7000855B9F4F0E945BF1882309F46AC081E003
:108E80008093810F11E08091810F882309F44DC0F8
:108E900060E08F2D0E9436B980917509882309F40E
:108EA00040C010936E0F40E050E0BA0188E091E0BE
:108EB0000E94396D8091810F882321F081E00F9409
:108EC000E823F8CF1092F90F1092FA0F1092FB0FCF
:108ED0001092FC0F109275090E945BFA0E94D7B89D
:108EE00010936E0F40E050E0BA0182EE90E00E94D5
:108EF000396D0E94CB5CDC01CB0188539045AF4FAC
:108F0000BF4F8093F90F9093FA0FA093FB0FB0938C
:108F1000FC0F109275091093810F61E08F2D0E9454
:108F200036B981E00F94E823AECF80E090E0A8E46A
:108F3000B2E489839A83AB83BC838091B80F882382
:108F400041F04F2DBE016F5F7F4FCE0180960E9492
:108F5000CDF2F1E0DF126EC00E941C746BC00E9463
:108F60002C9168C00E94D99065C00E94869062C012
:108F70000E94928F5FC00E94398F5CC0F0907A048B
:108F8000FF2029F1EDEFF1E284918F010F5F1F4F78
:108F9000882321F00F94452EF801F6CF84E50F9435
:108FA000452E6F2D70E080E090E04AE00F949E2EF9
:108FB00080E20F94452E0DE013E0D8018D918D01D4
:108FC000882311F40C94593D0F94452EF6CF10923E
:108FD000FB06EDEFF1E284918F010F5F1F4F8823B5
:108FE00021F00F94452EF801F6CF6091FB0670E05A
:108FF00086E598E00E941B998AE00F94452E1AC0DE
:10900000EDEFF1E284918F010F5F1F4F882321F074
:109010000F94452EF801F6CF6091B4157091B515F7
:1090200088E698E00E94349982E20F94452E8AE007
:109030000F94452E0F94A62742C2E0916604F0914A
:109040006704EF2B31F4FC013197F0936704E09350
:109050006604A0E0B0E00C94E32D80E00E946BAACF
:109060000E94C7AA83E50E946EB1882309F449C013
:109070000E9428B121E0482FBE016F5F7F4FCE01D3
:1090800080960E945F776B017C019B01AC010F947D
:10909000ED3E811131C02CEA35EC47E257E368A17F
:1090A00079A18AA19BA10F94413CAB01BC018BEE3D
:1090B00092E00E94BA982CEA35EC47E257E36981C6
:1090C0007A818B819C810F94413CAB01BC0186EE7F
:1090D00092E00E94BA982CEA35EC47E257E3C701C8
:1090E000B6010F94413CAB01BC0181EE92E00E94BD
:1090F000BA988AE00F94452E0E94ADAA0E9421B230
:1091000099CF81E0B7CF0E9407B1AB01BC0140937A
:10911000520F5093530F6093540F7093550F81EA81
:109120009EE00E94E3CD86CF61E0802F0E946B5BC2
:109130006E2D802F0E943C5BF12CB701802F0E9486
:10914000A75B0830110509F075CFF0926D06E0922B
:109150006C0670CFA1964EAD5FADA19714161506A3
:109160000CF061C1CE56DF4F488059806A807B8009
:10917000C259D040480E591E6A1E7B1ECE56DF4F84
:10918000288139814A815B81C259D040281B390B23
:109190004A0B5B0BCA01B901A50194010F94D43BA2
:1091A000A30192010F94053C6B968CAC9DACAEACC8
:1091B000BFAC6B97820E931EA41EB51E34E18316BE
:1091C0009104A104B1041CF14CEE84169104A10495
:1091D000B1043CF450E885169104A104B1043CF1BB
:1091E00005C07BEE872E912CA12CB12C6B968CAEFA
:1091F0009DAEAEAEBFAE6B978EEF90E0A0E0B0E05C
:1092000088199909AA09BB094C015D0116C024E11E
:1092100030E040E050E06B962CAF3DAF4EAF5FAF1B
:109220006B9764E1862E912CA12CB12C06C06B9615
:109230008CAE9DAEAEAEBFAE6B976B964CAD5DADDA
:109240006EAD7FAD6B9786EA97E00E94F498B5010A
:10925000A40181EA97E00E94F498CD57DF4F48813E
:10926000C358D040E4965FADE497E8966FADE897B9
:10927000C957DF4F7881C758D0408AE997E00E94EC
:10928000D798C857DF4F4881C858D040C757DF4FDD
:109290005881C958D040C657DF4F6881CA58D0405E
:1092A000C557DF4F7881CB58D04083E997E00E94C3
:1092B000D798A1964EAD5FADA197433051050CF400
:1092C000B2C0C501B4010F94DD3720E030E040E8C2
:1092D00050E40F943C386B017C01CD57DF4F28815F
:1092E000C358D040E4963FADE497E8964FADE89779
:1092F000C957DF4F5881C758D040C857DF4F6881E2
:10930000C858D040C757DF4F7881C958D040C6579A
:10931000DF4F8881CA58D040C557DF4F9881CB585E
:10932000D0400F94403C2BED3FE049E450E40F94D3
:109330003C3820E030E040E05FE30F943C389B0194
:10934000AC01C701B6010F941D3D6B017C01C30147
:10935000B2010F94DD372FE632E143E85AE30F9470
:109360003C382B013C01B701A6018DE897E00E9433
:10937000D798B301A20187E897E00E94D7982AE91D
:1093800039E949E15FE3C701B6010F943C386B014D
:109390007C019B01AC010F94413CA30192010F940D
:1093A0001D3DA7966CAF7DAF8EAF9FAFA797A30172
:1093B0009201C701B6010F943C3820E030E040E054
:1093C0005EE30F943C38AB966CAF7DAF8EAF9FAF32
:1093D000AB97E7E7F7E084913F015FEF651A750A05
:1093E000882321F00F94452EF301F5CFB701A60194
:1093F00081E797E00E94D798A7964CAD5DAD6EAD22
:109400007FADA7978BE697E00E94D798AB964CADBF
:109410005DAD6EAD7FADAB9785E697E00E94D798C6
:109420008AE00F94452E6B968CAD9DADAEADBFAD71
:109430006B97880D991DAA1DBB1DB595A79597958E
:109440008795EFEF2E163E0619F480931D1002C08B
:1094500080931F10A1962EAD3FADA1972F5F3F4F78
:10946000A1963FAF2EAFA197EC963FADEC97CD57AD
:10947000DF4F3883C358D040AC964FADAC97E496DD
:109480004FAFE497E0965FADE097E8965FAFE8975F
:10949000C158DF4F8881CF57D040C957DF4F8883ED
:1094A000C758D0406F964CAC5DAC6EAC7FAC6F973C
:1094B00091E0C357DF4F9883CD58D04056C9C55669
:1094C000DF4F0FB6F894DEBF0FBECDBFDF91CF9157
:1094D0001F910F91FF90EF90DF90CF90BF90AF90D2
:1094E0009F908F907F906F905F904F903F902F90C4
:1094F00008952F923F924F925F926F927F928F9238
:109500009F92AF92BF92CF92DF92EF92FF920F9312
:109510001F93CF93DF93CDB7DEB76E970FB6F89456
:10952000DEBF0FBECDBFE1E7FAE084918F010F5F90
:109530001F4F882321F00F94452EF801F6CFE9E65E
:10954000FAE084918F010F5F1F4F882321F00F9461
:10955000452EF801F6CF8091060182FF03C00EE58B
:1095600013E002C003E613E0D8018D918D0188233A
:1095700019F00F94452EF8CF8AE00F94452EE1E6BE
:10958000FAE084918F010F5F1F4F882321F00F9421
:10959000452EF801F6CF8091060187FF03C00EE546
:1095A00013E002C003E613E0F80181918F018823E4
:1095B00019F00F94452EF8CF8AE00F94452EE9E577
:1095C000FAE084918F010F5F1F4F882321F00F94E1
:1095D000452EF801F6CF1C9B03C00EE513E002C038
:1095E00003E613E0D8018D918D01882319F00F94C3
:1095F000452EF8CF8AE00F94452EE1E5FAE08491FC
:109600008F010F5F1F4F882321F00F94452EF80123
:10961000F6CF8091000184FD03C00EE513E002C087
:1096200003E613E0F80181918F01882319F00F946C
:10963000452EF8CF8AE00F94452EE0E4FAE08491BD
:109640008F010F5F1F4F882321F00F94452EF801E3
:10965000F6CF83E59BE00E944A966B017C01109255
:10966000B20B1092B30B1092B40B1092B50B42EBED
:109670005BE064E083E59BE00E9479954090B20B4B
:109680005090B30B6090B40B7090B50B8090620B50
:109690009090630BA090640BB090650B83E59BE00A
:1096A0000E9473971091A80BF0E14F225524662475
:1096B0007724A70196012227332744275074298352
:1096C0003A834B835C83A7019601222733274427E3
:1096D00050722D833E834F835887A701960122271E
:1096E00033274427507129873A874B875C87A70126
:1096F000960122273327442758702D873E874F87AE
:10970000588BA70196012227332744275470298BB1
:109710003A8B4B8B5C8BA70196012227332744277A
:1097200052702D8B3E8B4F8B588FA70196012227AD
:10973000307844275527298F3A8F4B8F5C8F14013F
:109740003FE12322332455274B2D3A2D292DD901D2
:10975000AF71BB27BE8FAD8FDC01CB0101E1B695A8
:10976000A795979587950A95D1F7082F0170ECE397
:10977000FAE084914F01BFEF8B1A9B0A882321F0F6
:109780000F94452EF401F5CFE6E3FAE084914F0102
:109790002FEF821A920A882321F00F94452EF401AC
:1097A000F5CFB1016F5F7F4F80E090E04AE00F940A
:1097B0009E2EE4E3FAE084915F013FEFA31AB30A1F
:1097C000882321F00F94452EF501F5CF6D8D7E8D08
:1097D0006F5F7F4F80E090E04AE00F949E2EEDE2B5
:1097E000FAE084915F014FEFA41AB40A882321F0B4
:1097F0000F94452EF501F5CF602F70E080E090E0EA
:109800000F94042F80916E0B90916F0BA091700BB1
:10981000B091710B892B8A2B8B2B09F45FC0EEE181
:10982000FAE084915F015FEFA51AB50A882321F061
:109830000F94452EF501F5CF1F77612F660F6078E5
:10984000612B062E000C770B880B990B0F94042FBD
:109850008091B0049091B104A091B204B091B3048E
:10986000892B8A2B8B2B19F1E5E1FAE084918F018A
:109870000F5F1F4F882321F00F94452EF801F6CF7C
:109880006091B4047091B5048091B6049091B704CE
:109890002091B0043091B1044091B2045091B304CE
:1098A0000F94E33BCA01B9014AE00F949E2EEDE00C
:1098B000FAE084918F010F5F1F4F882321F00F94EE
:1098C000452EF801F6CFB7016F71772780E090E061
:1098D0004AE00F949E2EE1E0FAE00CC0E4E2FAE0E8
:1098E00084918F010F5F1F4F8823A9F30F94452E9A
:1098F000F801F6CF84918F010F5F1F4F882321F06D
:109900000F94452EF801F6CF6091A0047091A10448
:109910008091A2049091A3042091B0043091B104ED
:109920004091B2045091B3040F94E33BCA01B901D2
:109930004AE00F949E2E45284628472861F4EDEF13
:10994000F9E084918F010F5F1F4F882321F00F945E
:10995000452EF801F6CFF7FE0CC0E9EFF9E084914F
:109960008F010F5F1F4F882321F00F94452EF801C0
:10997000F6CF89819A81AB81BC81892B8A2B8B2B75
:1099800061F0E4EFF9E084918F010F5F1F4F8823AE
:1099900021F00F94452EF801F6CF2D813E814F81A5
:1099A0005885232B242B252B61F0EFEEF9E08491D1
:1099B0008F010F5F1F4F882321F00F94452EF80170
:1099C000F6CF89859A85AB85BC85892B8A2B8B2B15
:1099D00061F0E9EEF9E084918F010F5F1F4F88235A
:1099E00021F00F94452EF801F6CF2D853E854F8549
:1099F0005889232B242B252B61F0E3EEF9E0849189
:109A00008F010F5F1F4F882321F00F94452EF8011F
:109A1000F6CF89899A89AB89BC89892B8A2B8B2BB4
:109A200061F0EDEDF9E084918F010F5F1F4F882306
:109A300021F00F94452EF801F6CF2D893E894F89EC
:109A4000588D232B242B252B61F0E9EDF9E084912F
:109A50008F010F5F1F4F882321F00F94452EF801CF
:109A6000F6CF898D9A8DAB8DBC8D892B8A2B8B2B54
:109A700061F0EFECF9E084918F010F5F1F4F8823B5
:109A800021F00F94452EF801F6CF8AE00F94452E71
:109A90008EED9AE00E944A966B017C0110923D0B7C
:109AA00010923E0B10923F0B1092400B4DE35BE087
:109AB00064E08EED9AE00E94799540903D0B5090C5
:109AC0003E0B60903F0B7090400B8090ED0A9090A1
:109AD000EE0AA090EF0AB090F00A8EED9AE00E9494
:109AE00073971091330BA0E14A2255246624772402
:109AF000A7019601222733274427507429833A83EC
:109B00004B835C83A7019601222733274427507299
:109B10002D833E834F835887A70196012227332741
:109B20004427507129873A874B875C87A7019601A4
:109B300022273327442758702D873E874F87588B1D
:109B4000A70196012227332744275470298B3A8B8B
:109B50004B8B5C8BA7019601222733274427527039
:109B60002D8B3E8B4F8B588FA70196012227307883
:109B700044275527298F3A8F4B8F5C8F14013FE183
:109B80002322332455274B2D3A2D292DD901AF718E
:109B9000BB27BE8FAD8FDC01CB01F1E1B695A79558
:109BA00097958795FA95D1F7082F0170EBECF9E0BE
:109BB00084914F01BFEF8B1A9B0A882321F00F94E9
:109BC000452EF401F5CFE5ECF9E084914F012FEF3C
:109BD000821A920A882321F00F94452EF401F5CFC2
:109BE000B1016F5F7F4F80E090E04AE00F949E2EBE
:109BF000E3ECF9E084915F013FEFA31AB30A8823F5
:109C000021F00F94452EF501F5CF6D8D7E8D6F5FA0
:109C10007F4F80E090E04AE00F949E2EECEBF9E05D
:109C200084915F014FEFA41AB40A882321F00F94A6
:109C3000452EF501F5CF602F70E080E090E00F94A5
:109C4000042F8091F90A9091FA0AA091FB0AB09131
:109C5000FC0A892B8A2B8B2B09F45FC0EDEAF9E013
:109C600084915F015FEFA51AB50A882321F00F9454
:109C7000452EF501F5CF1F77612F660F6078612BB8
:109C8000062E000C770B880B990B0F94042F8091F4
:109C9000B0049091B104A091B204B091B304892BA7
:109CA0008A2B8B2B19F1E4EAF9E084918F010F5F85
:109CB0001F4F882321F00F94452EF801F6CF6091B5
:109CC000B8047091B9048091BA049091BB042091BA
:109CD000B0043091B1044091B2045091B3040F9498
:109CE000E33BCA01B9014AE00F949E2EECE9F9E08A
:109CF00084918F010F5F1F4F882321F00F94452E11
:109D0000F801F6CFB7016F71772780E090E04AE065
:109D10000F949E2EE0E9F9E00CC0E3EBF9E08491AA
:109D20008F010F5F1F4F8823A9F30F94452EF80171
:109D3000F6CF84918F010F5F1F4F882321F00F947E
:109D4000452EF801F6CF6091A4047091A50480918E
:109D5000A6049091A7042091B0043091B1044091E1
:109D6000B2045091B3040F94E33BCA01B9014AE035
:109D70000F949E2E45284628472861F4ECE8F9E028
:109D800084918F010F5F1F4F882321F00F94452E80
:109D9000F801F6CFF7FE0CC0E8E8F9E084918F01F6
:109DA0000F5F1F4F882321F00F94452EF801F6CF47
:109DB00089819A81AB81BC81892B8A2B8B2B61F0A5
:109DC000E3E8F9E084918F010F5F1F4F882321F0B2
:109DD0000F94452EF801F6CF2D813E814F81588595
:109DE000232B242B252B61F0EEE7F9E084918F01E2
:109DF0000F5F1F4F882321F00F94452EF801F6CFF7
:109E000089859A85AB85BC85892B8A2B8B2B61F044
:109E1000E8E7F9E084918F010F5F1F4F882321F05D
:109E20000F94452EF801F6CF2D853E854F85588934
:109E3000232B242B252B61F0E2E7F9E084918F019D
:109E40000F5F1F4F882321F00F94452EF801F6CFA6
:109E500089899A89AB89BC89892B8A2B8B2B61F0E4
:109E6000ECE6F9E084918F010F5F1F4F882321F00A
:109E70000F94452EF801F6CF2D893E894F89588DD4
:109E8000232B242B252B61F0E8E6F9E084918F0148
:109E90000F5F1F4F882321F00F94452EF801F6CF56
:109EA000898D9A8DAB8DBC8D892B8A2B8B2B61F084
:109EB000EEE5F9E084918F010F5F1F4F882321F0B9
:109EC0000F94452EF801F6CF8AE00F94452E89E6CF
:109ED0009AE00E944A966B017C011092C80A109287
:109EE000C90A1092CA0A1092CB0A48EC5AE064E000
:109EF00089E69AE00E9479954090C80A5090C90A74
:109F00006090CA0A7090CB0A8090780A9090790A83
:109F1000A0907A0AB0907B0A89E69AE00E94739733
:109F20001091BE0AA0E14A22552466247724A70195
:109F30009601222733274427507429833A834B8381
:109F40005C83A701960122273327442750722D8373
:109F50003E834F835887A701960122273327442742
:109F6000507129873A874B875C87A7019601222782
:109F70003327442758702D873E874F87588BA7017A
:109F800096012227332744275470298B3A8B4B8B19
:109F90005C8BA701960122273327442752702D8B13
:109FA0003E8B4F8B588FA70196012227307844278C
:109FB0005527298F3A8F4B8F5C8F14013FE1232265
:109FC000332455274B2D3A2D292DD901AF71BB27AD
:109FD000BE8FAD8FDC01CB0151E1B695A79597956A
:109FE00087955A95D1F7082F0170EAE5F9E0849139
:109FF0004F01BFEF8B1A9B0A882321F00F94452E47
:10A00000F401F5CFE4E5F9E084914F012FEF821AD6
:10A01000920A882321F00F94452EF401F5CFB10167
:10A020006F5F7F4F80E090E04AE00F949E2EE2E564
:10A03000F9E084915F013FEFA31AB30A882321F06E
:10A040000F94452EF501F5CF6D8D7E8D6F5F7F4F9F
:10A0500080E090E04AE00F949E2EEBE4F9E08491DA
:10A060005F014FEFA41AB40A882321F00F94452E04
:10A07000F501F5CF602F70E080E090E00F94042FA1
:10A080008091840A9091850AA091860AB091870AEE
:10A09000892B8A2B8B2B09F45FC0ECE3F9E08491C8
:10A0A0005F015FEFA51AB50A882321F00F94452EB2
:10A0B000F501F5CF1F77612F660F6078612B062EB3
:10A0C000000C770B880B990B0F94042F8091B00430
:10A0D0009091B104A091B204B091B304892B8A2B62
:10A0E0008B2B19F1E3E3F9E084918F010F5F1F4F90
:10A0F000882321F00F94452EF801F6CF6091BC041F
:10A100007091BD048091BE049091BF042091B00471
:10A110003091B1044091B2045091B3040F94E33BE9
:10A12000CA01B9014AE00F949E2EEBE2F9E0849156
:10A130008F010F5F1F4F882321F00F94452EF801E8
:10A14000F6CFB7016F71772780E090E04AE00F9477
:10A150009E2EEFE1F9E00CC0E2E4F9E084918F017A
:10A160000F5F1F4F8823A9F30F94452EF801F6CFF8
:10A1700084918F010F5F1F4F882321F00F94452E8C
:10A18000F801F6CF6091A8047091A9048091AA0407
:10A190009091AB042091B0043091B1044091B2048D
:10A1A0005091B3040F94E33BCA01B9014AE00F9404
:10A1B0009E2E45284628472861F4EBE1F9E084917A
:10A1C0008F010F5F1F4F882321F00F94452EF80158
:10A1D000F6CFF7FE0CC0E7E1F9E084918F010F5F45
:10A1E0001F4F882321F00F94452EF801F6CF898167
:10A1F0009A81AB81BC81892B8A2B8B2B61F0E2E1A8
:10A20000F9E084918F010F5F1F4F882321F00F9495
:10A21000452EF801F6CF2D813E814F815885232BA5
:10A22000242B252B61F0EDE0F9E084918F010F5F85
:10A230001F4F882321F00F94452EF801F6CF898512
:10A240009A85AB85BC85892B8A2B8B2B61F0E7E047
:10A25000F9E084918F010F5F1F4F882321F00F9445
:10A26000452EF801F6CF2D853E854F855889232B45
:10A27000242B252B61F0E1E0F9E084918F010F5F41
:10A280001F4F882321F00F94452EF801F6CF8989BE
:10A290009A89AB89BC89892B8A2B8B2B61F0EBEFD8
:10A2A000F8E084918F010F5F1F4F882321F00F94F6
:10A2B000452EF801F6CF2D893E894F89588D232BE5
:10A2C000242B252B61F0E7EFF8E084918F010F5FDD
:10A2D0001F4F882321F00F94452EF801F6CF898D6A
:10A2E0009A8DAB8DBC8D892B8A2B8B2B61F0EDEE7B
:10A2F000F8E084918F010F5F1F4F882321F00F94A6
:10A30000452EF801F6CF8AE00F94452E84EF99E0B0
:10A310000E944A966B017C011092530A1092540AD3
:10A320001092550A1092560A43E55AE064E084EF11
:10A3300099E00E9479954090530A5090540A609099
:10A34000550A7090560A8090030A9090040AA090D3
:10A35000050AB090060A84EF99E00E947397109165
:10A36000490AA0E14A22552466247724A7019601D0
:10A37000222733274427507429833A834B835C83F5
:10A38000A701960122273327442750722D833E834D
:10A390004F835887A70196012227332744275071FE
:10A3A00029873A874B875C87A701960122273327A5
:10A3B000442758702D873E874F87588BA7019601F9
:10A3C0002227332744275470298B3A8B4B8B5C8B85
:10A3D000A701960122273327442752702D8B3E8BED
:10A3E0004F8B588FA7019601222730784427552795
:10A3F000298F3A8F4B8F5C8F14013FE12322332446
:10A4000055274B2D3A2D292DD901AF71BB27BE8F72
:10A41000AD8FDC01CB0131E1B695A7959795879576
:10A420003A95D1F7082F0170E8EEF8E084914F01DA
:10A43000BFEF8B1A9B0A882321F00F94452EF4015D
:10A44000F5CFE2EEF8E084914F012FEF821A920AE5
:10A45000882321F00F94452EF401F5CFB1016F5FF1
:10A460007F4F80E090E04AE00F949E2EE0EEF8E00F
:10A4700084915F013FEFA31AB30A882321F00F9460
:10A48000452EF501F5CF6D8D7E8D6F5F7F4F80E09E
:10A4900090E04AE00F949E2EE9EDF8E084915F0190
:10A4A0004FEFA41AB40A882321F00F94452EF5012A
:10A4B000F5CF602F70E080E090E00F94042F809142
:10A4C0000F0A9091100AA091110AB091120A892BDB
:10A4D0008A2B8B2B09F45FC0EAECF8E084915F01D2
:10A4E0005FEFA51AB50A882321F00F94452EF501D8
:10A4F000F5CF1F77612F660F6078612B062E000C59
:10A50000770B880B990B0F94042F8091B0049091D6
:10A51000B104A091B204B091B304892B8A2B8B2B88
:10A5200019F1E1ECF8E084918F010F5F1F4F882350
:10A5300021F00F94452EF801F6CF6091C004709180
:10A54000C1048091C2049091C3042091B004309161
:10A55000B1044091B2045091B3040F94E33BCA019B
:10A56000B9014AE00F949E2EE9EBF8E084918F0147
:10A570000F5F1F4F882321F00F94452EF801F6CF6F
:10A58000B7016F71772780E090E04AE00F949E2E2C
:10A59000EDEAF8E00CC0E0EDF8E084918F010F5F88
:10A5A0001F4F8823A9F30F94452EF801F6CF84910D
:10A5B0008F010F5F1F4F882321F00F94452EF80164
:10A5C000F6CF6091AC047091AD048091AE0490918F
:10A5D000AF042091B0043091B1044091B204509185
:10A5E000B3040F94E33BCA01B9014AE00F949E2ED5
:10A5F00045284628472861F4E9EAF8E084918F016C
:10A600000F5F1F4F882321F00F94452EF801F6CFDE
:10A61000F7FE0CC0E5EAF8E084918F010F5F1F4F51
:10A62000882321F00F94452EF801F6CF89819A8175
:10A63000AB81BC81892B8A2B8B2B61F0E0EAF8E09F
:10A6400084918F010F5F1F4F882321F00F94452EB7
:10A65000F801F6CF2D813E814F815885232B242B85
:10A66000252B61F0EBE9F8E084918F010F5F1F4F1C
:10A67000882321F00F94452EF801F6CF89859A851D
:10A68000AB85BC85892B8A2B8B2B61F0E5E9F8E043
:10A6900084918F010F5F1F4F882321F00F94452E67
:10A6A000F801F6CF2D853E854F855889232B242B25
:10A6B000252B61F0EFE8F8E084918F010F5F1F4FC9
:10A6C000882321F00F94452EF801F6CF89899A89C5
:10A6D000AB89BC89892B8A2B8B2B61F0E9E8F8E0E8
:10A6E00084918F010F5F1F4F882321F00F94452E17
:10A6F000F801F6CF2D893E894F89588D232B242BC5
:10A70000252B61F0E5E8F8E084918F010F5F1F4F82
:10A71000882321F00F94452EF801F6CF898D9A8D6C
:10A72000AB8DBC8D892B8A2B8B2B61F0EBE7F8E08E
:10A7300084918F010F5F1F4F882321F00F94452EC6
:10A74000F801F6CF8AE06E960FB6F894DEBF0FBE22
:10A75000CDBFDF91CF911F910F91FF90EF90DF90D0
:10A76000CF90BF90AF909F908F907F906F905F90B1
:10A770004F903F902F900D94452ECF92DF92EF9205
:10A78000FF920F931F93CF93DF936C017A018B019C
:10A79000C0E0D0E0CE15DF0589F0D8016D918D01C4
:10A7A000D601ED91FC910190F081E02DC601199543
:10A7B000892B11F47E0102C02196ECCFC701DF91F5
:10A7C000CF911F910F91FF90EF90DF90CF90089560
:10A7D000089580E090E0089580E008950B96FC01D4
:10A7E000849108950A96FC0184910895FC01849156
:10A7F0000895FCDF882321F0823011F083E0089572
:10A8000086E00895FC01E60FF11D849190E0982FF9
:10A8100088273196E4918E0F911D089568E0F2CF5C
:10A8200066E0F0CF0895FC01A681B7818281481BC4
:10A830008581483018F0A80FB11D4770382F369524
:10A8400036953695562F577080E890E002C0959562
:10A8500087955A95E2F7439F402D1124669566959A
:10A860006695E62FF0E0E40FF11DEA0FFB1F308143
:10A87000222311F0832B02C08095832380830895C7
:10A88000FB014181DC0112962C911297421760F076
:10A8900013962C911397241738F0608115962C91FC
:10A8A000621710F42481BFCF0895FC01808192814A
:10A8B000980F92832181921760F494819F5F948313
:10A8C0009381890F821710F08FEF820F838381E0CD
:10A8D000089580E00895FC01128280818150838375
:10A8E0001482089581E00895089590E0FC01319765
:10A8F000E231F10508F04EC08827EE58FF4F8F4F28
:10A900000D94303F809180008F7703C0809180004C
:10A910008F7D80938000089580918000877FF9CF9C
:10A9200084B58F7702C084B58F7D84BD08958091F2
:10A93000B0008F7703C08091B0008F7D8093B0000E
:10A940000895809190008F7707C0809190008F7D4F
:10A9500003C080919000877F80939000089580913C
:10A96000A0008F7707C08091A0008F7D03C08091E9
:10A97000A000877F8093A0000895809120018F77A9
:10A9800007C0809120018F7D03C080912001877FC7
:10A990008093200108958F929F92AF92BF92DF9291
:10A9A000EF92FF920F931F93CF93DF93162F072FF2
:10A9B000D42EFC0160817181828193812CE3822EEF
:10A9C000912CA12CB12CA50194010F94E33BCA0159
:10A9D000B901A50194010F94E33BCA01F62EE72EBD
:10A9E000C22FD32FDD2061F1B90128E130E040E032
:10A9F00050E00F94E33B49015A01EF92FF92CE01E0
:10AA000068E170E00F94093F9F938F939F928F921C
:10AA100083EF9AE09F938F930F931F930F94703758
:10AA20008DB79EB70A960FB6F8949EBF0FBE8DBF26
:10AA30009AE089169104A104B104B0F587E035C00D
:10AA4000C436D105D8F47F936F93CE0168E170E0EE
:10AA50000F94093F9F938F9389EE9AE09F938F9372
:10AA60000F931F930F947037EDB7FEB738960FB65C
:10AA7000F894FEBF0FBEEDBF85E017C07F936F93C4
:10AA80003F932F9381EE9AE09F938F930F931F93A1
:10AA90000F9470378DB79EB708960FB6F8949EBF87
:10AAA0000FBE8DBF86E001C088E0DF91CF911F917E
:10AAB0000F91FF90EF90DF90BF90AF909F908F909D
:10AAC00008954F925F926F927F92AF92BF92CF9212
:10AAD000DF92EF92FF92CF93DF93EB01FC01608155
:10AAE0007181828193812CE3C22ED12CE12CF12C37
:10AAF000A70196010F94E33BB62EA72ECA01B90118
:10AB0000A70196010F94E33B6B017C01CA01B901D7
:10AB100028E130E040E050E00F94E33B2B013C01A2
:10AB2000C9016DE671E00F94093F61157105D9F017
:10AB3000AF92BF92DF92CF925F924F929F938F938B
:10AB40007F936F938DEC9AE09F938F93DF93CF93D6
:10AB50000F9470378DB79EB70E960FB6F8949EBFC0
:10AB60000FBE8DBF61C00097C9F0AF92BF92DF9258
:10AB7000CF925F924F929F938F938DEB9AE09F932A
:10AB80008F93DF93CF930F947037EDB7FEB73C965A
:10AB90000FB6F894FEBF0FBEEDBF46C0411451047E
:10ABA00061047104B9F0AF92BF92DF92CF925F92CD
:10ABB0004F9281EB9AE09F938F93DF93CF930F9403
:10ABC00070378DB79EB70A960FB6F8949EBF0FBE2A
:10ABD0008DBF2AC0C114D104E104F104A9F0AF92E1
:10ABE000BF92DF92CF9289EA9AE09F938F93DF938F
:10ABF000CF930F947037EDB7FEB738960FB6F89431
:10AC0000FEBF0FBEEDBF10C0AF92BF9285EA9AE0C3
:10AC10009F938F93DF93CF930F9470370F900F9084
:10AC20000F900F900F900F90DF91CF91FF90EF90CA
:10AC3000DF90CF90BF90AF907F906F905F904F90DC
:10AC40000895FC01238121110C9416CF08952091C1
:10AC5000500C9091510C81E0291301C080E00895BF
:10AC60008091500C9091510C891B8F700895EF9238
:10AC7000FF920F931F93CF93DF93EC0119821882F9
:10AC80001B821A821D821C8261157105A9F17B014C
:10AC9000FB0101900020E9F731978F01061B170B8C
:10ACA000B8016F5F7F4F80E090E00F943E3F0097C8
:10ACB00059F0998388831B830A832C813D81232B40
:10ACC00081F4FC0110820DC088819981009711F0F8
:10ACD0000F94CC32198218821D821C821B821A8228
:10ACE0000BC01D830C83B701DF91CF911F910F9192
:10ACF000FF90EF900D946D40DF91CF911F910F91D8
:10AD0000FF90EF900895CF92DF92FF920F931F93E1
:10AD1000CF93DF931F921F92CDB7DEB76901DB019E
:10AD200012960D911C911397423309F470C0B8F438
:10AD3000453109F477C0473109F487C0443109F03F
:10AD40009DC0D80115962C9115971696ED91FC9102
:10AD50001797CF01820F911D820F911D5CC0463461
:10AD600009F483C0473409F484C04B3309F086C02A
:10AD7000F90181819381913029F0933031F4482F8A
:10AD8000885004C048E0480F01C0482F21E0D80196
:10AD900013963C91381708F420E031E0F801528115
:10ADA000451708F430E051E0481708F050E0822FD2
:10ADB000852B382319F4252309F460C0D601129697
:10ADC000FC90913051F030F0923049F0933051F4D2
:10ADD0002FEF09C020E031E007C021E004C020E0EF
:10ADE0003FEF02C020E030E0F7FE07C0B601C80127
:10ADF0002A83398345DD39812A81F6018081830FD9
:10AE000080838181820F8183FF0C71F737C0B90184
:10AE1000C80136DD33C01192E817F907E1F7C80120
:10AE20005ADD2CC0C80141DD882349F1F801258194
:10AE30000680F781E02DCF01820F911D820F911DB9
:10AE40001192E817F907E1F719C0D9011C92F8012E
:10AE5000828111968C9311978581815012968C93E3
:10AE60001297838113968C9309C0D80115968C9103
:10AE700003C0D80111968C91F601808381E00F9078
:10AE80000F90DF91CF911F910F91FF90DF90CF90A6
:10AE9000089588E290E00197F1F708952EE93FE0E8
:10AEA000009729F0F9013197F1F70197F9CF08954B
:10AEB0000F93FC010150040F84A996A9941718F070
:10AEC000081728F402C0081750F0041740F4215066
:10AED000260F83A995A9961720F4281720F480E05F
:10AEE00007C0281720F481E0261710F0F8CF81E082
:10AEF0000F910895DB01ED91FC9119942F923F92EF
:10AF00005F926F927F928F929F92AF92BF92CF92F9
:10AF1000DF92EF92FF920F931F93CF93DF931F92D5
:10AF2000CDB7DEB71C01C62E142FD22EDC0114962D
:10AF3000ED90FC901597C70159DC082FF101848131
:10AF4000958157DC982E013019F48FE0A82E02C0AD
:10AF5000AA24AA94D10114968D919C91159742DC54
:10AF6000082FF1018481958139DCB82ED101149626
:10AF70008D919C91159752DCB0E6BD1530F4009789
:10AF800021F0E80EF91E01E610C0F10184819581DF
:10AF900047DCF0E4FD1530F4009721F0E80EF91ECF
:10AFA00001E403C021E1E20EF11CBD1480F4D101E3
:10AFB00050961C92509753961C92539754961C92FD
:10AFC000549751961C92519752961C92C3C0B0163A
:10AFD00070F3892D90E0F70124912F3F21F4FFEFCA
:10AFE000EF1AFF0A59C00D114EC0D10114968D9170
:10AFF0009C911597FBDB97012F5F3F4FF70188234B
:10B0000011F08230E1F48491D10153968C935397DF
:10B01000F901249154962C935497F7013396E491B7
:10B020005096EC935097F7013496E4915196EC9337
:10B030005197F7013596E4915296EC9320C0849194
:10B04000982F9F709250D10152969C93529782955F
:10B050008F7051968C935197F9012491822F8F70A4
:10B0600054968C93549722952F7053962C93539704
:10B07000F7013296E491E295EF705096EC93E1146B
:10B08000F10479F467C0F7013296E491EA219C015A
:10B090002E0F311DE20EF31E0B1509F488CF0F5F42
:10B0A0009ACFF10184819581A4DBB82ED10153960A
:10B0B0009C9053975496DC90549751968C9151974D
:10B0C000C80E52969C919D0D512E591A0D2D292D69
:10B0D000452D6C2DC101ECDE8823C9F1C7018B0D14
:10B0E000911D5C0187E0890DF82EF694F694F69494
:10B0F000D50C41019CE1890E911C6F2C712C5D14C3
:10B1000031F15C2D8501802F8A198F15E0F4F8014B
:10B110008491D10112966D917C9113975C965C930A
:10B120005C975D965C925D975F961C925F975E96CA
:10B130008C9394014BE3C1015983DCDE0F5F1F4FF9
:10B140005981585FE0CFA60CB71C5394D8CFF101BA
:10B15000808901C080E00F90DF91CF911F910F9106
:10B16000FF90EF90DF90CF90BF90AF909F908F9027
:10B170007F906F905F903F902F9008958F929F9255
:10B18000BF92CF92DF92EF92FF920F931F93CF93D4
:10B19000DF931F92CDB7DEB74C01062FF42E122F8E
:10B1A000522FE62EE20EBB24BA946C018CE1C80E3D
:10B1B000D11C8E2D851B583078F0F401628173818B
:10B1C000848FF58E178EB68E96014BE3C40159839A
:10B1D00091DE59815850EDCF812F887F080F212FA4
:10B1E000277019F187E02827F40162817381048FA9
:10B1F000F58E178E2F5F27708FEF90E001C0880FBC
:10B200002A95EAF7868F9401245E3F4F4BE3C401F1
:10B210000F90DF91CF911F910F91FF90EF90DF90F2
:10B22000CF90BF909F908F9065CE0F90DF91CF9180
:10B230001F910F91FF90EF90DF90CF90BF909F9064
:10B240008F900895EF92FF920F931F93CF93DF9308
:10B250007C01D62F122FC42F040F212F4C2F6D2FBE
:10B26000C7018CDFCF5F0C13F8CFDF91CF911F9117
:10B270000F91FF90EF900895DF92EF92FF920F935E
:10B280001F93CF93DF93EC01162FF42EE22E10DEE6
:10B29000882329F02E2D4F2D612FCE01D3DFDF9192
:10B2A000CF911F910F91FF90EF90DF900895EF9253
:10B2B000FF920F931F93CF93DF931F92CDB7DEB70B
:10B2C0008C01DC011296ED90FC901397D196ED91D4
:10B2D000FC91D29782E0199520E030E04AE0B70176
:10B2E000C80108DEF82ED801D196ED91FC91D297D5
:10B2F00083E01995D801D196ED91FC91D29780E029
:10B300001995FF2081F1F801628173819E012F5F01
:10B310003F4F46E4C801EEDD8981D8018C93129637
:10B320006D917C9113979E012F5F3F4F47E4C801B9
:10B33000E1DD8981F80181836281738120E030E061
:10B3400048E4C801D7DDD8011B968C931B97980160
:10B350002D5C3F4F12966D917C91139747E1C80188
:10B36000C9DD81E001C080E00F90DF91CF911F9196
:10B370000F91FF90EF9008951F920F920FB60F92CA
:10B3800011240BB60F922F933F934F935F936F93BC
:10B390007F938F939F93AF93BF93EF93FF93E0912E
:10B3A0001402F09115021995FF91EF91BF91AF91A1
:10B3B0009F918F917F916F915F914F913F912F91CD
:10B3C0000F900BBE0F900FBE0F901F9018951F92FD
:10B3D0000F920FB60F9211240BB60F922F933F933B
:10B3E0004F935F936F937F938F939F93AF93BF938D
:10B3F000EF93FF93E0911202F09113021995FF91E0
:10B40000EF91BF91AF919F918F917F916F915F91DC
:10B410004F913F912F910F900BBE0F900FBE0F9049
:10B420001F9018951F920F920FB60F9211240BB612
:10B430000F922F933F934F935F936F937F938F93CD
:10B440009F93AF93BF93EF93FF93E0910802F09126
:10B4500009021995FF91EF91BF91AF919F918F9143
:10B460007F916F915F914F913F912F910F900BBE04
:10B470000F900FBE0F901F9018951F920F920FB64E
:10B480000F9211240BB60F922F933F934F935F931C
:10B490006F937F938F939F93AF93BF93EF93FF939C
:10B4A000E0910602F09107021995FF91EF91BF918B
:10B4B000AF919F918F917F916F915F914F913F914C
:10B4C0002F910F900BBE0F900FBE0F901F901895ED
:10B4D0001F920F920FB60F9211240BB60F922F935B
:10B4E0003F934F935F936F937F938F939F93AF930C
:10B4F000BF93EF93FF93E0911002F0911102199521
:10B50000FF91EF91BF91AF919F918F917F916F913B
:10B510005F914F913F912F910F900BBE0F900FBEF7
:10B520000F901F9018951F920F920FB60F92112433
:10B530000BB60F922F933F934F935F936F937F932D
:10B540008F939F93AF93BF93EF93FF93E0910E027E
:10B55000F0910F021995FF91EF91BF91AF919F91DB
:10B560008F917F916F915F914F913F912F910F90AC
:10B570000BBE0F900FBE0F901F9018951F920F9249
:10B580000FB60F9211240BB60F922F933F934F9348
:10B590005F936F937F938F939F93AF93BF93EF933B
:10B5A000FF93E0910C02F0910D021995FF91EF913C
:10B5B000BF91AF919F918F917F916F915F914F91CB
:10B5C0003F912F910F900BBE0F900FBE0F901F90C9
:10B5D00018951F920F920FB60F9211240BB60F926F
:10B5E0002F933F934F935F936F937F938F939F938B
:10B5F000AF93BF93EF93FF93E0910A02F0910B0298
:10B600001995FF91EF91BF91AF919F918F917F918C
:10B610006F915F914F913F912F910F900BBE0F90C3
:10B620000FBE0F901F901895CF93DF93282F30E017
:10B63000F901E65BF34E8491F901ED5FFA4DD49187
:10B64000F901ED59FA4DC491CC2389F081114DD9FE
:10B65000EC2FF0E0EE0FFF1FE557F54FA591B491E9
:10B66000EC91ED2381E090E021F480E002C080E0E5
:10B6700090E0DF91CF9108951F93CF93DF93282F10
:10B6800030E0F901E65BF34E8491F901ED5FFA4D8C
:10B69000D491F901ED59FA4DC491CC23C1F0162F84
:10B6A000811123D9EC2FF0E0EE0FFF1FE75BFA4D7D
:10B6B000A591B4918FB7F894111105C09C91ED2F0D
:10B6C000E095E92302C0EC91ED2BEC938FBFDF9165
:10B6D000CF911F910895CF93DF9390E0FC01ED5F30
:10B6E000FA4D2491FC01ED59FA4D8491882361F1C2
:10B6F00090E0880F991FFC01E158FF4DC591D4914E
:10B70000FC01E75BFA4DA591B491611109C09FB7A7
:10B71000F8948881209582238883EC912E230BC096
:10B72000623061F49FB7F8943881822F809583232B
:10B730008883EC912E2B2C939FBF06C08FB7F89473
:10B74000E8812E2B28838FBFDF91CF9108951F931F
:10B75000CF93DF93182FEB0161E0BDDF209711F449
:10B7600060E004C0CF3FD10531F461E0812FDF916B
:10B77000CF911F9181CFE12FF0E0E65BF34EE49192
:10B780004E2F50E0FA013197E231F10508F09DC0EB
:10B790008827EC57FF4F8F4F0D94303F84B580685A
:10B7A00084BDC7BD97C084B5806284BDC8BD92C04A
:10B7B00080918000806880938000D0938900C0933E
:10B7C000880088C080918000806280938000D09340
:10B7D0008B00C0938A007EC0809180008860809337
:10B7E0008000D0938D00C0938C0074C08091B00015
:10B7F00080688093B000C093B3006CC08091B000AB
:10B8000080628093B000C093B40064C080919000C7
:10B81000806880939000D0939900C09398005AC09C
:10B8200080919000806280939000D0939B00C093A1
:10B830009A0050C080919000886080939000D093CF
:10B840009D00C0939C0046C08091A00080688093BA
:10B85000A0008091A0008F7B8093A000D093A900CE
:10B86000C093A80037C08091A00080628093A000A0
:10B87000D093AB00C093AA002DC08091A000886037
:10B880008093A000D093AD00C093AC0023C0809102
:10B890002001806880932001D0932901C093280162
:10B8A00019C080912001806280932001D0932B01E8
:10B8B000C0932A010FC080912001886080932001ED
:10B8C000D0932D01C0932C0105C0C038D1050CF0D8
:10B8D0004CCF46CFDF91CF911F9108953FB7F89499
:10B8E0008091820490918304A0918404B091850496
:10B8F00026B5A89B05C02F3F19F00196A11DB11DCB
:10B900003FBFBA2FA92F982F8827820F911DA11D05
:10B91000B11DBC01CD0142E0660F771F881F991F42
:10B920004A95D1F708958F929F92AF92BF92CF928E
:10B93000DF92EF92FF926B017C01D0DF4B015C0143
:10B94000C114D104E104F104E9F0C8DFDC01CB014A
:10B9500088199909AA09BB09883E9340A105B10538
:10B9600078F321E0C21AD108E108F10888EE880EC8
:10B9700083E0981EA11CB11CC114D104E104F104A0
:10B9800021F7DECFFF90EF90DF90CF90BF90AF9088
:10B990009F908F9008952FB7F89460917E047091D6
:10B9A0007F0480918004909181042FBF0895F3DF7C
:10B9B0006093B6157093B7158093B8159093B91529
:10B9C00008951F920F920FB60F9211242F933F9359
:10B9D0008F939F93AF93BF9380917E0490917F0448
:10B9E000A0918004B091810430917D0423E0230F65
:10B9F0002D3720F40196A11DB11D05C026E8230FA7
:10BA00000296A11DB11D20937D0480937E04909326
:10BA10007F04A0938004B09381048091820490916C
:10BA20008304A0918404B09185040196A11DB11DE9
:10BA30008093820490938304A0938404B09385043C
:10BA4000BF91AF919F918F913F912F910F900FBE1A
:10BA50000F901F901895CF93DF93CDB7DEB7609707
:10BA60000FB6F894DEBF0FBECDBF789484B5826068
:10BA700084BD84B5816084BD85B5826085BD85B592
:10BA8000816085BD80916E00816080936E00109210
:10BA9000810080918100826080938100809181008B
:10BAA000816080938100809180008160809380001C
:10BAB0008091B10084608093B1008091B00081607A
:10BAC0008093B0008091910082608093910080917A
:10BAD00091008160809391008091900081608093BB
:10BAE00090008091A10082608093A1008091A100CC
:10BAF00081608093A1008091A00081608093A0006C
:10BB000080912101826080932101809121018160D7
:10BB10008093210180912001816080932001809198
:10BB20007A00846080937A0080917A0082608093AA
:10BB30007A0080917A00816080937A0080917A0007
:10BB4000806880937A001092C1003D98459A82E007
:10BB50008093C0001092C50087E08093C40080915C
:10BB6000C10080618093C1008091C1008860809392
:10BB7000C1008091C10080688093C1008091C100A4
:10BB80008F7D8093C10010928604ECE7FCE08491E5
:10BB90008F010F5F1F4F882321F00F94452EF8016E
:10BBA000F6CFEDEFF1E284918F010F5F1F4F8823F5
:10BBB00021F00F94452EF801F6CF14B710FF0DC0F9
:10BBC000E3E7FCE084917F019FEFE91AF90A8823FB
:10BBD00021F00F94452EF701F5CF11FF0DC0E2E6DD
:10BBE000FCE084917F019FEFE91AF90A882321F094
:10BBF0000F94452EF701F5CF12FF0DC0E0E5FCE0F4
:10BC000084917F019FEFE91AF90A882321F00F94AC
:10BC1000452EF701F5CF13FF0DC0EFE3FCE0849153
:10BC20007F019FEFE91AF90A882321F00F94452E2E
:10BC3000F701F5CF15FF0CC0EEE2FCE084918F0117
:10BC40000F5F1F4F882321F00F94452EF801F6CF88
:10BC500014BEE7E2FCE084918F010F5F1F4F882341
:10BC600021F00F94452EF801F6CF80E20F94452E77
:10BC7000E0E2FCE084918F010F5F1F4F882321F0E9
:10BC80000F94452EF801F6CF8AE00F94452EEDEF84
:10BC9000F1E284918F010F5F1F4F882321F00F94F1
:10BCA000452EF801F6CFE0E1FCE084918F010F5FB3
:10BCB0001F4F882321F00F94452EF801F6CFECEFAB
:10BCC000FBE084918F010F5F1F4F882321F00F94B9
:10BCD000452EF801F6CFE3ECFBE084918F010F5F76
:10BCE0001F4F882321F00F94452EF801F6CFEDEF7A
:10BCF000F1E284918F010F5F1F4F882321F00F9491
:10BD0000452EF801F6CFECEAFBE084918F010F5F3E
:10BD10001F4F882321F00F94452EF801F6CFEDEF49
:10BD2000F1E284918F010F5F1F4F882321F00F9460
:10BD3000452EF801F6CF8091A6179091A7178E0196
:10BD40000F5F1F4FB801009719F0681B790B02C0F5
:10BD50006C5A77418DE99BE00E941B9960ED74E07D
:10BD600086E89BE00E941B998AE00F94452E81E0B3
:10BD700080939C0480939D0480939E0480939F04F1
:10BD80000E948ADC8CE0E0E9F4E0A2E3B7E00190F5
:10BD90000D928A95E1F70E9417B06D9A9D9A809155
:10BDA000010180628093010188E00E94E675809124
:10BDB000010188608093010186E00E94E67587EDAD
:10BDC00080937A0010927E0010927D0080917E0018
:10BDD000816080937E0080917E00846080937E00ED
:10BDE00080E888BD80916E00846080936E006AEF69
:10BDF00070E080E090E097DD85E090E090938C0427
:10BE000080938B0460E080911802909119020E9447
:10BE100071F920E030E040EA50E40F94D73787FF13
:10BE20000AC08091180290911902409790931902CC
:10BE300080931802E7CF81E391E090931B028093F7
:10BE40001A0260E08091890490918A040E9471F93D
:10BE500020E030E848E953E40F94673E181654F4A4
:10BE60008091890490918A04409690938A048093EB
:10BE70008904E7CF80911602909117020E94C4FABC
:10BE800020E030E040EA50E40F94D73787FF0AC043
:10BE90008091160290911702409790931702809319
:10BEA0001602E8CF80918704909188040E94C4FA1A
:10BEB00020E030E046E153E40F94673E181654F456
:10BEC0008091870490918804409690938804809391
:10BED0008704E8CF98E288E10FB6F894A89580939C
:10BEE00060000FBE9093600080910A01886080938B
:10BEF0000A0180910A01806180930A0180910A0100
:10BF0000806280930A010E9465FF80912101887FF1
:10BF100081608093210180E1E6EAF2E0D80101909E
:10BF20000D928A95E1F7980148E450E060E070E0F6
:10BF300083E59BE00E94147664E083E59BE00E9429
:10BF40005D969E012B5F3F4F48E450E060E070E05B
:10BF50008EED9AE00E94147664E08EED9AE00E94E5
:10BF60005D969E01275F3F4F44E050E060E070E047
:10BF700089E69AE00E9414769E01235F3F4F4EE1CE
:10BF800050E060E070E084EF99E00E94147661E098
:10BF900083E59BE00E94CB9661E08EED9AE00E94E3
:10BFA000CB9661E083E59BE00E945E9761E08EEDB9
:10BFB0009AE00E945E9764E083E59BE00E942E97E2
:10BFC00064E08EED9AE00E942E9760E083E59BE0AE
:10BFD0000E94FB9660E08EED9AE00E94FB9661E085
:10BFE00089E69AE00E945E9760E089E69AE00E9406
:10BFF0002E9760E089E69AE00E94FB9661E089E670
:10C000009AE00E94CB9664E089E69AE00E945D96F1
:10C0100061E089E69AE00E94249640E050E0BA018F
:10C0200089E69AE00E949F9760E089E69AE00E9484
:10C03000B69660E089E69AE00E94899661E089E61A
:10C040009AE00E945E9760E089E69AE00E942E974F
:10C0500060E089E69AE00E94FB9661E089E69AE05A
:10C060000E94CB9660E084EF99E00E9424964FEF07
:10C070005FEF6FE070E084EF99E00E949F9761E0CE
:10C0800084EF99E00E94B69663E084EF99E00E9405
:10C09000899680910A01816080930A0180910A014A
:10C0A000826080930A0180910A01846080930A0172
:10C0B00080910A01806480930A010F9A179A0E9A60
:10C0C000169A0D9A159A0C9A149A809107018B7FF3
:10C0D000809307019FB7F894809108018460809352
:10C0E00008019FBF24982C9A809107018F77809335
:10C0F00007019FB7F8948091080180688093080138
:10C100009FBF809101018F7E809301019FB7F894BA
:10C11000809102018061809302019FBF389A40980C
:10C12000179A10925207399A4198169A109253070B
:10C130003A9A4298159A109254073B9A4398149A47
:10C14000809180008C7F8093800080918100877E29
:10C15000886080938100809180008F73809380003D
:10C1600080918100887F82608093810080E090E4EC
:10C17000909389008093880010928500109284002B
:10C1800080916F00826080936F0081E080938E04C5
:10C1900078940F94540D10928F048091010188605F
:10C1A00080930101549A2091590C222339F1009176
:10C1B0005A0C10915B0C215051F030E040E050E0FF
:10C1C0006FEF7FEF80E090E00F94053C02C020E02D
:10C1D00030E0F8014091560C5091570CCF01801B74
:10C1E000910B8417950740F44081429FC001439F03
:10C1F000900D11249193EECF1092590C8091580C10
:10C2000087FD06C061E067DA60E08091580C34DA9F
:10C2100081E08093530C0E9467DB60E070E080E077
:10C220009FEF0E94E0AC0E9440F064EC79E080E077
:10C2300090E00E945C9E80911C02811117C064EC0A
:10C2400079E080E090E00E945C9E10928E04109253
:10C250008D0470E6572EEDE04E2EFAE9CF2EFCE06D
:10C26000DF2EA0E0AA2EA0E0BA2E97C010921C02EA
:10C270002091CE0B30E0790188E3E81AF108F7FE4F
:10C2800004C0790197E3E91AF108F594E7942E5177
:10C29000310936952795F22E0E94F7A001E01BE0A8
:10C2A00023E147E06CE08E2D0E9436D884E00F94A5
:10C2B000142A0091CE0B10E002571109169507952C
:10C2C0006091CF0B62514DE653E08F2D0E94B6D89E
:10C2D0006091CF0B665043E753E0802F0E94B6D8A1
:10C2E0000E94FCD78111DACFAACF80911D0780FD73
:10C2F000CBC280911D0784FDC7C290E2F92E8091C8
:10C300001D0781FDDEC280911D0785FDDAC200E2B6
:10C3100080911D0782FDF1C280911D0786FDEDC24F
:10C3200010E28AE00F94452E1F926F921F921F9386
:10C330001F920F931F92FF92DF92CF921F920E9443
:10C34000D3DA10921D070FB6F894DEBF0FBECDBF33
:10C350008091C504882391F01092AF0C81EA9EE091
:10C360000E94E5CE81EA9EE00E9416CF1092AE0CAC
:10C370001092AD0C0E94F4910E94A6FA80911D02C9
:10C38000815009F4F0C080931D0280E00F94E823EF
:10C39000A114B10431F00E9400002AE0722E30E2B4
:10C3A000632E80916306843010F40E947BAD8091EF
:10C3B0005A0F8823E9F0EFDA0091560F1091570FCA
:10C3C0002091580F3091590FDC01CB01801B910B4C
:10C3D000A20BB30BB7FD0CC010925A0F8091B00C9A
:10C3E00081114FC20E949CA78091B00C811149C25B
:10C3F00080916306882309F498C08091AD0C88234E
:10C4000009F480C000916206509E800111240E51F3
:10C410001B4F6DED7CE0C8010F945637892BF9F066
:10C4200081EA9EE00E94E5CE81EA9EE00E9416CF5E
:10C430001092AE0C1092AD0CEAECFCE084918F01EE
:10C440000F5F1F4F882341F00F94452EF801F6CF60
:10C450008091AE0C811156C00F94A62755C0F801EB
:10C4600001900020E9F731977F01E01AF10A10925C
:10C47000A10E6EE470E0C8010F9462404C01009779
:10C4800029F4F7013197E00FF11F0EC060E270E070
:10C490000F9462408C010F5F1F4F6AE270E0C4018D
:10C4A0000F946240FC013197418272821382F8013D
:10C4B00001900020E9F73197AF01401B510BB80103
:10C4C00081EA9EE00E94D9CF8091A10E882309F4D1
:10C4D000BFCFE2EEF1E284918F010F5F1F4F8823FF
:10C4E00021F00F94452EF801F6CFE3E8FCE08491AB
:10C4F0008F010F5F1F4F882309F4AACF0F94452E99
:10C50000F801F5CF0E94CD2C80916306882369F055
:10C51000815080936306809162068F5F843018F4A7
:10C520008093620602C01092620680911D078823E4
:10C5300009F424CFEDEFF1E284918F010F5F1F4FDB
:10C54000882321F00F94452EF801F6CFEBEBFCE0A9
:10C5500084918F010F5F1F4F882309F4C6CE0F947B
:10C56000452EF801F5CF70921D020E9427568823B0
:10C5700009F40BCF8091510C9091C404981709F4E1
:10C580004CC08091510C8093C4041092C00410924E
:10C59000C1041092C2041092C3041092BC04109201
:10C5A000BD041092BE041092BF041092B804109201
:10C5B000B9041092BA041092BB041092B404109201
:10C5C000B5041092B6041092B7041092B004109201
:10C5D000B1041092B2041092B3041092AC04109201
:10C5E000AD041092AE041092AF041092A804109201
:10C5F000A9041092AA041092AB041092A404109201
:10C60000A5041092A6041092A7041092A004109200
:10C61000A1041092A2041092A3041092B20B1092E3
:10C62000B30B1092B40B1092B50B42EB5BE062E1DE
:10C6300083E59BE00E9479954091A0045091A1046C
:10C640006091A2047091A3048091B20B9091B30BFE
:10C65000A091B40BB091B50B840F951FA61FB71F07
:10C660008093A0049093A104A093A204B093A30488
:10C6700010923D0B10923E0B10923F0B1092400B0C
:10C680004DE35BE062E18EED9AE00E947995409186
:10C69000A4045091A5046091A6047091A704809110
:10C6A0003D0B90913E0BA0913F0BB091400B840F3E
:10C6B000951FA61FB71F8093A4049093A504A09371
:10C6C000A604B093A7041092C80A1092C90A109247
:10C6D000CA0A1092CB0A48EC5AE062E189E69AE075
:10C6E0000E9479954091A8045091A9046091AA04F0
:10C6F0007091AB048091C80A9091C90AA091CA0AAE
:10C70000B091CB0A840F951FA61FB71F8093A80472
:10C710009093A904A093AA04B093AB041092530A77
:10C720001092540A1092550A1092560A43E55AE0A4
:10C7300062E184EF99E00E9479954091AC045091B8
:10C74000AD046091AE047091AF048091530A909152
:10C75000540AA091550AB091560A840F951FA61F3E
:10C76000B71F8093AC049093AD04A093AE04B09334
:10C77000AF0483E59BE00E944A96DC01CB019170F7
:10C78000AA27BB270091B4041091B5042091B604E8
:10C790003091B704800F911FA21FB31F8093B40480
:10C7A0009093B504A093B604B093B7048EED9AE0CD
:10C7B0000E944A96DC01CB019170AA27BB27009109
:10C7C000B8041091B9042091BA043091BB04800FD1
:10C7D000911FA21FB31F8093B8049093B904A09334
:10C7E000BA04B093BB0489E69AE00E944A96DC0141
:10C7F000CB019170AA27BB270091BC041091BD0406
:10C800002091BE043091BF04800F911FA21FB31F5F
:10C810008093BC049093BD04A093BE04B093BF0466
:10C8200084EF99E00E944A96DC01CB019170AA271F
:10C83000BB270091C0041091C1042091C204309123
:10C84000C304800F911FA21FB31F8093C004909355
:10C85000C104A093C204B093C3048091B00490912A
:10C86000B104A091B204B091B3040196A11DB11D11
:10C870008093B0049093B104A093B204B093B30436
:10C8800084CD0E94EBA6B4CD6091D6047091D704FC
:10C890008091D8049091D9040F94DD372091C6047B
:10C8A0003091C7044091C8045091C9040F943C389A
:10C8B000AB01BC0187EB9CE00E94D79888E5F82E7D
:10C8C0001ECD6091DA047091DB048091DC049091BC
:10C8D000DD040F94DD372091CA043091CB044091E0
:10C8E000CC045091CD040F943C38AB01BC0183EBD8
:10C8F0009CE00E94D79809E50BCD6091DE04709111
:10C90000DF048091E0049091E1040F94DD372091E1
:10C91000CE043091CF044091D0045091D1040F94B3
:10C920003C38AB01BC018FEA9CE00E94D7981AE525
:10C93000F8CC0D948A14EF92FF920F931F93CF932C
:10C94000DF9300D01F92CDB7DEB71092790F8091A0
:10C95000E6069091E706A091E806B091E9068130DD
:10C960009048A105B10540F01092E6061092E70646
:10C970001092E8061092E9061091E6068091A8064A
:10C980001816DCF4282F082E000C330B2150310927
:10C99000412F012E000C550B4217530774F01FEF67
:10C9A000180F812F90E0A0E0B0E08093E60690930E
:10C9B000E706A093E806B093E9061092371080913D
:10C9C0004010181714F41093401080914010082E56
:10C9D000000C990B0496212F012E000C330B8217AB
:10C9E000930724F48CEF810F80934010E090401067
:10C9F000F12CE1101DC08091800F811106C0809143
:10CA00002D02882309F479C109C01111F8CF0E94C1
:10CA1000626D80913710882391F377C181E0111105
:10CA200080E024E04FE85EE06F2D0E9407EC65C1D6
:10CA300081E0E81228C08091800F811106C08091AA
:10CA40002D02882309F459C111C01130C1F720E02B
:10CA500030E040E251E464EA76E089E89EE00E943A
:10CA6000EE7B80913710882351F34FC184EA96E022
:10CA70000E94D59C9C0181E0113009F080E000E02B
:10CA800043E85EE038C122E0E21228C08091800FC6
:10CA9000811106C080912D02882309F42EC111C096
:10CAA0001230C1F720E030E048EC52E460EA76E072
:10CAB00089E79EE00E94EE7B80913710882351F336
:10CAC00024C180EA96E00E94D59C9C0181E012304E
:10CAD00009F080E000E04FE65EE00DC183E0E8127F
:10CAE00028C08091800F811106C080912D0288237B
:10CAF00009F403C111C01330C1F720E030E048EC65
:10CB000052E46CE976E086E69EE00E94EE7B80913E
:10CB10003710882351F3F9C08CE996E00E94D59C28
:10CB20009C0181E0133009F080E000E04DE55EE01B
:10CB3000E2C024E0E21236C08091800F811106C06D
:10CB400080912D02882309F4D8C011C01430C1F798
:10CB500024E630E040E050E06CE876E086E59EE0D8
:10CB60000F94CE3080913710882351F3CEC060915E
:10CB70008C0670918D0680918E0690918F060F9491
:10CB8000DB3769837A838B839C83CE0101960E9475
:10CB9000D59C9C0181E0143009F080E000E04FE476
:10CBA0005EE0A9C085E0E81236C08091800F811157
:10CBB00006C080912D02882309F49FC011C0153052
:10CBC000C1F724E630E040E050E060E976E088E438
:10CBD0009EE00F94CE3080913710882351F395C09A
:10CBE00060919006709191068091920690919306C3
:10CBF0000F94DB3769837A838B839C83CE01019604
:10CC00000E94D59C9C0181E0153009F080E000E095
:10CC100041E45EE070C026E0E21236C08091800FF1
:10CC2000811106C080912D02882309F466C011C0CD
:10CC30001630C1F72AE030E040E050E064E976E0E9
:10CC40008AE39EE00F94CE3080913710882351F311
:10CC50005CC06091940670919506809196069091C3
:10CC600097060F94DB3769837A838B839C83CE018D
:10CC700001960E94D59C9C0181E0163009F080E06D
:10CC800000E043E35EE037C087E0E81236C0809101
:10CC9000800F811105C080912D02882371F111C090
:10CCA0001730C9F724E630E040E050E068E976E06C
:10CCB0008CE29EE00F94CE3080913710882359F398
:10CCC00024C0609198067091990680919A0690917F
:10CCD0009B060F94DB3769837A838B839C83CE0119
:10CCE00001960E94D59C9C0181E0173009F080E0FC
:10CCF00000E045E25EE06F2DBED7F394E39425E0BB
:10CD0000F21277CE88E08093A8060F900F900F90D4
:10CD10000F90DF91CF911F910F91FF90EF900895A9
:10CD20002F924F926F927F928F929F92AF92BF926B
:10CD3000CF92DF92EF92FF920F931F93CF93DF93E7
:10CD40001092790F8091E6069091E706A091E8068F
:10CD5000B091E90681309048A105B10540F01092EC
:10CD6000E6061092E7061092E8061092E906D091C6
:10CD7000E60680918B061816DCF4282F082E000C8E
:10CD8000330B215031094D2F0D2E000C550B42173E
:10CD9000530774F0DFEFD80F8D2F90E0A0E0B0E0E4
:10CDA0008093E6069093E706A093E806B093E90621
:10CDB0001092371080914010D81714F4D09340107F
:10CDC00080914010082E000C990B04962D2F0D2EEB
:10CDD000000C330B8217930724F48CEF8D0F809394
:10CDE0004010C0914010412C63E0262E76EE672E55
:10CDF0007DE0772EEBEFCE2EEDE0DE2EF9E0AF2ECC
:10CE0000FEE0BF2EA0E18A2EAEE09A2EC1111CC01A
:10CE10008091800F811106C080912D02882309F432
:10CE2000A3C108C0D111F8CF4DD680913710882307
:10CE300099F3A2C181E0D11180E024E04EE15EE0EF
:10CE4000642D0E9407EC90C1C13009F03EC0809172
:10CE5000800F811106C080912D02882309F484C1BE
:10CE600016C0D130C1F7E12C10ECF12E09E714E423
:10CE700020E030E040E85FE36BE776E087E19EE0AA
:10CE80000E948EF080913710882329F375C12F926C
:10CE900087EE8F931F9281E08F938BE796E09F93AD
:10CEA0008F93BF92AF929F928F924F9281E0D13039
:10CEB00009F080E08F934ED78DB79EB70C960FB6D2
:10CEC000F8949EBF0FBE8DBF4FC1C23009F040C065
:10CED0008091800F811106C080912D02882309F472
:10CEE00043C116C0D230C1F7E12C10ECF12E09E796
:10CEF00014E420E030E040E85FE36FE776E082E0B2
:10CF00009EE00E948EF080913710882329F334C16F
:10CF10002F9287EE8F931F9281E08F938FE796E099
:10CF20009F938F93A4EFBDE0BF93AF93DF92CF9217
:10CF30004F9281E0D23009F080E08F930BD78DB70C
:10CF40009EB70C960FB6F8949EBF0FBE8DBF0CC156
:10CF5000C33009F040C08091800F811106C08091DC
:10CF60002D02882309F400C116C0D330C1F7E12C8B
:10CF700010ECF12E09E714E420E030E040E85FE334
:10CF800063E876E08DEE9DE00E948EF08091371090
:10CF9000882329F3F1C02F9287EE8F931F9281E0AF
:10CFA0008F9383E896E09F938F93AFEDBDE0BF939F
:10CFB000AF937F926F924F9281E0D33009F080E07F
:10CFC0008F93C8D68DB79EB70C960FB6F8949EBFB8
:10CFD0000FBE8DBFC9C0C43009F042C08091800F20
:10CFE000811106C080912D02882309F4BDC016C0AE
:10CFF000D430C1F7E12C10ECF12E09E714E420E065
:10D0000030E040E85FE367E876E088ED9DE00E946D
:10D010008EF080913710882329F3AEC02F9287EECF
:10D020008F931F9281E08F9387E896E09F938F9371
:10D03000AAECBDE0BF93AF93A1EDBDE0BF93AF936A
:10D040004F9281E0D43009F080E08F9383D68DB782
:10D050009EB70C960FB6F8949EBF0FBE8DBF84C0CE
:10D06000C53009F040C08091800F811106C08091C9
:10D070002D02882309F478C015C0D530C1F7E12C02
:10D0800010ECF12E09E714E420E030E0A90167E795
:10D0900076E085EC9DE00E948EF080913710882329
:10D0A00031F36AC02F9287EE8F931F921F9287E70A
:10D0B00096E09F938F93ABEBBDE0BF93AF93A0EC53
:10D0C000BDE0BF93AF934F9281E0D53009F080E08F
:10D0D0008F9340D68DB79EB70C960FB6F8949EBF2F
:10D0E0000FBE8DBF41C0C63009F03EC08091800F99
:10D0F000811105C080912D028823B1F115C0D63071
:10D10000C9F7E12C10ECF12E09E714E420E030E03F
:10D11000A90163E776E081EB9DE00E948EF08091AB
:10D120003710882339F328C02F9287EE8F931F92F0
:10D130001F9283E796E09F938F93ADE9BDE0BF9385
:10D14000AF93A7EABDE0BF93AF934F9281E0D63093
:10D1500009F080E08F93FED58DB79EB70C960FB681
:10D16000F8949EBF0FBE8DBF4394CF5F95E04912E8
:10D170004DCE87E080938B06DF91CF911F910F9169
:10D18000FF90EF90DF90CF90BF90AF909F908F90E7
:10D190007F906F904F902F9008950D94B715FF9248
:10D1A0000F931F93CF93DF931092790F8091E60630
:10D1B0009091E706A091E806B091E9068130904889
:10D1C000A105B10540F01092E6061092E706109214
:10D1D000E8061092E906C091E606809172061816DC
:10D1E000DCF4282F082E000C330B215031094C2F72
:10D1F0000C2E000C550B4217530774F0CFEFC80FDD
:10D200008C2F90E0A0E0B0E08093E6069093E706D4
:10D21000A093E806B093E906109237108091401071
:10D22000C81714F4C093401080914010082E000CD1
:10D23000990B04962C2F0C2E000C330B821793079E
:10D2400024F48CEF8C0F8093401010914010D0E0AC
:10D25000FF24F394111119C08091800F811106C031
:10D2600080912D02882309F4D7C008C0C111F8CFDE
:10D2700029D480913710882399F3D5C081E0C1115A
:10D2800080E024E048E95DE0C4C01130A1F5809160
:10D29000800F811106C080912D02882309F4BCC043
:10D2A0001BC0C130C1F7C093790F1092750F109257
:10D2B000760F1092770F1092780F22E031E042E261
:10D2C00051E060E776E081E99DE00E949D7B8091DE
:10D2D0003710882301F3A7C08091700690917106E2
:10D2E0000E94269E9C0181E0C13009F080E000E0B0
:10D2F0004AE85DE06BC01230A1F58091800F81118A
:10D3000006C080912D02882309F486C01BC0C2305C
:10D31000C1F7F092790F1092750F1092760F10925C
:10D32000770F1092780F26EF30E047E850E06EE676
:10D3300076E086E89DE00E949D7B809137108823EF
:10D3400001F371C080916E0690916F060E94269E37
:10D350009C0181E0C23009F080E000E042E85DE03D
:10D3600035C01330B1F58091800F811106C08091D6
:10D370002D02882309F450C01BC0C330C1F7F092BE
:10D38000790F1092750F1092760F1092770F1092FE
:10D39000780F2FEF30E040E050E06CE676E088E771
:10D3A0009DE00E9405F180913710882301F33BC076
:10D3B00080916C0690916D060E94269E9C0181E0F2
:10D3C000C33009F080E000E04EE65DE06D2F53D4FD
:10D3D00023C0143009F58091800F811105C0809120
:10D3E0002D028823C9F00EC0C430C9F710926D0613
:10D3F00010926C060E94A6FA5FD3809137108823A2
:10D4000071F311C081E0C43009F080E020E245E60C
:10D410005DE06D2F0E9407ECDF5F1F5FD53009F0E4
:10D4200019CFD0937206DF91CF911F910F91FF908A
:10D4300008951F93CF93DF931092790F8091E606A2
:10D440009091E706A091E806B091E90681309048F6
:10D45000A105B10540F01092E6061092E706109281
:10D46000E8061092E906C091E60680916B06181650
:10D47000DCF4282F082E000C330B215031094C2FDF
:10D480000C2E000C550B4217530774F0CFEFC80F4A
:10D490008C2F90E0A0E0B0E08093E6069093E70642
:10D4A000A093E806B093E9061092371080914010DF
:10D4B000C81714F4C093401080914010082E000C3F
:10D4C000990B04962C2F0C2E000C330B821793070C
:10D4D00024F48CEF8C0F8093401010914010D0E01A
:10D4E000111119C08091800F811106C080912D0209
:10D4F000882309F48CC008C0C111F8CFE3D2809111
:10D500003710882399F38AC081E0C11180E024E0BC
:10D510004CE55DE079C01130E9F48091800F811114
:10D5200006C080912D02882309F471C00BC0C13060
:10D53000C1F78BE99CE60E9479F08091371088232F
:10D5400081F36CC081E0C13009F080E023E045E563
:10D550005DE05AC01230E9F48091800F811106C05D
:10D5600080912D02882309F452C00BC0C230C1F74C
:10D570008FE99CE60E9479F080913710882381F32F
:10D580004DC081E0C23009F080E023E04EE45DE070
:10D590003BC01330E1F48091800F811105C0809170
:10D5A0002D028823A1F10BC0C330C9F783EA9CE6A2
:10D5B0000E9479F080913710882389F32FC081E091
:10D5C000C33009F080E023E047E45DE01DC0143083
:10D5D000F1F48091800F811105C080912D02882384
:10D5E000B1F00BC0C430C9F787EA9CE60E9479F01D
:10D5F00080913710882389F311C081E0C43009F08D
:10D6000080E023E04EE35DE06D2F0E9407ECDF5FDA
:10D610001F5FD53009F064CFD0936B06DF91CF91B7
:10D620001F91089562E088EE9CE00D94BA1B61E0C2
:10D6300081EE9CE00D94BA1B0F931F93CF93DF9361
:10D64000082F70936A06609369061092790F809193
:10D65000E6069091E706A091E806B091E9068130D0
:10D660009048A105B10540F01092E6061092E70639
:10D670001092E8061092E906C091E60680916806CD
:10D680001816DCF4282F082E000C330B215031091A
:10D690004C2F0C2E000C550B4217530774F0CFEF94
:10D6A000C80F8C2F90E0A0E0B0E08093E606909346
:10D6B000E706A093E806B093E90610923710809130
:10D6C0004010C81714F4C093401020914010022E4F
:10D6D000000C330B2C5F3F4F8C2F0C2E000C990B42
:10D6E0002817390724F48CEF8C0F80934010109189
:10D6F0004010D0E091E0013049F1023009F44AC015
:10D7000001116CC0111191C09923B1F01C16A4F045
:10D710008091E6069091E706A091E806B091E906AF
:10D720000196A11DB11D8093E6069093E706A09394
:10D73000E806B093E906CF5F80912D02882309F4B3
:10D74000EDC021E041E067E37DE06BC011116DC0E9
:10D750009923B1F01C16A4F08091E6069091E7069B
:10D76000A091E806B091E9060196A11DB11D809334
:10D77000E6069093E706A093E806B093E906CF5F2C
:10D7800080912D02882309F4C9C021E041E060E3C3
:10D790007DE047C0111149C09923B1F01C16A4F0D7
:10D7A0008091E6069091E706A091E806B091E9061F
:10D7B0000196A11DB11D8093E6069093E706A09304
:10D7C000E806B093E906CF5F80912D02882309F423
:10D7D000A5C021E041E069E27DE023C0111125C030
:10D7E0009923B1F01C16A4F08091E6069091E7060B
:10D7F000A091E806B091E9060196A11DB11D8093A4
:10D80000E6069093E706A093E806B093E906CF5F9B
:10D8100080912D02882309F481C021E041E060E27B
:10D820007DE08D2F0E94407B79C01130D1F4809132
:10D83000800F811106C080912D02882309F46EC0EB
:10D8400008C0C130C1F73ED180913710882399F3C9
:10D850006DC081E0C13009F080E024E046E15DE088
:10D860005AC01230E9F48091800F811106C0809176
:10D870002D02882309F452C00BC0C230C1F78EEBD1
:10D880009CE60E9479F080913710882381F34EC086
:10D8900081E0C23009F080E023E04CE05DE03BC075
:10D8A0001330E1F48091800F811105C080912D0229
:10D8B0008823A1F10BC0C330C9F783EC9CE60E941A
:10D8C00079F080913710882389F330C081E0C3302C
:10D8D00009F080E023E043E05DE01DC01430F1F486
:10D8E0008091800F811105C080912D028823B1F0B5
:10D8F0000BC0C430C9F788EC9CE60E9479F0809197
:10D900003710882389F312C081E0C43009F080E029
:10D9100023E048EF5CE06D2F0E9407ECDF5F1F5FA4
:10D9200090E0D53009F0E7CED0936806DF91CF9133
:10D930001F910F91089564E171E080E07DCE67E171
:10D940007BE681E079CE62E17BE682E075CE6DEC2C
:10D950007CE683E071CE21E020936E0F6093640635
:10D9600070936506809366069093670640E050E0EA
:10D97000BA018091690690916A067BC060E070E010
:10D9800080E291E4E8CF60E070E080E89FE3E3CFDD
:10D990006DEC7CEC8CEC9DE3DECF8091800F8111EF
:10D9A00091C06091E6067091E7068091E80690913B
:10D9B000E906611571058105910571F10F94DD3757
:10D9C0002091640630916506409166065091670685
:10D9D0000F943C389B01AC0160913E0770913F076A
:10D9E00080914007909141070F94413C60933E071E
:10D9F00070933F0780934007909341071092E6068B
:10DA00001092E7061092E8061092E90683E00F9460
:10DA1000841B81E080932D0280912D02882341F0A8
:10DA20008EE397E00E94779DBC018FEE9CE05FC083
:10DA300008958091CD068630D8F496E0899FF00154
:10DA40001124E755F94F20911E0230911F023183B6
:10DA500020834091E6065091E7066091E8067091B8
:10DA6000E90642835383648375838F5F8093CD0679
:10DA7000089520911E0230911F0228173907D9F00E
:10DA800090931F0280931E024093E6065093E70690
:10DA90006093E8067093E90687539F4621F410923D
:10DAA0006E0F1092CD0682E080932D0281E080936C
:10DAB000371010927A0F089540E050E0BA0187E3E2
:10DAC0009FE6D7CFE091CD06EE2381F0E150E093C1
:10DAD000CD0686E0E89FF0011124E755F94F428119
:10DAE00053816481758180819181C3CFE5CFAF92ED
:10DAF000BF92CF92DF92EF92FF920F931F93CF933B
:10DB0000DF935C017B0120E030E0F501E20FF31FC1
:10DB1000E491EE2319F02F5F3F4FF7CFF701CF01CC
:10DB20008E199F0941914111FACF04E110E0081BC1
:10DB300011093327021713071CF0DD24D39402C008
:10DB400082E0D82E8091CF0B90E06D2D70E06F5F5A
:10DB50007F4F0F941D3FC62EC6E0C60F8091020C6A
:10DB6000C81750F08091040C90E02C2F30E02B501F
:10DB70003109821793079CF5D0E0E114F104C1F15B
:10DB80008AE30E9438D982E0D8120FC0CC0D809170
:10DB9000020CC81768F12091040C30E08C2F90E043
:10DBA0000B97281739071CF423C0DD2309F1802FB8
:10DBB000880F080F000F0093050CC093060C80E23D
:10DBC0000E9438D9C701DF91CF911F910F91FF902B
:10DBD000EF90DF90CF90BF90AF900D94662A109297
:10DBE000050CC093060CC5010F94592AD1E0C5CF8E
:10DBF000DF91CF911F910F91FF90EF90DF90CF9029
:10DC0000BF90AF9008950F934CE0849F402D112456
:10DC100021E0240F2093F9068CE0840F8093FA060C
:10DC2000E091020CF0E090E002968E179F070CF155
:10DC3000822F90E02091040C30E082179307CCF4FF
:10DC4000662371F081E08093EE0B4D5F0BE020E8DE
:10DC500060E08EEC9BE00E943C591092EE0B03C0FA
:10DC600081E08093EE0B8091FA061092050C809370
:10DC7000060C0F910895CF92DF92EF92FF920F93CF
:10DC8000CF93DF93982F862F6A017901692FBBDF2D
:10DC90009091020C8091FA06891708F453C0909174
:10DCA000040C8091F906981708F44CC0002359F031
:10DCB00060E070E0F701E60FF71FE491EE2351F00A
:10DCC0006F5F7F4FF7CFD701BD016E197F098D912F
:10DCD0008111FACFC62FD4E1D61BF6018491882397
:10DCE00039F00F942E2AD81BFFEFCF1ADF0AF5CF99
:10DCF0008AE30E9438D9DD2329F080E20E9438D9D6
:10DD0000D150F9CF8091FA066AEFC69F602D112499
:10DD100060586093050C8093060CC701002349F0FE
:10DD2000DF91CF910F91FF90EF90DF90CF900D9406
:10DD3000592ADF91CF910F91FF90EF90DF90CF9014
:10DD40000D94662ADF91CF910F91FF90EF90DF90B5
:10DD5000CF9008950F93CF93DF93CDB7DEB7ED85C6
:10DD6000FE8560817181828193810F94853DCB0115
:10DD70000E94269E00E09C0149855A8568858F8116
:10DD80007ADFDF91CF910F9108959CE0899F802DDC
:10DD9000112421E0280F2093F906845F8093FA066E
:10DDA0006091020C70E0482F50E04E5F5F4F4617C5
:10DDB0005707CCF130E04091040C50E024173507B0
:10DDC00094F59EE39093050C8093060C85E40F94E4
:10DDD000452A8091FB068F5C0F94452A80E20F94C0
:10DDE000452A60914A1570914B1580914C15909180
:10DDF0004D150F94853DCB010E94269E0F94662AF7
:10DE00008FE20F94452A0E9408F0811104C080918E
:10DE10007509811108C080917006909171060E9469
:10DE2000269E0D94662A0895CF93DF931F92CDB757
:10DE3000DEB78091070C811107C081E08093070C49
:10DE40008EEC9BE00E9457596091D00B7091D10BE2
:10DE500019829E012F5F3F4F4FE08EEC9BE00E94A6
:10DE60007A570F94D3290F90DF91CF9108954F9255
:10DE70005F926F927F928F929F92AF92BF92FF922A
:10DE80000F931F93CF93DF93CDB7DEB72E970FB6C7
:10DE9000F894DEBF0FBECDBF1092790F8091800F36
:10DEA000882341F0C1DF40E050E0BA018EE091E00C
:10DEB000E0DD5DC420918402309185024091E60648
:10DEC0005091E7066091E8067091E906C901840F58
:10DED000951F2436310524F4853691053CF416C08F
:10DEE0002436310531F08436910584F484E690E0DF
:10DEF0000DC04B3051056105710514F00A9706C03D
:10DF0000463F5F4F6F4F7F4F6CF40A9690938502A8
:10DF1000809384021092E6061092E7061092E806BB
:10DF20001092E90680918402909185028A309105D1
:10DF30003CF0883E23E092072CF087EE93E002C08D
:10DF40008AE090E090938502809384020E9408F01A
:10DF5000F82E0E9446EC8091020C853198F4FF2047
:10DF600049F080916C0690916D06892B19F008E6B6
:10DF70001AE102C00BE419E123E14FE061E089E01E
:10DF80000E9436D88091020C8D3108F084C188300F
:10DF900008F03FC080917509F11002C0811139C0AD
:10DFA0006091700670917106072E000C880B990B1A
:10DFB0000F94DD3720E030E040E05FE30F94413C18
:10DFC0000F94853D643671052CF46A30710524F494
:10DFD00046E003C042E101C04CE022E130E0241BF6
:10DFE000310937FF02C02F5F3F4F35952795319597
:10DFF000219531092B5F2093050C27E02093060C17
:10E00000CB010E94269E0F94662A88E499E10F9422
:10E01000592A8091020C8D31D0F58091040C853104
:10E02000B0F120E030E040E05FE360914A1570918C
:10E030004B1580914C1590914D150F94413C0F94C8
:10E04000853D9B01643671050CF098C22A3031057C
:10E050000CF092C246E022E130E0241B310937FF88
:10E0600002C02F5F3F4F3595279531952195310996
:10E070002B5F2093050C2CE12093060CCB010E9412
:10E08000269E0F94662A88E499E10F94592A80917C
:10E09000020C853140F58091040C813120F16091B2
:10E0A000700670917106072E000C880B990B0F9467
:10E0B000DD3720914A1530914B1540914C15509108
:10E0C0004D150F94673E18160CF05AC21092EE0BC5
:10E0D00002E022E041E16DE08EEC9BE00E943C59C1
:10E0E00081E08093EE0B8091020C883008F03FC0F5
:10E0F00080916C09F11002C0811139C060916E06E7
:10E1000070916F06072E000C880B990B0F94DD376A
:10E1100020E030E040E05FE30F94413C0F94853D08
:10E12000643671052CF46A30710524F446E003C0AE
:10E1300042E101C04CE022E130E0241B310937FF0D
:10E1400002C02F5F3F4F35952795319521953109B5
:10E150002F5A2093050C27E02093060CCB010E9438
:10E16000269E0F94662A88E499E10F94592A80919B
:10E17000020C8D31D0F58091040C8531B0F120E096
:10E1800030E040E05FE36091CE067091CF06809171
:10E19000D0069091D1060F94413C0F94853D9B0190
:10E1A000643671050CF0F7C12A3031050CF0F1C16D
:10E1B00046E022E130E0241B310937FF02C02F5F27
:10E1C0003F4F359527953195219531092F5A209349
:10E1D000050C2CE12093060CCB010E94269E0F9487
:10E1E000662A88E499E10F94592A8091020C8531BE
:10E1F00040F58091040C813120F160916E067091A0
:10E200006F06072E000C880B990B0F94DD372091B9
:10E21000CE063091CF064091D0065091D1060F9492
:10E22000673E18160CF0B9C11092EE0B02E022E026
:10E2300042E168E58EEC9BE00E943C5981E08093CE
:10E24000EE0B8091020C8C3130F58091040C8431FE
:10E2500010F180916C0690916D06019644E6489FFE
:10E260009001499F300D112437FF02C021503F4FCC
:10E27000832F932F990F990B009769F028E620932D
:10E28000050C2BE12093060C0E94269E0F94662A13
:10E2900085E20E9438D98091020C843328F4809161
:10E2A000040C8A3208F082C18091020C853328F474
:10E2B0008091040C813308F09FC18091AF0C8823BA
:10E2C00009F44BC08091020C843308F046C0809161
:10E2D000040C823308F441C02091A40E222319F1CA
:10E2E00080914E0F90914F0FA091500FB091510F10
:10E2F0000097A105B10509F484C1BC01CD016D5998
:10E300007F4F8F4F9F4F24E630E040E050E00F9466
:10E31000E33B6091520F7091530F8091540F909195
:10E32000550F0F94E33B88E4289FB0011124072E7A
:10E33000000C880B990B0F94DD372AE037ED43E290
:10E340005CE30F943C380F948A3D262F02E042E3B1
:10E3500067E38EEC9BE00E943C598091020C813374
:10E3600028F48091040C893208F04DC1E091C80B6B
:10E37000F091C90B84818111CBC0609132077091FB
:10E38000330780913407909135070F94853DCB0179
:10E390000E94BF9DBC0181EE96E00F946D4060919C
:10E3A00036077091370780913807909139070F949D
:10E3B000853DCB010E94BF9DBC018CED96E00F9482
:10E3C0006D402CEA35EC47E257E360913A077091D3
:10E3D0003B0780913C0790913D070F94413C20E022
:10E3E00030E048EC52E40F943C380F94853D4B01EB
:10E3F0005C0197FD16C0603127E272078105910527
:10E40000D4F020E137E240E050E00F94053CCA012F
:10E41000B9012AE030E040E050E00F94053C605D37
:10E420000BC0B094A09490948094811C911CA11C6A
:10E43000B11C6DE201C060E260939C1788EE881603
:10E4400083E09806A104B10494F0C501B40128EE5C
:10E4500033E040E050E00F94053CCA01B9012AE0E6
:10E4600030E040E050E00F94053C605D01C060E2A8
:10E4700060939D17C501B40124E630E040E050E010
:10E480000F94053C8AE0482E512C612C712CCA0156
:10E49000B901A30192010F94053C605D60939E1742
:10E4A000C501B401A30192010F94053C4B015C012D
:10E4B000672B682B692B79F08EE280939F17CA0136
:10E4C000B901A30192010F94053C605D6093A01710
:10E4D00080E3880D15C0CA01B901A30192010F9410
:10E4E000053C662339F08EE280939F17605D609350
:10E4F000A01705C080E28093A01780939F1780E249
:10E500008093A1176CE977E185ED96E00F946D405B
:10E510008091020C8632A8F48091040C8E3188F030
:10E5200008E020E84EE160E08EEC9BE00E943C5960
:10E530008091020C863228F48091040C8F3108F00F
:10E5400087C08091020C823328F48091040C8C32B5
:10E5500008F0EEC08091020C8F3308F008C1809162
:10E56000040C883308F403C11092050C8EE38093E9
:10E57000060C0E94E7A0FBC04CE06DCD42E16BCDE4
:10E5800002E022E041E16DE08EEC9BE00E943C590C
:10E59000AACD4CE00ECE42E10CCE02E022E042E1F8
:10E5A00068E58EEC9BE00E943C594BCE07E028E0EA
:10E5B0004AE26AE28EEC9BE00E943C5905E022E0D0
:10E5C0004CE262E38EEC9BE00E943C596AE08AE2F6
:10E5D0000E948CD86091D00B7091D10B82E3809314
:10E5E000EA0B8BE28093EB0B2AEE3BE042E38EECEE
:10E5F0009BE00E947A5758CE6AE486E30E948CD84A
:10E600005CCE20E090CE85E89CE00E94809E6B87E7
:10E610007C878D879E8741E06138714581409105F7
:10E6200008F440E0BE016F5F7F4FCE010B960E9461
:10E63000CB54982F990F890F8195855A8093050C9B
:10E6400080E38093060CCE0101960F94662A8ECE4D
:10E650001092EE0B83E08093050C85E28093060C0C
:10E66000FF2029F086E499E10F94592A0DC080918A
:10E67000D206811102C08FE305C08091520781113B
:10E68000F1CF80E20E9438D98BE08093050C15E22F
:10E690001093060C81EE96E00F94662A8BE280932D
:10E6A000050C1093060CFF2029F084E499E10F94E7
:10E6B000592A0DC08091D306811102C08FE305C095
:10E6C000809153078111F1CF80E20E9438D983E312
:10E6D0008093050C15E21093060C8CED96E00F94D8
:10E6E000662A83E58093050C1093060CFF2029F021
:10E6F00082E499E10F94592A0DC08091D4068111CA
:10E7000002C08FE305C0809154078111F1CF80E2F0
:10E710000E9438D98BE58093050C85E28093060C26
:10E7200085ED96E00F94662A81E08093EE0B09CF89
:10E7300084E00F94142A83E08093050C12E3109375
:10E74000060C86E00F94452A0E9446EC8CE08093EC
:10E75000050C1093060C80918402909185020E9412
:10E76000269E0F94662A85E20E9438D9F3CE2E9613
:10E770000FB6F894DEBF0FBECDBFDF91CF911F91D2
:10E780000F91FF90BF90AF909F908F907F906F9070
:10E790005F904F9008950F931F93CF93DF93CDB762
:10E7A000DEB728970FB6F894DEBF0FBECDBF00E0EE
:10E7B00010E020E830EC0D831E832F83388720E0A3
:10E7C00030E040E752E40F941D3D69837A838B83E8
:10E7D0009C83BE016F5F7F4FCE0105960E9413ACF4
:10E7E00010911D0710921D070F94352781E197E0C6
:10E7F0000E94B1C88091190790911A07A0911B0738
:10E80000B0911C0780933A0790933B07A0933C0775
:10E81000B0933D070E9417B012FB112710F981E059
:10E82000812728960FB6F894DEBF0FBECDBFDF91CB
:10E83000CF911F910F910895CF938091850CC1E0E6
:10E840008230E9F0C0E0813009F446C010928A0CB1
:10E8500010928B0C10928C0C10928D0C10928E0CCE
:10E8600010928F0C1092900C1092910C1092860CBA
:10E870001092870C1092880C1092890C0CC085E8BD
:10E880009CE00E94809E6093860C7093870C80931E
:10E89000880C9093890C81E08093850C0E94CB5C5E
:10E8A00060938A0C70938B0C80938C0C90938D0CDE
:10E8B000C11112C08091920C9091930C019690938B
:10E8C000930C8093920C1092A80C1092A90C1092A9
:10E8D000AA0C1092AB0CC1E08C2FCF910895EF924F
:10E8E000FF921F93CF93DF93D091520781E0D827F7
:10E8F000109153071827C0915407C827D11102C09F
:10E90000112319F0EDEFF1E203C0C111FBCF7EC07E
:10E9100084917F019FEFE91AF90A882321F00F946F
:10E92000452EF701F5CFE0EBFCE184917F019FEFED
:10E93000E91AF90A882321F00F94452EF701F5CF43
:10E94000DD2369F0EEEAFCE184917F019FEFE91A93
:10E95000F90A882321F00F94452EF701F5CF1123F2
:10E9600069F0ECEAFCE184917F019FEFE91AF90A72
:10E97000882321F00F94452EF701F5CFC11103C074
:10E98000E2EAFCE10DC0EAEAFCE184917F019FEF3D
:10E99000E91AF90A8823A1F30F94452EF701F5CF60
:10E9A00084917F019FEFE91AF90A882321F00F94DF
:10E9B000452EF701F5CFC11103C041EF53E002C06E
:10E9C00047E853E0111103C021EF33E002C029E80A
:10E9D00033E0D11103C081EF93E002C08BE893E0F4
:10E9E0005F934F933F932F939F938F9380E99CE185
:10E9F0009F938F931F920E94D3DA8DB79EB709968B
:10EA00000FB6F8949EBF0FBE8DBFC1E08C2FDF9173
:10EA1000CF911F91FF90EF900895CF92DF92EF92E8
:10EA2000FF92C0903E07D0903F07E0904007F090E3
:10EA3000410720914E0730914F0740915007509168
:10EA40005107C701B6010F943C380F94723E609392
:10EA50004C0C70934D0C80934E0C90934F0CC7014F
:10EA6000B6010F94853D2FB7F89460932E077093ED
:10EA70002F0780933007909331072FBF10923C0CE3
:10EA800010923D0C10923E0C10923F0CFF90EF90B4
:10EA9000DF90CF900895CF92DF92EF92FF92CF93C5
:10EAA000DF93CDB7DEB728970FB6F894DEBF0FBE61
:10EAB000CDBF80E090E0A0EAB0E48D839E83AF8379
:10EAC000B887C0901E07D0901F07E0902007F090F5
:10EAD000210720E030E0A901C701B6010F94D73724
:10EAE00087FF0CC0A701960160E070E080EA90E427
:10EAF0000F94403C6D837E838F83988720913A07E3
:10EB000030913B0740913C0750913D076D817E81DC
:10EB10008F8198850F94673E18165CF419821A82CB
:10EB20001B821C82BE016F5F7F4FCE0105960E9443
:10EB300013AC28960FB6F894DEBF0FBECDBFDF91A1
:10EB4000CF91FF90EF90DF90CF9008950F931F9398
:10EB5000CF93DF93FC018491EF012196882321F06C
:10EB60000F94452EFE01F7CFC0E0D3E0DC0F84E028
:10EB7000C89F80011124F801E85FF34F20E030E0E6
:10EB8000A90160817181828193810F94673E87FD25
:10EB900003C08BE20F94452EF801E85FF34F6081CC
:10EBA00071818281938146E00F941E2F80E20F9441
:10EBB000452ECF5FCD13DBCF8AE00F94452EC930B1
:10EBC000A1F6DF91CF911F910F910895E82FF0E00A
:10EBD000E65BF34EE4918E2F90E0FC013797EC302A
:10EBE000F10508F58827EA56FF4F8F4F0D94303F07
:10EBF0008091B100887F84608093B10008958091F6
:10EC00009100887F84608093910008958091A10095
:10EC1000887F84608093A100089580912101887F7E
:10EC200084608093210108954F925F926F927F924A
:10EC30008F929F92AF92BF92EF92FF920F931F938A
:10EC4000CF93DF93EC014A015B0179010E94A99700
:10EC5000FE01ED58FF4F60817181CE010E9460D9A5
:10EC60008E01015B1F4FF80180819181A281B381E8
:10EC7000B07FB46080839183A283B383A8016CEEDC
:10EC8000CE010E94799562E0CE010E94CB9665E0AC
:10EC9000CE010E945E97F80180819181A281B381AB
:10ECA000B06180839183A283B383A8016CEECE010F
:10ECB0000E947995AE014D595F4F80E890E0A0E049
:10ECC000B0E0FA0180839183A283B38361E9CE012E
:10ECD0000E9479956FEFCE010E942E9764E0CE01DD
:10ECE0000E94FB968B859C85AD85BE859F7E8B871C
:10ECF0009C87AD87BE8704541109A80160E8CE0146
:10ED00000E9479958B859C85AD85BE859F7D8B877F
:10ED10009C87AD87BE87A80160E8CE010E947995E7
:10ED20008B859C85AD85BE8591608B879C87AD87E3
:10ED3000BE87A80160E8CE010E9479958B859C85ED
:10ED4000AD85BE8580618B879C87AD87BE87A80116
:10ED500060E8CE010E9479958B859C85AD85BE8546
:10ED60008E7F8B879C87AD87BE87A80160E8CE0128
:10ED70000E9479958B859C85AD85BE858D7F8B871F
:10ED80009C87AD87BE87A80160E8CE010E94799577
:10ED9000005B1F4FF80180819181A281B381AC7F1C
:10EDA00080839183A283B383A80160EFCE010E9488
:10EDB0007995F80180819181A281B381A4608083DB
:10EDC0009183A283B383A80160EFCE010E9479955D
:10EDD000F80180819181A281B38199279560808318
:10EDE0009183A283B383A80160EFCE010E9479953D
:10EDF000F80180819181A281B3818F6F808391839B
:10EE0000A283B383A80160EFCE010E94799561E0EF
:10EE1000CE010E942496CE010E948297DC0120E15F
:10EE200036E041EC50E00F94213C0F94DB372B018E
:10EE30003C019A2D892D782D66270F94DB37F70139
:10EE400020813181428153810F943C389B01AC0178
:10EE5000C301B2010F941D3D0F948A3D6F8B788FD3
:10EE6000898F9A8FAE01495E5F4F63E9CE01DF91D2
:10EE7000CF911F910F91FF90EF90BF90AF909F9017
:10EE80008F907F906F905F904F900C947995FC01DC
:10EE9000DB018C9120813181382798E0A901440F52
:10EEA000551F37FD06C09A019150C1F73183208369
:10EEB00008959A01B1E22B27B0E13B27F5CF2F92BD
:10EEC0003F924F925F926F927F928F929F92AF92FA
:10EED000BF92CF92DF92EF92FF920F931F93CF9347
:10EEE000DF93CDB7DEB76B970FB6F894DEBF0FBEDA
:10EEF000CDBF9F8B8E8B1B01488F298FFC016081BA
:10EF0000718182819381698B7A8B8B8B9C8BF101D0
:10EF1000C080D180E280F380CD86DE86EF86F88ADD
:10EF20004090090750900A0760900B0770900C07FB
:10EF30002091050730910607409107075091080777
:10EF40000F94403C4B015C0122E630E140E450EC80
:10EF50000F94673E87FD24C022E430E042E253E490
:10EF6000C501B4010F94D7371816D4F0A30192014C
:10EF7000C701B6010F94403C6B017C0121E338E0EE
:10EF800040EE50EC0F94673E87FD0AC022E430E06B
:10EF90004EE353E4C701B6010F94D73718162CF48B
:10EFA000A12CB12C00EC1FE744C3C0902502D090E7
:10EFB0002602E0902702F09028028091FD06811140
:10EFC00007C0809124028093FC0681E08093FD06B7
:10EFD0008091200290912102A0912202B0912302FF
:10EFE0008093250290932602A0932702B0932802D3
:10EFF00052DD19821A821B821C82AE014F5F5F4F65
:10F00000BE01635F7F4FCE0141960E940FAC81E04D
:10F010000E94C9AB811192C20E94D75C04E010E04B
:10F02000812C912CE8E4AE2EE2E4BE2E412C512C32
:10F03000F0E26F2EF1E47F2E60E070E88BE395E460
:10F04000AADB882309F4FFC00150110909F0C1C0EF
:10F05000E6EFFBE184918F010F5F1F4F882321F0C2
:10F060000F94452EF801F6CF60E087EE9BE10E94F9
:10F07000C5EC50E7C52E53E0D52EDE82CD8269E186
:10F08000E62EF12CFA82E982BE016B5F7F4FCE0142
:10F0900001960E94E6A81E821D8202E310E01A83F8
:10F0A0000983BE016B5F7F4FCE0101960E94E6A8E7
:10F0B000DE82CD82FA82E982BE016B5F7F4FCE0194
:10F0C00001960E94E6A81E821D821A830983BE0152
:10F0D0006B5F7F4FCE0101960E94E6A8DE82CD8253
:10F0E000FA82E982BE016B5F7F4FCE0101960E94DA
:10F0F000E6A81E821D821A830983BE016B5F7F4FC3
:10F10000CE0101960E94E6A880E090E0A8E4B2E477
:10F110008D839E83AF83B88780E090E0A8ECB2E453
:10F1200089839A83AB83BC83BE016B5F7F4FCE0123
:10F1300001960E9413AC10923E0710923F07109266
:10F14000400710924107C090FB0680913A079091CA
:10F150003B07A0913C07B0913D0740913607509185
:10F160003707609138077091390700913207109185
:10F170003307209134073091350709831A832B8395
:10F180003C834D835E836F83788789879A87AB87BB
:10F19000BC87AE01475F5F4FBE016B5F7F4FCE0103
:10F1A00001960E9420CAE12CF12C00EA1FE32EE315
:10F1B00037E0AE01475F5F4FBE016B5F7F4FCE010F
:10F1C00001960E9408BC29DC0E94CAFF88ED9BE1E1
:10F1D0001EC1EFE0FCE184919F012F5F3F4F882328
:10F1E00041F02A8F3B8F0F94452E2A8D3B8DF901DC
:10F1F000F2CF60E08FEC9BE10E94C5EC8D829E8295
:10F20000AF82B88649825A826B827C82BE016B5F74
:10F210007F4FCE0101960E9413AC1D8A19821A827B
:10F220001B821C82FCE0F9871D829E012B5E3F4FF2
:10F23000AE014F5F5F4FBE01675F7F4FCE01059606
:10F240000E945C99F9CE80E090E0A8E4B2E48D835E
:10F250009E83AF83B88720E030E040EA50E46091BD
:10F260003A0770913B0780913C0790913D070F94BE
:10F27000413C69837A838B839C83BE016B5F7F4FA4
:10F28000CE0101960E9413AC04E010E0812C912C79
:10F2900030E8A32E3FE3B32E412C512C40E2642EE4
:10F2A00041E4742EDFC060E08DE99BE10E94C5EC73
:10F2B00080E7C82E83E0D82EDE82CD8299E1E92E48
:10F2C000F12CFA82E982BE016B5F7F4FCE0101967D
:10F2D0000E94E6A81E821D8202E310E01A830983C1
:10F2E000BE016B5F7F4FCE0101960E94E6A8DE82D1
:10F2F000CD82FA82E982BE016B5F7F4FCE0101961B
:10F300000E94E6A81E821D821A830983BE016B5FDC
:10F310007F4FCE0101960E94E6A8DE82CD82FA825E
:10F32000E982BE016B5F7F4FCE0101960E94E6A885
:10F330001E821D821A830983BE016B5F7F4FCE013F
:10F3400001960E94E6A880E090E0A8E4B2E48D83F4
:10F350009E83AF83B88780E090E0A8ECB2E4898315
:10F360009A83AB83BC83BE016B5F7F4FCE01019656
:10F370000E9413AC10923E0710923F071092400774
:10F3800010924107C090FB0680913A0790913B078D
:10F39000A0913C07B0913D07409136075091370747
:10F3A0006091380770913907009132071091330747
:10F3B000209134073091350709831A832B833C83CE
:10F3C0004D835E836F83788789879A87AB87BC87F5
:10F3D000AE01475F5F4FBE016B5F7F4FCE0101966D
:10F3E0000E9420CAE12CF12C00EA1FE32EE337E053
:10F3F000AE01475F5F4FBE016B5F7F4FCE0101964D
:10F400000E9408BC0ADB0E94CAFF8EE89BE10E94B2
:10F4100076F560E085E89BE10E94C5EC8D829E82D6
:10F42000AF82B88649825A826B827C82BE016B5F52
:10F430007F4FCE0101960E9413AC1D8A19821A8259
:10F440001B821C828CE089871D829E012B5E3F4FB0
:10F45000AE014F5F5F4FBE01675F7F4FCE010596E4
:10F460000E945C9960E070E080E792E494D9882380
:10F4700009F10150110969F4ECEAFBE184918F0173
:10F480000F5F1F4F882309F40ECF0F94452EF8010C
:10F49000F5CFE5ECFBE184919F012F5F3F4F88237F
:10F4A00009F4B7CF2A8F3B8F0F94452E2A8D3B8DC1
:10F4B000F901F1CF40903A0750903B0760903C072C
:10F4C00070903D0720910D0730910E0740910F0776
:10F4D00050911007C301B2010F94403C20911E07C8
:10F4E00030911F0740912007509121070F94413C14
:10F4F0005B018C01988D91111CC080E090E0A8E424
:10F50000B2E489839A83AB83BC8320E030E040EA95
:10F5100050E4C301B2010F94413C6D837E838F831D
:10F520009887BE016F5F7F4FCE0105960E9413AC96
:10F5300009C080E00E94C9AB882321F0A12CB12C26
:10F5400000EC1FE78091FC0680932402E98DE330F4
:10F5500008F440C0E2E4FCE184914F019FEF891A76
:10F56000990A882321F00F94452EF401F5CFEE89F6
:10F57000FF89608171818281938143E00F941E2F06
:10F58000EDE3FCE184914F019FEF891A990A8823EA
:10F5900021F00F94452EF401F5CFF10160817181C6
:10F5A0008281938143E00F941E2FE8E3FCE1849174
:10F5B0004F019FEF891A990A882321F00F94452E55
:10F5C000F401F5CF43E0B501C8010F941E2F8AE086
:10F5D0000F94452EC0922502D0922602E092270277
:10F5E000F09228029501A801B501C8010F94ED3EE3
:10F5F0008823F9F060E089E29CE10E94C5ECE2EE2C
:10F60000F1E284917F019FEFE91AF90A882321F042
:10F610000F94452EF701F5CFE9E1FCE184917F01DC
:10F620009FEFE91AF90A882321F00F94452EF7017C
:10F63000F5CFB501C8016B960FB6F894DEBF0FBECB
:10F64000CDBFDF91CF911F910F91FF90EF90DF9091
:10F65000CF90BF90AF909F908F907F906F905F9072
:10F660004F903F902F900895BC0180E090E04AE0D9
:10F670000F949E2E8DE00F94452E8AE00D94452E1A
:10F68000EF92FF920F931F93CF93DF931F92CDB70B
:10F69000DEB78B01622F49830E94036E9091020CAA
:10F6A0008091FA064981891708F43FC09091040CB3
:10F6B0008091F906981708F438C0442399F120E0A6
:10F6C00030E0F801E20FF31FE491EE2319F02F5F11
:10F6D0003F4FF7CF86E190E0821B930B97FD019699
:10F6E0009595879536E1F32E49EEE42EE80E8E2DA2
:10F6F0008F0D87FD0EC080E20E9438D9FA94F7CFB3
:10F70000F8018491882339F00F942E2AF81A0F5F9C
:10F710001F4F1F14ACF31F1444F480E20E9438D929
:10F72000FA94F9CF86E1F82EF4CF0F90DF91CF91C4
:10F730001F910F91FF90EF900895CF92DF92EF927B
:10F74000FF920F931F93CF93DF937C018B016A018C
:10F75000E9010E94196D83E080932D02F092F50675
:10F76000E092F4061093F3060093F2061092EE0670
:10F770001092EF061092F0061092F106A601DD0C31
:10F78000660B770B4093EA065093EB066093EC060A
:10F790007093ED06F80180819181092E000CAA0B6F
:10F7A000BB0B8093E6069093E706A093E806B09320
:10F7B000E90683E79AEE90931F0280931E02D0938E
:10F7C000F806C093F7061092F606DF91CF911F91CD
:10F7D0000F91FF90EF90DF90CF900895CF92DF923E
:10F7E000EF92FF920F931F93CF93DF9300D01F925E
:10F7F000CDB7DEB77C018B01CA01B90129837A83B9
:10F800008B839C830E94196D23E020932D02F0923C
:10F81000F506E092F4061093F3060093F2062AE050
:10F8200037ED43E25CE369817A818B819C810F949F
:10F830003C380F94853D6093EE067093EF068093FD
:10F84000F0069093F1060F94DD376B017C019B016C
:10F85000AC0160E070E887E794E40F94403C0F94BB
:10F86000853D6093EA067093EB068093EC069093D7
:10F87000ED062AE037ED43E25CE3F8016081718137
:10F88000828193810F943C38A70196010F94403CEC
:10F890000F948A3D6093E6067093E7068093E8062E
:10F8A0009093E90689E897EE90931F0280931E02D9
:10F8B0000F900F900F900F90DF91CF911F910F91AC
:10F8C000FF90EF90DF90CF900895EF92FF921F93FB
:10F8D000CF93DF931F92CDB7DEB7182FE8EDFCE191
:10F8E00084917F012FEFE21AF20A882331F0998385
:10F8F0000F94452EF7019981F3CFE12FF92F8491D1
:10F900007F019FEFE91AF90A882321F00F94452E11
:10F91000F701F5CFEFEBFCE184917F012FEFE21AC5
:10F92000F20A882321F00F94452EF701F5CF0F90AE
:10F93000DF91CF911F91FF90EF900895CF92DF92CA
:10F94000EF92FF920F931F93CF9300916604109153
:10F95000670480E50E949DB1882359F00E94F7B0AA
:10F960006B017C01C1E0672B682B692B31F4C0E08F
:10F9700004C0C0E0C12CD12C760183E50E949DB16A
:10F980008823F1F00E9437B120E030E04AE754E4E8
:10F990000F943C380F948A3D6B017C01C11112C059
:10F9A000672B682B692B71F40115110559F0F801CB
:10F9B0008081882339F061E0C8010E94E3EC07C030
:10F9C000CC2391F360E08EEF9EE10E94C5EC81E0D4
:10F9D0008093810F0E94CAFF0E94D75CC114D1049A
:10F9E000E104F104F1F08091B6159091B715A09162
:10F9F000B815B091B915C80ED91EEA1EFB1E0E949B
:10FA0000CB5CDC01CB018C199D09AE09BF09B7FFA6
:10FA10001CC08091810F8823C1F080E00F94E823FF
:10FA2000EECF8091810F882321F080E00F94E823AE
:10FA3000F8CF8091AF0C60E0882319F08FEE9EE143
:10FA400002C085ED9EE10E94C5EC1092810FCF911E
:10FA50001F910F91FF90EF90DF90CF900895CF927C
:10FA6000DF92FF920F931F93CF93DF9385E40E9461
:10FA70009DB1D82F811102C00E94CAFF8AE5C82E0D
:10FA800083E0D82E02E317E0C0E0F12CF60181916B
:10FA90006F010E949DB1882359F00E9437B1F8018F
:10FAA0006083718382839383C33011F0FF24F394C6
:10FAB000CF5F0C5F1F4FC43049F7FF2019F00E9441
:10FAC00017B003C0D1110E940D75DF91CF911F9126
:10FAD0000F91FF90DF90CF900C9421B22F923F9224
:10FAE0004F925F926F927F928F929F92AF92BF924E
:10FAF000CF92DF92EF92FF920F931F93CF93DF93FA
:10FB0000CDB7DEB7DA950FB6F894DEBF0FBECDBF26
:10FB10000E946F7481110C948E8BFE0131968CE3E0
:10FB2000DF011D928A95E9F700915D15C352DF4F01
:10FB30000883CD5DD0408AE40E946EB1882321F015
:10FB40000E9480AA0C948E8B86E50E949DB188232A
:10FB500049F00E9407B1C153DF4F79836883CF5CBE
:10FB6000D04006C0C153DF4F19821882CF5CD0400D
:10FB7000C153DF4F08811981CF5CD040053011059A
:10FB800070F0EDEAFEE184918F010F5F1F4F882333
:10FB900011F40C948E8B0F94452EF801F4CF84E46D
:10FBA0000E946EB1C152DF4F8883CF5DD040882361
:10FBB00039F00E9428B1C152DF4F8883CF5DD04019
:10FBC000C153DF4F08811981CF5CD040033011054C
:10FBD0006CF484E50E946EB1882379F00E9428B10C
:10FBE000C252DF4F8883CE5DD0400CC011E0C252BC
:10FBF000DF4F1883CE5DD04005C0C252DF4F188260
:10FC0000CE5DD04088E50E949DB1882321F00E94FE
:10FC100007B1162F01C012E089E50E949DB188232B
:10FC200021F00E9407B1062F01C002E080E50E948A
:10FC30009DB1811103C0212E302E04C00E9407B156
:10FC4000262E362E21E0221518F0E8E7FEE104C04A
:10FC500031E0331568F0F9CF84918F010F5F1F4FAA
:10FC6000882311F40C948E8B0F94452EF801F4CF59
:10FC700083E50E949DB1882319F00E9437B104C02A
:10FC800060E070E88BEB95E420E030E040E752E480
:10FC90000F941D3D609320027093210280932202F5
:10FCA00090932302C0900507D0900607E0900707C5
:10FCB000F09008078CE40E949DB1811109C020E0FA
:10FCC00030E040E450E4C701B6010F94403C02C06C
:10FCD0000E9437B10F94853D6B017C01CF52DF4FFD
:10FCE00079836883C15DD0408090050790900607B6
:10FCF000A0900707B090080782E50E949DB181118E
:10FD000009C020E030E042E253E4C501B4010F94A1
:10FD1000413C02C00E9437B10F94853D4B015C010C
:10FD2000C154DF4F79836883CF5BD040409009078F
:10FD300050900A0760900B0770900C0786E40E94B1
:10FD40009DB1811109C020E030E040EE50E4C301D4
:10FD5000B2010F94403C02C00E9437B10F94853D20
:10FD6000C554DF4F688379838A839B83CB5BD04004
:10FD7000C554DF4F08811981CB5BD040C752DF4F9C
:10FD800019830883C95DD0404090090750900A0745
:10FD900060900B0770900C0782E40E949DB1811166
:10FDA00009C020E030E044E253E4C301B2010F9403
:10FDB000413C02C00E9437B10F94853DCB52DF4FCA
:10FDC000688379838A839B83C55DD040CB52DF4FA4
:10FDD00008811981C55DD040CD53DF4F1983088359
:10FDE000C35CD040B6010D2C000C880B990B0F940E
:10FDF000DD37CC51DF4F688379838A839B83C45E70
:10FE0000D04040900507509006076090070770901B
:10FE1000080720E030E040E450E4C301B2010F9451
:10FE2000403C9B01AC01CC51DF4F688179818A81D4
:10FE30009B81C45ED0400F94D73711E0C954DF4F87
:10FE40001883C75BD04087FD10C0C4010997CF520B
:10FE5000DF4F08811981C15DD040081719072CF4C4
:10FE6000C954DF4F1882C75BD040B401990C880B8E
:10FE7000990B0F94DD374B015C0120E030E042E24A
:10FE800053E4C301B2010F94413C9B01AC01C50195
:10FE9000B4010F94673E18167CF029E0C20ED11C05
:10FEA00001E0C154DF4F88819981CF5BD040C816F3
:10FEB000D9061CF400E001C001E0C554DF4FA88161
:10FEC000B981CB5BD040BD01BB0F880B990B0F9460
:10FED000DD37C851DF4F688379838A839B83C85E8F
:10FEE000D040C0900907D0900A07E0900B07F0902F
:10FEF0000C0720E030E040EE50E4C701B6010F945B
:10FF0000403C9B01AC01C851DF4F688179818A81F7
:10FF10009B81C85ED0400F94D73711E087FD11C098
:10FF2000CB52DF4F88819981C55DD0400997C75278
:10FF3000DF4FE881F981C95DD040E817F9070CF47B
:10FF400010E0CB52DF4F28813981C55DD040B90127
:10FF5000330F880B990B0F94DD374B015C0120E0C8
:10FF600030E04EE353E4C701B6010F94413C9B01DE
:10FF7000AC01C501B4010F94673E1816A4F0C55436
:10FF8000DF4F88819981CB5BD0400996FF24F394A1
:10FF9000CD53DF4FA881B981C35CD0408A179B073E
:10FFA00024F4F12C02C0FF24F394C954DF4FB8812C
:10FFB000C75BD040B1110BC0002321F089E69EE160
:10FFC00084DC0AC0111108C0F1100BC013C081E716
:10FFD0009EE17BDC0111F2CF112319F081E69EE155
:10FFE00074DCFF2011F40C948E8B8AE59EE16DDCAD
:10FFF0000C948E8BC153DF4F08811981CF5CD040A8
:020000021000EC
:10000000012BF9F0E3E4FEE184918F010F5F1F4FB4
:10001000882321F00F94452EF801F6CFC152DF4F0F
:100020001881CF5DD040112361F0EAE2FEE18491B6
:100030008F010F5F1F4F882321F00F94452EF80189
:10004000F6CF0E94CAFF10925D15C152DF4F0881A2
:10005000CF5DD04001110AC00F94352781E197E0B0
:100060000E94B1C80E94FAF30E9417B081E00E947A
:10007000C9AB882349F0C352DF4F1881CD5DD04012
:1000800010935D150C948E8B0E94C7AA85E40E9484
:100090006EB1582E882319F00E9428B1582E022DD7
:1000A00010E0C351DF4F19830883CD5ED040032D8C
:1000B00010E0C151DF4F19830883CF5ED040239CED
:1000C00080011124CB52DF4F19830883C55DD040D6
:1000D000122D1170C553DF4F1883CB5CD040CB522B
:1000E000DF4F08811981C55DD040000F111F000F3F
:1000F000111FCD50DF4F19830883C35FD040CB520F
:10010000DF4F08811981C55DD04023E0000F111F2A
:100110002A95E1F7CF50DF4F19830883C15FD040A4
:10012000C554DF4F19821882CB5BD04066246A9495
:10013000762CC154DF4F08811981CF5BD040CF525C
:10014000DF4F28813981C15DD040021B130BC154A0
:10015000DF4F19830883CF5BD040CD53DF4F088139
:100160001981C35CD040C752DF4F28813981C95DF6
:10017000D040021B130BCD53DF4F19830883C35CA0
:10018000D040C953DF4F288139814A815B81C75CE8
:10019000D040CA01B9010F94ED3E8111F6C2C5539A
:1001A000DF4F0881CB5CD040002369F0CF52DF4F96
:1001B0003882C15DD04001E0C752DF4F0883C95D7E
:1001C000D040412C0FC044244A94430C1FEFC75227
:1001D000DF4F1883C95DD0400FEFCF52DF4F088348
:1001E000C15DD04081E0C553DF4F1881CB5CD0406A
:1001F0001827C553DF4F1883CB5CD040C30101964D
:10020000880F991F880F991F0DE310E00C0F1D1F19
:10021000080F191FC954DF4F19830883C75BD040EB
:10022000C351DF4F08811981CD5ED04001501109C3
:10023000CB50DF4F19830883C55FD040C554DF4FD3
:1002400088819981CB5BD040092E000CAA0BBB0B97
:10025000C950DF4F88839983AA83BB83C75FD0408F
:10026000C151DF4F08811981CF5ED0400150110983
:10027000C550DF4F19830883CB5FD040C554DF4F93
:1002800008811981CB5BD040000F111FC350DF4F95
:1002900019830883CD5FD040CF52DF4F1881C15DF5
:1002A000D040411609F460C2C154DF4F8881998162
:1002B000CF5BD040CB50DF4F68817981C55FD040A4
:1002C0000F941D3F072E000C880B990B0F94DD3700
:1002D0006B017C01C950DF4F688179818A819B81E4
:1002E000C75FD0400F94DD379B01AC01C701B60159
:1002F0000F943C389B01AC01CC51DF4F6881798170
:100300008A819B81C45ED0400F94413C4B015C01CB
:10031000CD53DF4F88819981C35CD040C550DF4FFA
:1003200068817981CB5FD0400F941D3F072E000C70
:10033000880B990B0F94DD376B017C01642D042C25
:10034000000C770B880B990B0F94DD379B01AC01E8
:10035000C701B6010F943C389B01AC01C851DF4F77
:10036000688179818A819B81C85ED0400F94413C2D
:100370006B017C0120E030E0A901C501B4010F94BC
:10038000D73787FD05C020E030E040E05FE303C0E1
:1003900020E030E0A901C501B4010F94413C0F9465
:1003A000B63DC355DF4F688379838A839B83CD5ADB
:1003B000D04020E030E0A901C701B6010F94D73743
:1003C00087FD05C020E030E040E05FE303C020E0AF
:1003D00030E0A901C701B6010F94413C0F94B63D2E
:1003E000C755DF4F688379838A839B83C95AD0407E
:1003F0001FEF611A710AC350DF4FE881F981CD5FA9
:10040000D040E40DF11D47FCFA95EE0FFF1F21EAE5
:1004100030E02C0F3D1FE20FF31F71826082C15349
:10042000DF4F2881CF5CD040452DBE0167557F4FFF
:10043000CE0183559F4F0E945F77C953DF4F68837A
:1004400079838A839B83C75CD0409B01AC010F9466
:10045000ED3E882341F0C352DF4F0881CD5DD0408F
:1004600000935D1581C1C953DF4F288139814A81CD
:100470005B81C75CD040C052DF4F688179818A813F
:100480009B81C05ED0400F94413CC052DF4F6883D7
:1004900079838A839B83C05ED040F301EE0FFF1FF8
:1004A000EE0FFF1F2DE630E02C0F3D1FE20FF31F74
:1004B000C953DF4F88819981AA81BB81C75CD04035
:1004C00080839183A283B383C355DF4F8880998053
:1004D000AA80BB80CD5AD040C954DF4FA881B981D2
:1004E000C75BD0408D929D92AD92BC921397C75539
:1004F000DF4FC880D980EA80FB80C95AD040FD0117
:10050000CD50DF4F08811981C35FD040E00FF11F4C
:10051000C082D182E282F382FD01CF50DF4F088199
:100520001981C15FD040E00FF11F80E090E0A0E8AA
:10053000BFE380839183A283B383A5019401698182
:100540007A818B819C810F94413C69837A838B8370
:100550009C83A70196016D817E818F8198850F9480
:10056000413C6D837E838F839887C953DF4F2881F9
:1005700039814A815B81C75CD04069857A858B85EA
:100580009C850F94413C69877A878B879C87A5015E
:100590009401C501B4010F943C389B01AC016D85F9
:1005A0007E858F8598890F94413C6D877E878F87E4
:1005B000988BA7019601C701B6010F943C389B01A7
:1005C000AC0169897A898B899C890F94413C698B3C
:1005D0007A8B8B8B9C8BC953DF4F288139814A8161
:1005E0005B81C75CD040CA01B9010F943C389B01C4
:1005F000AC016D897E898F89988D0F94413C6D8BFC
:100600007E8B8F8B988FA7019601C501B4010F9443
:100610003C389B01AC01698D7A8D8B8D9C8D0F943C
:10062000413C698F7A8F8B8F9C8FC953DF4F288114
:1006300039814A815B81C75CD040C501B4010F9408
:100640003C389B01AC016D8D7E8D8F8D98A10F94F0
:10065000413C6D8F7E8F8F8F98A3C953DF4F2881C8
:1006600039814A815B81C75CD040C701B6010F94D4
:100670003C389B01AC0169A17AA18BA19CA10F948C
:10068000413C69A37AA38BA39CA3E894B7F80DA17E
:10069000C352DF4F0883CD5DD0401EA1C451DF4F50
:1006A0001883CC5ED0400FA118A5C352DF4F28811C
:1006B000CD5DD040C451DF4F3881CC5ED040A80121
:1006C000C501B4010F94673E18165CF0C352DF4FAA
:1006D0008880CD5DD040C451DF4F9880CC5ED04043
:1006E00058018DA29EA2AFA2B8A6E894F7F8A9A4DB
:1006F000BAA40BA51CA59501A801C701B6010F94CA
:10070000673E181614F065017801C9A6DAA6EBA6B3
:10071000FCA620E030E040E85FE369AD7AAD8BAD48
:100720009CAD0F94413C69AF7AAF8BAF9CAF80E03A
:100730000F94E823C752DF4F0881C95DD040400EB7
:10074000C954DF4F08811981C75BD0400C5F1F4F30
:10075000C954DF4F19830883C75BD040C352DF4FB2
:100760001882CD5DD04098CDC554DF4F08811981E6
:10077000CB5BD0400F5F1F4FC554DF4F19830883F9
:10078000CB5BD040021508F4FCCC80E00E94C9ABE2
:10079000882341F0C352DF4F1881CD5DD0401093C4
:1007A0005D15B3C7C953DF4F288139814A815B8109
:1007B000C75CD040CA01B9010F94ED3E8111A5C7B5
:1007C00089AC9AACABACBCAC20E030E0A901C5016F
:1007D000B4010F94D737882309F408C2A501940106
:1007E00069817A818B819C810F941D3DC954DF4FB3
:1007F000688379838A839B83C75BD04069837A83CC
:100800008B839C83A50194016D817E818F81988566
:100810000F941D3DC554DF4F688379838A839B8382
:10082000CB5BD0406D837E838F839887A501940135
:1008300069857A858B859C850F941D3DC154DF4F5A
:10084000688379838A839B83CF5BD04069877A876B
:100850008B879C87A50194016D857E858F859889FE
:100860000F941D3D6B017C01C954DF4F28813981F4
:100870004A815B81C75BD040CA01B9010F943C3803
:100880009B01AC01C701B6010F94403CC553DF4F3B
:10089000688379838A839B83CB5CD0406D877E8716
:1008A0008F87988BA501940169897A898B899C89A6
:1008B0000F941D3D6B017C01C554DF4F28813981A8
:1008C0004A815B81CB5BD040CA01B9010F943C38AF
:1008D0009B01AC01C701B6010F94403CCF52DF4FE2
:1008E000688379838A839B83C15DD040698B7A8BCF
:1008F0008B8B9C8BA50194016D897E898F89988D46
:100900000F941D3D6B017C01C154DF4F288139815B
:100910004A815B81CF5BD040CA01B9010F943C385A
:100920009B01AC01C701B6010F94403C6D8B7E8BDF
:100930008F8B988FA5019401698D7A8D8B8D9C8DFD
:100940000F941D3D6B017C01C554DF4F2881398117
:100950004A815B81CB5BD040C954DF4F688179818C
:100960008A819B81C75BD0400F943C389B01AC01CE
:10097000C701B6010F94403CCD53DF4F68837983A4
:100980008A839B83C35CD040698F7A8F8B8F9C8FC7
:10099000A501940169A17AA18BA19CA10F941D3D91
:1009A0006B017C01C154DF4F288139814A815B8111
:1009B000CF5BD040C554DF4F688179818A819B81AC
:1009C000CB5BD0400F943C389B01AC01C701B60112
:1009D0000F94403C6B017C0169A37AA38BA39CA379
:1009E000A50194016D8D7E8D8F8D98A10F941D3D75
:1009F0004B015C01C154DF4F288139814A815B8101
:100A0000CF5BD040C954DF4F688179818A819B8157
:100A1000C75BD0400F943C389B01AC01C501B401C9
:100A20000F94403C4B015C016D8F7E8F8F8F98A39C
:100A3000CF52DF4F288139814A815B81C15DD0402F
:100A4000C553DF4F688179818A819B81CB5CD0401F
:100A50000F943C382B013C01CD53DF4F2881398165
:100A60004A815B81C35CD040CA01B9010F943C3814
:100A70009B01AC01C301B2010F94403CC752DF4F50
:100A8000688379838A839B83C95DD0402B013C01B5
:100A9000E89477F829A53AA54BA55CA56DA17EA1A0
:100AA0008FA198A50F94413C2FEF36EE4BED5EE2FF
:100AB0000F943C389B01AC01C301B2010F94D737AE
:100AC00018160CF093C0CD53DF4F288139814A812D
:100AD0005B81C35CD040C701B6010F943C382B0149
:100AE0003C01CF52DF4F288139814A815B81C15D52
:100AF000D040C501B4010F943C389B01AC01C30147
:100B0000B2010F94403CC752DF4F288139814A819E
:100B10005B81C95DD0400F941D3D2B013C016DA749
:100B20007EA78FA798ABCD53DF4F288139814A81AB
:100B30005B81C35CD040C501B4010F943C384B01CC
:100B40005C01C553DF4F288139814A815B81CB5CD1
:100B5000D040C701B6010F943C389B01AC01C501E0
:100B6000B4010F94403CC752DF4F288139814A813C
:100B70005B81C95DD0400F941D3D6B017C0169AB69
:100B80007AAB8BAB9CABC954DF4F288139814A814A
:100B90005B81C75BD040C301B2010F943C389B011D
:100BA000AC01C154DF4F688179818A819B81CF5B21
:100BB000D0400F94413C4B015C01C554DF4F28816C
:100BC00039814A815B81CB5BD040C701B6010F946C
:100BD0003C389B01AC01C501B4010F94413CDC01E0
:100BE000CB01B0588DAB9EABAFABB8AFCDA4DEA4FC
:100BF000EFA4F8A82601370177FA709477F870947B
:100C000089A89AA8ABA8BCA88DA99EA9AFA9B8AD80
:100C1000C954DF4F88839983AA83BB83C75BD040C5
:100C2000CB52DF4F08811981C55DD040B801110F4B
:100C3000880B990B0F94DD379B01AC01C052DF4F3D
:100C4000688179818A819B81C05ED0400F941D3D6F
:100C5000C553DF4F688379838A839B83CB5CD04005
:100C6000C153DF4F08811981CF5CD040012B09F4BB
:100C700061C0E4E1FEE184918F010F5F1F4F882383
:100C800021F00F94452EF801F6CF48E0C301B201E0
:100C90000F941E2FEFE0FEE184918F010F5F1F4F35
:100CA000882321F00F94452EF801F6CF48E0C501C6
:100CB000B40190580F941E2FEAE0FEE184918F0159
:100CC0000F5F1F4F882321F00F94452EF801F6CFB8
:100CD000C954DF4F688179818A819B81C75BD0408D
:100CE000905848E00F941E2F8AE00F94452EC15370
:100CF000DF4F08811981CF5CD04003301105D4F05B
:100D0000E1EFFDE184918F010F5F1F4F882321F0F8
:100D10000F94452EF801F6CF48E0C553DF4F6881A8
:100D200079818A819B81CB5CD0400F941E2F8AE011
:100D30000F94452EC152DF4F1881CF5DD040111165
:100D4000D1C1CB56DF4FC882D982EA82FB82C55916
:100D5000D040C756DF4F88829982AA82BB82C95988
:100D6000D040C12CD12C60E8E62E6FE3F62EC3569E
:100D7000DF4FC882D982EA82FB82CD59D040CE01B2
:100D80008B569F4F0E9462EBC757DF4FC882D982B4
:100D9000EA82FB82C958D040C357DF4F18821982BC
:100DA0001A821B82CD58D040CF56DF4F48825982DD
:100DB0006A827B82C159D040CE0187579F4F0E94E3
:100DC00062EBCB56DF4F88819981AA81BB81C559DF
:100DD000D040C954DF4F88839983AA83BB83C75B04
:100DE000D040C756DF4F488059806A807B80C95900
:100DF000D040C356DF4F88809980AA80BB80CD59F0
:100E0000D040C757DF4F088119812A813B81C958DB
:100E1000D040C554DF4F088319832A833B83CB5BC3
:100E2000D040C357DF4F88819981AA81BB81CD58BB
:100E3000D040C154DF4F88839983AA83BB83CF5BA3
:100E4000D040CF56DF4FC880D980EA80FB80C1599F
:100E5000D040A7019601C301B2010F943C38CD5395
:100E6000DF4F688379838A839B83C35CD040C154FE
:100E7000DF4F288139814A815B81CF5BD040C5013A
:100E8000B4010F943C389B01AC01CD53DF4F688116
:100E900079818A819B81C35CD0400F94403CC358C8
:100EA000DF4F688379838A839B83CD57D040C554B5
:100EB000DF4F288139814A815B81CB5BD040C501FE
:100EC000B4010F943C384B015C01A7019601C95451
:100ED000DF4F688179818A819B81C75BD0400F9405
:100EE0003C389B01AC01C501B4010F94403CCF5785
:100EF000DF4F688379838A839B83C158D040C15474
:100F0000DF4F288139814A815B81CF5BD040C95452
:100F1000DF4F688179818A819B81C75BD0400F94C4
:100F20003C386B017C01C554DF4F288139814A81EF
:100F30005B81CB5BD040C301B2010F943C389B0175
:100F4000AC01C701B6010F94403CCB57DF4F68831B
:100F500079838A839B83C558D040CE0183589F4FA5
:100F60000E9462EBC757DF4F088119812A813B81BC
:100F7000C958D040C357DF4F488059806A807B8072
:100F8000CD58D040CF56DF4F88809980AA80BB8053
:100F9000C159D040C358DF4F88819981AA81BB8154
:100FA000CD57D040C954DF4F88839983AA83BB8330
:100FB000C75BD040CF57DF4F88819981AA81BB8121
:100FC000C158D040C554DF4F88839983AA83BB831F
:100FD000CB5BD040CB57DF4F88819981AA81BB8101
:100FE000C558D040C154DF4F88839983AA83BB83FF
:100FF000CF5BD040CB56DF4FC880D980EA80FB80E2
:10100000C559D040C756DF4F488159816A817B81DD
:10101000C959D040C356DF4F88819981AA81BB81CD
:10102000CD59D0400093080C1093090C20930A0C62
:1010300030930B0C40920C0C50920D0C60920E0CE5
:1010400070920F0C8092100C9092110CA092120CC6
:10105000B092130CC954DF4F088119812A813B815A
:10106000C75BD0400093140C1093150C2093160C02
:101070003093170CC554DF4F088119812A813B81B9
:10108000CB5BD0400093180C1093190C20931A0CD2
:1010900030931B0CC154DF4F088119812A813B8199
:1010A000CF5BD04000931C0C10931D0C20931E0CA2
:1010B00030931F0CC092200CD092210CE092220C95
:1010C000F092230C4093240C5093250C6093260C33
:1010D0007093270C8093280C9093290CA0932A0CD2
:1010E000B0932B0CC252DF4F1881CE5DD04011233C
:1010F00009F46CC2EEE2FDE184918F010F5F1F4F96
:10110000882321F00F94452EF801F6CFCC24CA9401
:10111000C30CDC2CC554DF4F1882CB5BD04000ECF5
:10112000C154DF4F0883CF5BD04019E7CD53DF4F69
:101130001883C35CD04004E4C252DF4F0883CE5D05
:10114000D0408E010B561F4FCF54DF4F19830883B9
:10115000C15BD0400C501109CD54DF4F1983088377
:10116000C35BD0400C501109CB54DF4F1983088367
:10117000C55BD040D7FC29C10D2D000F110BCF52FC
:10118000DF4F19830883C15DD040C954DF4F1982F6
:101190001882C75BD040312CC954DF4FE881F981F8
:1011A000C75BD040CF52DF4F08811981C15DD0406D
:1011B000E00FF11F21EA30E02C0F3D1FE20FF31F7B
:1011C000008111817801EE0CFF1CEE0CFF1CEDE696
:1011D000F0E0EC0FFD1FEE0DFF1D4080518062809E
:1011E0007380C553DF4F288139814A815B81CB5C95
:1011F000D040C301B2010F94403C4B015C01E1E0DF
:10120000F0E0EC0FFD1FEE0DFF1D84AD95ADA6AD1A
:10121000B7ADCB56DF4F88839983AA83BB83C5596B
:10122000D040CB52DF4FE881F981C55DD040E00F5F
:10123000F11FEE0FFF1FEE0FFF1F81E090E08C0FFC
:101240009D1FE80FF91F84AD95ADA6ADB7ADC7578B
:10125000DF4F88839983AA83BB83C958D040C35882
:10126000DF4F188219821A821B82CD57D040CA5490
:10127000DF4F9881C65BD0409F93CB54DF4FA8814E
:10128000C55BD040AF93CC54DF4FB881C45BD04036
:10129000BF93CD54DF4FE881C35BD040EF93CE5472
:1012A000DF4FF881C25BD040FF93CF54DF4F0881FE
:1012B000C15BD0400F932DB73EB7245231090FB612
:1012C000F8943EBF0FBE2DBFADB7BEB71196E8E094
:1012D000FCE084E201900D928A95E1F70E947DEA9C
:1012E000C358DF4F288139814A815B81CD57D04077
:1012F000C301B2010F94403C7B018C010FB6F894FE
:10130000DEBF0FBECDBF9B01AC01C554DF4F68816E
:10131000CB5BD040C154DF4F7881CF5BD040CD5301
:10132000DF4F8881C35CD040C252DF4F9881CE5DD1
:10133000D0400F94673E1816A4F4C554DF4FE882DE
:10134000CB5BD040C154DF4FF882CF5BD040CD5350
:10135000DF4F0883C35CD040C252DF4F1883CE5D9D
:10136000D04020E030E0A901C501B4010F94673EF0
:1013700087FD0CC0EBE2FDE184918F010F5F1F4FF1
:10138000882339F00F94452EF801F6CF80E20F94B0
:10139000452E45E0C501B4010F941E2F3394C95466
:1013A000DF4F08811981C75BD0400C5F1F4FC954C4
:1013B000DF4F19830883C75BD040321408F4ECCEAA
:1013C0008AE00F94452EDA94D5CE8AE00F94452E0C
:1013D000C153DF4F08811981CF5CD0400430110523
:1013E00009F0F4C0E2E0FDE184918F010F5F1F4F2F
:1013F00081110CC03E0115E9610E711C2E0129E816
:10140000420E511C8E0103581F4F16C00F94452EDB
:10141000F801EACF80E20F94452E45E0C501B40102
:101420000F941E2FD394F4E0EF0EF11CD214A0F011
:101430008AE00F94452ECA94C7FCC4C02C2D220FFD
:10144000330BC153DF4F39832883CF5CD040E12C6D
:10145000F12CD12C84E2382EC153DF4FE881F98181
:10146000CF5CD040EE0DFF1D81EA90E08C0F9D1FF8
:10147000E80FF91F808191815C01AA0CBB1CAA0CAA
:10148000BB1CE1E0F0E0EC0FFD1FEA0DFB1D44ADDD
:1014900055AD66AD77ADD3014D935D936D937C9360
:1014A0001397CB52DF4FE881F981C55DD040E80F3B
:1014B000F91FEE0FFF1FEE0FFF1F21E030E02C0F92
:1014C0003D1FE20FF31F84AD95ADA6ADB7ADF201A0
:1014D00080839183A283B383D8011D921D921D92B4
:1014E0001C9213971F930F935F924F927F926F926C
:1014F000EDB7FEB7B4970FB6F894FEBF0FBEEDBFC1
:10150000ADB7BEB71196E8E0FCE0832D01900D92D7
:101510008A95E1F70E947DEAEDE6F0E0EC0FFD1F11
:10152000EA0DFB1DD8012D913D914D915C9160819B
:101530007181828193810F94403CC554DF4F288193
:10154000CB5BD040C154DF4F3881CF5BD040CD530F
:10155000DF4F4881C35CD040C252DF4F5881CE5D1F
:10156000D0400F94403C4B015C010FB6F894DEBFB5
:101570000FBECDBF20E030E0A9010F94673E87FD8C
:1015800049CFEFEFFCE184919F012F5F3F4F88230C
:1015900009F443CFC150DF4F2883CF5FD040C05004
:1015A000DF4F3883C050D1400F94452EC150DF4FDC
:1015B0002881CF5FD040C050DF4F3881C050D1402C
:1015C000F901E1CF8AE00F94452E08C0C153DF4FE7
:1015D00008811981CF5CD040012B21F080EE9CE185
:1015E0000E94A675C152DF4F1881CF5DD040111106
:1015F00085C08CE0E2E3F7E0DE01A358BF4F019025
:101600000D928A95E1F781E080935D15CE018358B4
:101610009F4F0E94B1C8C355DF4F288139814A814D
:101620005B81CD5AD0406091320770913307809131
:101630003407909135070F94403C6B017C012DEBF2
:1016400037E346E855EB0F94673E87FD4BC02DEB23
:1016500037E346E855E3C701B6010F94D7371816AC
:101660000CF440C0C755DF4F288139814A815B8126
:10167000C95AD0406091360770913707809138077A
:10168000909139070F94403C6B017C012DEB37E3BF
:1016900046E855EB0F94673E87FD24C02DEB37E3FA
:1016A00046E855E3C701B6010F94D7371816D4F0B2
:1016B000C953DF4F288139814A815B81C75CD040A3
:1016C00060913A0770913B0780913C0790913D07EC
:1016D0000F94403CCB57DF4F688379838A839B8389
:1016E000C558D0408CE0FE01E358FF4FA2E3B7E0BD
:1016F00001900D928A95E1F781E005C0C352DF4F5A
:101700008881CD5DD04080935D150E94ADAA0E9476
:1017100021B280915D1581110E9417B0D3950FB64B
:10172000F894DEBF0FBECDBFDF91CF911F910F9117
:10173000FF90EF90DF90CF90BF90AF909F908F90F1
:101740007F906F905F904F903F902F900895DF9221
:10175000EF92FF920F931F93CF93DF93CDB7DEB736
:101760002C970FB6F894DEBF0FBECDBF182F0E9486
:10177000CAFFD0905D1580E00E946BAA0E94C7AAA4
:1017800081E080938E04111119C088E50E946EB12A
:10179000F82E89E50E946EB1082F8AE50E946EB18D
:1017A000E82EF11006C0011113C0882369F0F02E55
:1017B00010C0002369F0F02E182F0BC0FF24F39403
:1017C00001E0EE24E39402C0F82E082F11E001C0DE
:1017D00010E00E941AAC111105C0E11003C0F11015
:1017E00006C033C082E00E9404F41123C1F320E05C
:1017F00030E040E850E460910D0770910E07809151
:101800000F07909110070F94413C60939F0F7093C6
:10181000A00F8093A10F9093A20F20913A073091CF
:101820003B0740913C0750913D070F94673E1816C7
:101830007CF419821A821B821C82BE016F5F7F4F6B
:101840008FE99FE00E9413AC03C00111D0CF0CC000
:10185000111102C0FF20A9F080E00E9404F41123BE
:1018600081F081E00E9404F40E9417B01D821E8264
:101870001F821886112369F080E090E0A2E3B3E4B0
:1018800012C00111EECF0E9417B01D821E821F826E
:101890001886E110F1CF80913A0790913B07A09113
:1018A0003C07B0913D0789839A83AB83BC83BE011B
:1018B0006B5F7F4FCE0101960E9413AC80E090E0F9
:1018C000A0EAB0E489879A87AB87BC8711110BC067
:1018D000011109C0409136075091370760913807D0
:1018E0007091390704C040E050E069E373E44D8330
:1018F0005E836F83788711110BC0F11009C040918E
:10190000320750913307609134077091350704C056
:1019100040E050E060EA70E449835A836B837C8343
:10192000AE01475F5F4FBE016B5F7F4FCE010196F7
:101930000E940FAC80918D0480938E048D2D0E94A7
:101940006BAA0E94ADAA83E080932D020E9421B26F
:101950002C960FB6F894DEBF0FBECDBFDF91CF91AE
:101960001F910F91FF90EF90DF900895CF93DF9339
:10197000CDB7DEB727970FB6F894DEBF0FBECDBF49
:101980000E946F7481113BC080E50E949DB1882345
:1019900019F00E9407B101C060E06F8383E50E94E7
:1019A0009DB1882319F00E9407B101C06CE06E83DD
:1019B00084E50E949DB1882319F00E9407B101C0FF
:1019C00063E06D8382E50E949DB1882319F00E9437
:1019D00037B104C060E070E080ED90E469837A8301
:1019E0008B839C839E012B5F3F4FAE014F5F5F4F08
:1019F000BE016A5F7F4FCE0107960E945C992796D1
:101A00000FB6F894DEBF0FBECDBFDF91CF91089522
:101A1000CF92DF92EF92FF9280E50E949DB18823E2
:101A200029F00E94F7B06B017C0103C0C12CD12CBE
:101A3000760183E50E949DB1882361F00E9437B151
:101A400020E030E04AE754E40F943C380F948A3D9C
:101A50006B017C010E94CAFF80912E02811105C09A
:101A600060E086EB9CE10E94C5EC0E94D75C80910F
:101A7000B6159091B715A091B815B091B915C80ECB
:101A8000D91EEA1EFB1E0E94CB5CDC01CB018C1927
:101A90009D09AE09BF09B7FF04C080E00F94E82399
:101AA000F2CFFF90EF90DF90CF900895BF92CF924A
:101AB000DF92EF92FF920F931F93CF93DF9387E90B
:101AC000E82E8FE0F82E02E317E095E7C92E94E0A8
:101AD000D92ECAE5D3E0BC2E84E0B80E89910E94CD
:101AE0006EB18823D9F00E9437B1F601208121110F
:101AF00004C020917904222331F0F8012081318142
:101B00004281538103C020E030E0A9010F94413CA1
:101B1000F70160837183828393830AC0F801808117
:101B20009181A281B381F70180839183A283B383E2
:101B3000F4E0EF0EF11C0C5F1F4F8FEFC81AD80AAC
:101B4000BC12CCCF86E40E949DB18823C9F00E94CC
:101B500037B120E030E0A9010F94673E181684F4F5
:101B60000E9437B120E030E040E752E40F941D3D81
:101B70006093250270932602809327029093280297
:101B80008091F31683FD2AC06091A30F7091A40F7A
:101B90008091A50F9091A60F20913E0730913F07AD
:101BA0004091400750914107E091AC0CEE23B1F019
:101BB0000F94403C9B01AC0160919E0C70919F0C76
:101BC0008091A00C9091A10C0F94413C60939E0CCD
:101BD00070939F0C8093A00C9093A10CDF91CF91F8
:101BE0001F910F91FF90EF90DF90CF90BF900895DD
:101BF000CF93DF93FC011682862F0F94452EE7E1E9
:101C0000F0E28491EF012196882321F00F94452E74
